:1000000000560020212501007124010081240100F7
:1000100099240100B1240100C9240100000000005E
:10002000000000000000000000000000E1240100CA
:10003000F12401000000000001250100112501004C
:100040005924010000000000000000008D5E000047
:10005000B55D00002D5E0000000000000000000003
:10006000E10601007142000051420000D55E00002F
:10007000000000000000000000000000F55E00002D
:100080002DE9F843054688464FF0A0441C4EDFF8A2
:1000900078901C4F237E002BFCD1A37E2BB94FF010
:1000A00001022274A37E002BFBD072B6735DF3B9FC
:1000B00000F02EF8C0B90122D9F8103043F0040343
:1000C000C9F8103087F83220BFF34F8F00BF30BF20
:1000D00087F83200D9F8103023F00403C9F8103043
:1000E000BFF34F8F62B6D5E700BF30BFFAE70023FA
:1000F0007355B8F1000F00D0C04762B6BDE8F88371
:10010000A41400200000105000ED00E000000000EA
:100110005FF800F029060100FFFFFFFFFFFFFFFF70
:10012000FFFFFFFFFFFFFFFFFFFFFFFFFFFFFFFFDF
:10013000FFFFFFFFFFFFFFFFFFFFFFFFFFFFFFFFCF
:10014000FFFFFFFFFFFFFFFFFFFFFFFFFFFFFFFFBF
:10015000FFFFFFFFFFFFFFFFFFFFFFFFFFFFFFFFAF
:10016000FFFFFFFFFFFFFFFFFFFFFFFFFFFFFFFF9F
:10017000FFFFFFFFFFFFFFFFFFFFFFFFFFFFFFFF8F
:10018000FFFFFFFFFFFFFFFFFFFFFFFFFFFFFFFF7F
:10019000FFFFFFFFFFFFFFFFFFFFFFFFFFFFFFFF6F
:1001A000FFFFFFFFFFFFFFFFFFFFFFFFFFFFFFFF5F
:1001B000FFFFFFFFFFFFFFFFFFFFFFFFFFFFFFFF4F
:1001C000FFFFFFFFFFFFFFFFFFFFFFFFFFFFFFFF3F
:1001D000FFFFFFFFFFFFFFFFFFFFFFFFFFFFFFFF2F
:1001E000FFFFFFFFFFFFFFFFFFFFFFFFFFFFFFFF1F
:1001F000FFFFFFFFFFFFFFFFFFFFFFFFFFFFFFFF0F
:10020000FFFFFFFFFFFFFFFFFFFFFFFFFFFFFFFFFE
:10021000FFFFFFFFFFFFFFFFFFFFFFFFFFFFFFFFEE
:10022000FFFFFFFFFFFFFFFFFFFFFFFFFFFFFFFFDE
:10023000FFFFFFFFFFFFFFFFFFFFFFFFFFFFFFFFCE
:10024000FFFFFFFFFFFFFFFFFFFFFFFFFFFFFFFFBE
:10025000FFFFFFFFFFFFFFFFFFFFFFFFFFFFFFFFAE
:10026000FFFFFFFFFFFFFFFFFFFFFFFFFFFFFFFF9E
:10027000FFFFFFFFFFFFFFFFFFFFFFFFFFFFFFFF8E
:10028000704700BF034613F8012B002AFBD1181A50
:10029000013870470048704754B301002020704770
:1002A0000620704708B512F059F808BD08B512F0DD
:1002B000CFF843690148984708BD00BF5CB301000F
:1002C00010B50C4611461A46012807D010B1022875
:1002D0000BD010BDE0B200F039F8FAE7BDF80830F5
:1002E000C9B2E0B200F06EF8F3E7E0B200F00CF94A
:1002F000EFE700BF044B00229A80DA805A819A818E
:10030000B4221A81704700BF00200020014B1878EA
:10031000704700BF0020002010B40446034B0FCBF1
:1003200084E80F00204610BC704700BF0420002066
:1003300082B0054B9B8A0020DAB262F307001B0AE9
:1003400063F30F2002B070470020002010B5044670
:100350001A4B1B7813F0030F02D010F00C0F15D1BD
:1003600014F0030F1AD113F0080F02D014F0040F89
:100370001CD113F0040F13D014F0080F10D00F4B42
:1003800000229A80DA80B4221A8109E011F0E6FF97
:1003900002690A4B1A61FFF7ADFF01E0FFF7AAFF00
:1003A000064B1C70064800F043F910BD034B0022B9
:1003B0009A80DA80B4221A81F2E700BF0020002080
:1003C00064B3010010B5044600F04CFA042C00D0D0
:1003D00010BD4A4800F07AF9494B1A78042A37D000
:1003E000082A4AD0464B5B89B3F5616F05D3444B6D
:1003F00000215981998901319981414B99894EF6A2
:100400006023994251D03E4BD9884EF660239942E1
:100410004FD03B4B99884EF6602399424DD012F055
:10042000080FD5D000F027FA03689847036898476B
:10043000002846D1324B1B7813F0080FC8D02F4844
:1004400000F07CF9002848D02D4BB4221A81BFE778
:100450002B49CB8801339BB2CB802A49A1FB0301F6
:100460000909C1EB0111A3EB41039BB2002BB9D1E8
:1004700023494B8901334B81B4E721490B89013B67
:100480000B818B8801339BB28B801E49A1FB03013A
:100490004909C1EB0111A3EB81039BB2002BA1D150
:1004A00017494B8901334B819CE7154B00219981FA
:1004B000A9E7134B0021D980ABE7114B00219980AC
:1004C000ADE700F0D8F90368984700F066F8012816
:1004D000B0D10B4BB4221A81ACE7094B1B7813F057
:1004E000080F3FF475AF064B1B89002B7FF470AFEC
:1004F00011F0AEFF036898476AE700BF64B30100DC
:10050000002000208988888808B5032808D8DFE8FB
:1005100000F008020C0FFFF7EDFE074800F088F826
:1005200008BD054800F0A8F8FAE7044B1975F7E78D
:10053000024B5975F4E700BF64B3010000200020AE
:10054000134672B1128882420DD89A8882420CD327
:10055000DA888A420BD3588888428CBF0020012059
:10056000704700207047002070470020704700202F
:10057000704708B5002300F042FD08BD08B500F043
:100580003EFD08BD08B5002100F069FDC0B208BD00
:1005900008B500F064FDC0B208BD08B500F09AFCD3
:1005A00008BD08B500F0AEFC08BD08B500F0C2FCFF
:1005B00008BD08B500F0D6FC08BD08B500F0EAFC9F
:1005C00008BD08B500F0FEFC08BD08B500F06AFCE7
:1005D00008BD08B500F068FD08BD000070B506460E
:1005E000124B1B689BB100242346104D55F8232065
:1005F00032B155F82330984743683046984730B9B0
:100600000134E4B2234655F82420002AEED111F03B
:100610001FFF8368012203210220984711F018FF71
:100620008368012203210420984770BD1C1000201C
:10063000F8B507460F4B1B68BBB1002425460D4E8D
:1006400056F8253053B156F82530984703682BB13A
:1006500056F8253098470368384698470134E4B285
:10066000254656F82430002BEAD13846FFF7B6FF6E
:10067000F8BD00BF1C100020F8B50746124B1B68E0
:10068000F3B100242546104E56F825308BB156F8AC
:100690002530984743683846984750B156F825307A
:1006A0009847C3682BB156F825309847C368384639
:1006B00098470134E4B2254656F82430002BE3D1A4
:1006C0003846FFF78BFFF8BD1C1000202DE9F041E4
:1006D0000746194B1B6863B300242546164E05E0F8
:1006E0000134E4B2254656F8243013B356F82530C9
:1006F000002BF5D056F82530984743683846984780
:100700000028EDD056F82530984790F81480BB6843
:10071000984718EA000FE3D056F8253098478368C9
:10072000002BDDD056F82530984783683846984727
:10073000D6E7BDE8F08100BF1C1000202DE9F04194
:1007400007461C4B1B68002B32D000242646194D4F
:1007500005E00134E4B2264655F824302BB355F8B1
:100760002630002BF5D055F8263098474368384698
:1007700098470028EDD055F82630984790F8148017
:10078000BB68984718EA000FE3D055F82630984721
:100790000369002BDDD055F82630984703693846A9
:1007A00098470028D5D0012000E00020BDE8F08166
:1007B0000020FBE71C10002008B543689847012083
:1007C00008BD704710B586B00446036898470368B3
:1007D000984702461A4903A800F0A2FE9DF815307A
:1007E00013F0020F11D0BDF80C30A3F5C9739BB202
:1007F000B3F58A7F09D8BDF80E30B92B05D99DF81D
:100800001430043BDBB2382B01D906B010BD0023F5
:10081000019302934FF00203012262F387138DF8D4
:10082000043011F015FE436801A8984763689847A3
:1008300090F8603043F0020380F86030E5E700BFD5
:100840001820002008B54FF4B473542252210248F6
:1008500000F051FE08BD00BF18200020004870477E
:1008600078B3010008B5022800D008BD194610462B
:1008700000F0EAFEF9E70148704700BF90B30100BD
:10088000F8B507460E464B68984704460E4DAB88B0
:1008900003EB83025200F432A0F8F220F43003EBB1
:1008A00083030A4A52F82720314600EB4300904761
:1008B000AB8801339BB2AB8094F8F1209A4201D807
:1008C0000022AA80F8BD00BF3420002094B30100AC
:1008D0007047704730B585B0044643689847462353
:1008E00080F8F1300A2380F8F0301B4B1B7813F0AE
:1008F000030F09D0A368984710F0080F21D1A3680F
:10090000984710F0040F1CD1134B1B7813F00C0FF9
:1009100009D0A368984710F0020F17D1A368984731
:1009200010F0010F12D1A36898470B4D2870E368AF
:1009300068469847BDF808306B800023EB8005B00F
:1009400030BD21460220FFF79BFFDDE72146032053
:10095000FFF796FFE7E700BF342000200120704733
:10096000704730B589B004468368984710F0080F87
:1009700004D1A368984710F0040F2AD02368984741
:10098000036898470546FFF708FE20B1214600207E
:10099000FFF776FF04E02846FFF703FE0028F5D1B5
:1009A00063689847B0F86030ABB9134B5D88013588
:1009B000E36804A89847BDF818309D4217D0E36853
:1009C000684698470C4BBDF808205A80DA880132F7
:1009D000DA8009B030BD21460120FFF751FF63687E
:1009E00098470023A0F86030034AD380DDE7214612
:1009F0000420FFF745FFE2E73420002030B58DB03A
:100A000004460D4611F024FDC3680A220021204649
:100A100098472378042262F302032370EB68684648
:100A200098472388BDF8062062F30F132380EB68F4
:100A300004A89847BDF81E306380EB6808A8984763
:100A40000B9BA3800DB030BD30B591B004460D4670
:100A500011F0FEFCC3680A22002120469847237843
:100A6000032262F3020323706B689847238802888D
:100A700062F30B132380104BDB881B09627863F34E
:100A800007126270EB6868469847BDF802306380D1
:100A9000EB6804A89847BDF81030A380EB6808A85D
:100AA0009847BDF82E30E380EB680CA898470F9B61
:100AB000238111B030BD00BF3420002030B58DB08F
:100AC00004460D4611F0C4FCC3680A2200212046EA
:100AD00098472378022262F302032370EB6868468A
:100AE00098472388BDF8062062F30F132380EB6834
:100AF00004A89847BDF81E306380EB6808A89847A3
:100B00000B9BA3800DB030BDF0B589B004460D46F7
:100B10000B689847036898470746EB68684698470C
:100B20003846FFF756FD064611F092FCC3680A22CC
:100B30000021204698472378012262F302032370A4
:100B4000EB6804A898472388BDF8162062F30F13BA
:100B500023806B68984790F8603013F0020F2CD117
:100B60006B68984790F8603013F0040F27D16B68DA
:100B7000984790F8603013F0080F22D16B689847BF
:100B800090F8603003F01003002B14BF06220022FF
:100B9000A37862F30303A370F6B2FB68304698476C
:100BA000638860F30F1363803B6930469847A388DE
:100BB00060F30F13A38009B0F0BD0122E8E704221F
:100BC000E6E70522E4E72DE9F04788B004460D4644
:100BD0000B689847036898470646EB6803A8984750
:100BE000BDF810803046FFF7ECFC074611F030FCF2
:100BF000C3680A2200212046984723786FF3020336
:100C00002370F36938469847012814BF002001205B
:100C1000237860F3C30323702388BDF8122062F3A6
:100C20000F1323804FEA1812A37862F30303A37013
:100C3000237968F303032371F36838469847638880
:100C400060F30F136380336938469847A38860F3D5
:100C50000F13A3802B699847ADF81C00A379C0B28D
:100C600060F30103A371B36938469847A37960F331
:100C70008303A371F3683846984733693846984729
:100C80002B689847036898478146FFF7A2FC804687
:100C90006B689847C388ADF804306B689847038940
:100CA000ADF806306B6898474388BDF804201344BC
:100CB000ADF808306B6898478388BDF80620134468
:100CC000ADF80A305FFA88F8D9F80C3040469847FA
:100CD0008246D9F810304046984701AA014650464E
:100CE000FFF72EFC00283ED14FF4C973ADF8043055
:100CF00040F2F273ADF8063040F2A623ADF80830AA
:100D000040F6AC03ADF80A30D9F80C3040469847AD
:100D10008246D9F810304046984701AA014650460D
:100D2000FFF70EFC003018BF0120A37960F34513D4
:100D3000A3716B68984790F86320237A62F30203EB
:100D400023726B68984790F86220238962F38813B6
:100D50002381F36938469847E38860F38F13E38073
:100D600008B0BDE8F0870120DFE70148704700BF09
:100D7000B0B3010038B543689847C58804894188F5
:100D8000294482882244034B1D805C809980DA804C
:100D900038BD00BF3C20002070B584B00446036815
:100DA0009847036898470246224902A800F0A0FA33
:100DB0009DF80830012B01D004B070BDBDF80A6069
:100DC000BDF80C501C4A29463046FFF7B9FB78BBEA
:100DD00063689847037813F0200FEDD001210023BA
:100DE00001934FF00203012262F3850362F387133C
:100DF0008DF800308DF8011033118DF802302B1171
:100E00008DF8033005F00F0545EA06158DF80450FE
:100E100011F01EFB43686846984700F0ABFA636820
:100E2000984790F8603043F0040380F86030C3E7DF
:100E30000021D4E7442000203C20002008B543686E
:100E40009847037813F0240F14BF012100210248B2
:100E500000F07BFA012008BD4420002030B583B0AB
:100E600005460D4C46230193642300931E23122252
:100E7000022104F1080000F02BFA6B689847C5883E
:100E8000018942882A4483880B4425806180A2809E
:100E9000E38003B030BD00BF3C2000200048704715
:100EA000C8B3010070B506460368984780B10024B6
:100EB000E5B233689847ABB2834207D2B36828469D
:100EC000984701340028F3D0012002E0002000E020
:100ED000002070BD70B506460368984780B10024B5
:100EE000E5B233689847ABB2834207D2F36928462C
:100EF000984701340128F3D1012002E0002000E0EE
:100F0000002070BD70B506460368984780B1002484
:100F1000E5B233689847ABB2834207D2F3692846FB
:100F2000984701340328F3D1012002E0002000E0BB
:100F3000002070BD70B506460368984778B100255B
:100F4000ECB233689847A3B2834206D2F3692046D5
:100F5000984701350128F3D102E0FF2400E0002486
:100F6000204670BD70B506460368984778B10025E5
:100F7000ECB233689847A3B2834206D2F3692046A5
:100F8000984701350328F3D102E0FF2400E0002454
:100F9000204670BD70B506460368984778B10025B5
:100FA000ECB233689847A3B2834206D2F369204675
:100FB000984701350228F3D102E0FF2400E0002425
:100FC000204670BD70B5054603689847A0B100265D
:100FD000F4B22B689847A3B283420BD2EB69204648
:100FE0009847012809D0EB69204698470136032825
:100FF000EED102E0FF2400E00024204670BD2DE980
:10100000F84F82468946154698460026374607E03F
:101010007B1CDBB20AF807404B451ED01F46013649
:10102000F4B22B689847A3B2834216D2EB692046EC
:1010300098470028F3D0EB682046984783462B69F1
:1010400020469847B8F1000FE2D042460146584684
:10105000FFF776FA0028DBD1E1E7BDE8F88F2DE94C
:10106000F843074688460026354602E00135EDB2D2
:101070000136F4B23B689847A3B2834211D2FB68B1
:101080002046984781463B6920469847B8F1000FB3
:10109000ECD0424601464846FFF752FA0028E5D117
:1010A000E6E768B2BDE8F88310B5044603689847E0
:1010B00030B123689847B0FA80F04009404210BD33
:1010C0004FF0FF30FBE70000002303704370838282
:1010D00043820382C3704FF6FF72C2800281837025
:1010E000704770B504460E46154663B1CB6810468E
:1010F0009847E0803369284698472081F36928465D
:101100009847A07270BD4FF6FF73C3800381002320
:101110008372F7E710B50446028A43899A4202D9DE
:101120000123C3730373A27B054B53F8223020467F
:101130009847E38B0133E383003018BF012010BDD3
:101140002C100020437823B10078003018BF012014
:10115000704701207047B0F90230B0F906209B1AA1
:10116000002BB8BF5B428B420CDCB0F90430B0F905
:101170000800181A0028B8BF40428142B4BF0020BE
:101180000120704700207047B0F91C2003889A4264
:1011900007DCB0F91E3040888342CCBF002001201C
:1011A00070470020704710B5044601891030FFF7E2
:1011B000D2FF034628B12046FFF7E6FF031C18BF05
:1011C0000123184610BD38B50446857E012D05D98A
:1011D000AB1EDBB2012B08D9002038BD01230373FD
:1011E0000020A0730323E373F7E7FFF7DCFF08B9E0
:1011F00001232373032D04D0A38B0133A383002089
:10120000EBE70023A373627BA3799A4201D000200D
:10121000E3E7207B40B9054B5B7B012B4FF00003DC
:10122000637318BF0120D8E70020D6E72C100020F8
:1012300038B50446837E012B01D0002038BDFFF76E
:10124000B2FF18B90223E3730123237304F10C05E1
:101250002846FFF777FF60B90123A3830022228489
:10126000637B01336373A37B0133A373054B5A7311
:10127000E3E72846FFF728FFE38A6382238BA382F4
:10128000EAE700BF2C10002010B5837E012B07D1A8
:101290000024847344730D4B1B689847204610BD8F
:1012A000002BFCD1038C01331BB203844288934290
:1012B00007DB00230384037B2BB983734373012073
:1012C000EDE70020EBE70020E9E700BF2C1000204D
:1012D00008B5028043809B1A83808171BDF8083075
:1012E0000381BDF80C3043810C30FFF7EDFE08BDE3
:1012F000F0B585B004460F461546002301930293CE
:10130000ADF80C301046FFF73DF90646012806D926
:10131000002323706380A380204605B0F0BD2A46D9
:101320000A2101A8FFF725F933469DF80420294634
:1013300007F11000FFF7D5FE3846FFF7EBFE7A8A7B
:10134000BB8A20706280A380E6E749B908498279A8
:10135000012303FA02F20B7B23EA02030B737047AB
:10136000034A817901238B40117B0B431373704730
:101370002C100020014B01225A7370472C100020C2
:1013800070B504460E46CB6900209847012801D06D
:10139000012070BD002525806580A580E580258120
:1013A0006581A581E58125746574237E03F0F803CA
:1013B00065F3C3032376F36828469847A081336911
:1013C00028469847E081237C01332374E0E7F8B591
:1013D00004460E46CB680020984707463369002034
:1013E00098470546F3690020984703283FD0A38912
:1013F000FB1A1BB22380B4F902209A42B8BF1A46E6
:1014000016466280B4F904709F42A8BF1F46A780A9
:10141000E089281A00B2E080B4F908208242B8BFFF
:1014200002462281B4F90A108142A8BF01466181B7
:10143000B4F9125001EB050C604552DA491B8842A1
:101440004FDD521B904203DC227E42F002022276E4
:10145000EA1993424ADA7F1BBB4247DD721B934273
:10146000DEBF237E43F0080323760120F8BD00236E
:101470002374B4F90020E38A9A4222DB217E01F032
:101480000801002914BF0020102059428A4206DCBE
:10149000227E12F0040F04BF40F00800C0B2B4F97D
:1014A000062093420FDC237E13F0020F0BD140F095
:1014B0000400C0B29142D9DB237E13F0010F08D0A3
:1014C000D4E70020E1E7914207DB237E13F0010F10
:1014D00003D140F00200C0B2C8E7002808BF0120D5
:1014E000C4E7217E41F001012176AAE7227E42F085
:1014F00004022276B2E741828282C3820023038003
:1015000043808380C380038143818381C3810374CB
:101510004374027E02F0F80263F3C302027670475E
:101520002DE9F04182B006460D461446294B93E85A
:10153000030002AB03E90300D3680020984780460C
:10154000236900209847074623689847E3690020ED
:10155000984730B323689847012822D16369002057
:101560009847AB8A83421CD3A36800209847C0B930
:101570002B7C02AA02EB830353F8083C2146284641
:101580009847A989EA896B7C5C1C6C7431807280F5
:10159000A6F80480F78033727072304602B0BDE85E
:1015A000F08100232B806B80AB80EB802B816B81E3
:1015B000AB81EB812B746B742A7E02F0F80263F32B
:1015C000C3022A7633807380B380F38033720123A1
:1015D0007372E2E7E0B30100014B1888704700BF67
:1015E000682000200A207047024B5B6803EB001064
:1015F000807B704768200020024B5B680001185C0C
:10160000704700BF68200020024B5B6803EB0010AE
:101610004088704768200020024B5B6803EB001095
:101620008088704768200020024B5B6803EB001045
:101630000089704768200020024B5B6803EB0010B4
:101640004078704768200020014B1980586070472F
:101650006820002000487047E8B3010010B5044638
:1016600012F09AFD04F1440104F1140014F02EFA72
:1016700004F1740011F03AFD04F5927011F0DAFBF8
:1016800004F5947014F018F904F59E7012F0AAF89D
:1016900004F5B67014F070FB04F5D27014F012FC6F
:1016A00004F5DA7012F072FD04F22D2000F0D6FB82
:1016B00004F5DD7012F0AAF894F8BA310BB912F003
:1016C000ABF804F5DE7011F0F3FF04F5047014F0CC
:1016D00059F804F5067012F04BFD0022014B1A6018
:1016E00010BD00BF3C10002038B9064A1368013312
:1016F0008B4205DD10600120704700231846014A27
:10170000136070473C10002008B511F003FC14F082
:1017100041F814F0E3FB12F07FF811F0D1FFBDE8BF
:10172000084000F093BB00BF0022014B1A607047D5
:1017300040100020024A136801331360704700BF55
:1017400040100020014B1868704700BF4010002077
:101750002DE9F04F013883B0002801916CDD01289C
:1017600072D04FF000094FF0010C09EB000303EBBE
:10177000D3735B1032F9131032F910404500A142C7
:1017800004DD22F813400C4622F8101032F919102B
:101790004FEA490BA14202EB0B0A04DD22F8194083
:1017A000515332F9191032F913408C4205DD22F8F9
:1017B000131022F80B4032F9134006460BF10201D8
:1017C000555E02EB4C0E22F81350545232F90B5076
:1017D0003EF9028F0CF1010CA845F9DB711E02EBFA
:1017E000410301E00E4601391F4633F90249AC427C
:1017F000F8DC8C4507DCAEF80040A7F800800E4608
:10180000BAF90050E4E7019B22F80B408B423D807F
:1018100018DBE14616DD48450EDD09F1010C844573
:10182000A3D102EB49094000B9F90030115E8B42A7
:10183000C4BFA9F800101352019B32F9130003B082
:10184000BDE8F08FB01EE6E791460220ECE700BF4E
:101850002DE9F04F013800EBD07383B05B10002806
:1018600001936CDD012872D04FF000094FF0010C9C
:1018700009EB000303EBD3735B1031F9132031F94B
:1018800010404500A24204DD21F81340144621F81F
:10189000102031F919204FEA490BA24201EB0B0A43
:1018A00004DD21F819404A5331F9192031F9134068
:1018B000944205DD21F8132021F80B4031F9134043
:1018C00006460BF102028D5E01EB4C0E21F813501F
:1018D0008C5231F90B503EF9028F0CF1010CA845E6
:1018E000F9DB721E01EB420301E01646013A1F4686
:1018F00033F90249AC42F8DC944507DCAEF800400D
:10190000A7F800801646BAF90050E4E7019B21F8D9
:101910000B4093423D8018DBE14616DD48450EDD65
:1019200009F1010C8445A3D101EB49094000B9F943
:1019300000300A5E9342C4BFA9F800200B52019BFD
:1019400031F9130003B0BDE8F08FB01EE6E7894619
:101950000220ECE7831A042B10B413DDDC1EB1F96E
:101960000430002A0B804B8031F9143008DD400030
:10197000A0EB42020A44014421F8023D8A42FBD115
:1019800010BC70475C1E032C08BF9C1EE7E700BF1D
:10199000F0B40446049E0846DDE90551A642DDF890
:1019A0001CC019DD04F10044AF1E013C07EB4607E3
:1019B00005EB44058E1C06E09C42B8BF1C46BD42A8
:1019C00026F8024F08D035F9024F9442F4DD144650
:1019D000BD4226F8024FF6D1F0BC6246FFF7BABF0F
:1019E000F0B400280F46DDE90561DDF81CC014DB0A
:1019F000013006EB40048D1C06E09842B8BF184643
:101A0000B44225F8020F08D034F9020D9042F4DDFB
:101A10001046B44225F8020FF6D13846F0BC6246B3
:101A2000FFF798BF2DE9F043B1F9009002284FEA83
:101A30004918DDE90767C2E90088DDE909CE21DD43
:101A40008C1E5B0176017F01043204EB4000023101
:101A500003E0A84631F9029C0432B1F90050B1F913
:101A6000024006FB05F503FB0454156802310CFB2C
:101A7000054407FB094408FB0E4481424FEAA424B5
:101A80005460E6D1BDE8F0832DE9F041884684B08A
:101A90004C00083404AFBD6B24F00704ADEB040D1B
:101AA000BE690395FD6904AC0195009602947D6BB7
:101AB000FFF76EFF3B6B21460293FB6A0395019390
:101AC000BB6A40460093D7E90823FFF7ABFFBD464A
:101AD000BDE8F0812DE9F041884684B04C0008341F
:101AE00004AFBD6B24F00704ADEB040DBE69039594
:101AF000FD6904AC0195009602947D6BFFF770FFC1
:101B00003B6B21460293FB6A03950193BB6A4046F7
:101B10000093D7E90823FFF785FFBD46BDE8F081B4
:101B20002DE9F04F8FB00AAF7D6D9A461B1A023334
:101B300000F103088B465919FB6B18EB05080446A6
:101B40001646FB6000F0AA804FEA8809002934D1CC
:101B500009F10A0929F00709C7F808D0ADEB090D0A
:101B600008953E6D0DF128090796FE6C1346069602
:101B7000BE6C5A4605967E6C414604963E6C0396B2
:101B8000BE6BCDF80890CDE900A6FFF7A3FF002CAF
:101B90000DDBFE680235013409EB850906EB4404D0
:101BA00059F8043B5B1124F8023DA642F8D1D7F85E
:101BB00008D01437BD46BDE8F08F8B000A3323F000
:101BC0000703C7F804D0ADEB030D08953A6D0AABD7
:101BD0000792FA6C09F10A090692BA6C29F0070912
:101BE00005927A6C04923A6C0392BA6BCDE900A22A
:101BF000BB605A4602933346FFF746FFADEB090D33
:101C00000895396D0DF128090791F96C3346069155
:101C1000B96C5A460591796C20460491396C039150
:101C2000B96BCDF80890CDE900A14146FFF752FF0E
:101C3000631C9A4511DDFE68BA68E91CB31E02EB0D
:101C4000810103EB4A0A06EB440251F8043B5B11A5
:101C500022F8023F5245F8D1FE60002C0DDDFE68EF
:101C6000E91C09EB810106EB440251F8043B5B11CE
:101C700022F8023D9642F8D1FE60BB68023559F861
:101C8000252053F825301344FA689B1122F81430AC
:101C9000D7F804D01437BD46BDE8F08F8B000A3367
:101CA00023F00703E946ADEB030D08953E6D0DF1FA
:101CB00028080796FE6C13460696BE6C5A46059693
:101CC0007E6C04963E6C0396BE6BCDF80880CDE921
:101CD00000A6FFF7D9FE544512DAFA6804F1004471
:101CE000013C0335931E02EB440608EB850803EB29
:101CF0004A0A58F8043B5B1126F8023FB245F8D176
:101D0000CD461437BD46BDE8F08F00BF2DE9F04742
:101D100088B099464FEA430808F1080424F0070404
:101D200008AFADEB040DD7E90D563C6BCDE9065677
:101D3000BD6AFE6A059403953C6A7D6A049608AE06
:101D4000CDE901650094FD6BFFF7EAFEB9F1000FE4
:101D500010DD023CA044A6F1020A34F9023F3AF930
:101D6000022F9B1AAB42CCBF5B1B03EAE3734445D3
:101D70002380F2D1BD46BDE8F08700BF1E232DE9C8
:101D8000F041264E86B00D468046009324493346E6
:101D90006420144600220CF095FE00274FF01F0C23
:101DA000012204211F482B46CDF814C00091039056
:101DB000114664200496CDE901770CF03BFE4FF00C
:101DC000240C0120184AA5EB080149090090039250
:101DD0000496CDE901774346CDF814C02022642053
:101DE0000CF028FE294651F8043BA342FBD02B27D8
:101DF00000220124C5F11F030C481944CDE901223A
:101E00000390049649092B460597009420226420EC
:101E10000CF010FE06B0BDE8F08100BF586D010067
:101E2000646D0100786D0100846D01009C6D0100FE
:101E30000B68934209D070B50D46144606462246FB
:101E400029463046FFF79AFFF9E770470022024B18
:101E5000C3E900221A817047C01000200278014BAC
:101E60001A707047BC100020314B1B78002B5AD0E1
:101E70002DE9F04F16462F4A87B089468046002448
:101E80002D4F1368DFF8B4B0DFF8B4A0013E14E0C2
:101E90003D5D38F91410022D2BF8101005F1010EDC
:101EA00039F914109CBF5FFA8EF53D55032D2AF8C1
:101EB000101017D001340A2C0CD04FEA440C0CEB54
:101EC0000401C81816F8011F0029E1D13955013461
:101ED0000A2CF2D10133022BC8BF0023136007B0D4
:101EE000BDE8F08F0CEB04035B000BEB030108680B
:101EF000534402901868B1F804C09B88049002A96A
:101F000028460192ADF81430ADF80CC0FFF7A0FCE4
:101F100004A928F814002846FFF79AFC019A29F82A
:101F200014001368C6E7044AC2E9003313817047FE
:101F3000BC100020CC100020C01000204410002055
:101F40008010002092F83230002B43D1F0B50028E9
:101F50008BB00E460546144610DD936A42189A422D
:101F600010DB00231A4684F8313094F82430934271
:101F70009CBF012384F830300BB0F0BDF1D1D36A9F
:101F80008B42EEDD2B2294F83130134F013384F86D
:101F9000313012493B460092642000220CF092FD41
:101FA0004FF0310C0020012104220D4B049794F8CE
:101FB0003170CDE90110009203930322CDF814C0D3
:101FC00007AB6420CDE9086507970CF033FD94F862
:101FD0003120CAE7704700BFB06D0100C46D010039
:101FE000EC6D010070B19A4215DC0F4A1368C72BE3
:101FF00001DC013313600D4B187808B181F001004A
:1020000019707047084B1A68C72AF4DD1860074B2F
:102010000120197070470022034B1A60034B187897
:102020000028EDD0EAE700BFD8100020DC10002027
:10203000002832DDF0B400260439B20002F18042FB
:1020400092F8807292F88152FFB292F8824267F35E
:102050000703EDB292F8832265F30F23E4B264F331
:102060001743D2B2013662F31F6317B1013F67F322
:1020700007031E2D9CBF013565F30F2314B1013CEE
:1020800064F317430D2A9CBF013262F31F63B04211
:1020900041F8043FD1D1F0BC704770472DE9F04FB3
:1020A000C24CADF20C4D20AF0B932378CDE9091251
:1020B000DDF848443C22002138460C9314F061FDC1
:1020C00078220021A8A814F05CFDA8A92046FFF7FB
:1020D000AFFF20210F22DDF840348AAE0593DDF8F2
:1020E0004434CDE902210493A8AB00934EA93B46AA
:1020F000DDF848046CAA019610F050FD231C18BFAF
:102100000123DDF848140E93002940F39A833B46DF
:10211000002007EB410133F9022B02B101308B4261
:10212000F9D11090012340F2E31200240093DFF86C
:1021300094B29F4B059203932022DDF844340F2183
:102140006C20CDE90144CDF810B00CF073FC2022D6
:102150000F23DDF84014CDE902320591DDF8441477
:10216000DDF848040491A8A9009101963B466CAAA9
:102170004EA912F053FADDF84804A04208DD3B46B0
:1021800007EB400133F9022B02B101348B42F9D144
:102190000F9420250F24DDF840346CAA0593DDF858
:1021A00044344EA90493A8AB009301963B46CDE975
:1021B000024512F073FBDDF840344EA90593DDF8BB
:1021C0004434DDF848040493A8AB0093CDE90245FC
:1021D00001963B466CAA12F0B9F9DDF848140029C3
:1021E00040F332833B46002007EB410133F9022BD9
:1021F00002B101308B42F9D11190002440F2172234
:1022000001236B490592039100932022DDF84434A9
:102210000F216C20CDF810B0CDE901440CF00AFC80
:1022200021467822C6A814F0ACFC21467822E4A806
:1022300014F0A7FC20220F235E49E4AD0968DDF805
:1022400048044978CDE903320791C6A90091DDF829
:1022500040143B460691DDF8441401950591A8A968
:1022600002916CAA4EA913F057FCDDF848340DF129
:10227000BC08A34210DDC2460DF54679E4AD55F821
:10228000041B59F8040B14F063FADDF848340134E8
:10229000A3422AF8020BF2DC0F212024DDF84004CF
:1022A000DDF87424B2F924200690DDF84404CDE969
:1022B00003140590A8A8CDE90080079218466CAADF
:1022C0003B464EA9029612F075FC3B466CAA4EA9FD
:1022D000DDF8480410F044FFDDF848146CAB4EAA5A
:1022E0000020009710F0ACFD0120DDF848140097A5
:1022F000E4ABC6AA10F0A4FDDDF8480400280CDD0C
:102300004246662408EB4001B2F9003004FB03F3B7
:102310009B1222F8023B8A42F6D10026A8AB029318
:10232000DDF838346CAACDE900834EA93B4613F0A2
:10233000D7FADDF848343EACB34226605ADDDFF808
:1023400084904FF418724B4600921B490022702073
:102350000CF0B8FB012540F26122042317490592D5
:10236000CDE902612A462946009370202346CDF824
:1023700010B001950CF05EFB4FF0020A40F26220B3
:1023800023680F4A2946CDE9026205902A4608EBE8
:10239000430370200195CDF810B0CDF800A00CF0EB
:1023A00049FB40F2632023680EE000BFAE15002019
:1023B000A4850100D80C0020FC6D0100146E010002
:1023C000186E0100B06D01008E4A0590CDE90262E1
:1023D00007EB43032A46CDE900A5CDF810B0294606
:1023E00070200CF027FB2368DDF848242B4493422F
:1023F0002360A6DB012240F2652100250420824BE8
:10240000CDE904B1CDE901251146009003936D207B
:102410000DF589630CF00EFBDDF890340B9E0693EE
:10242000DDF834346CAA0593DDF83034DDF8480467
:1024300004930A9B03960293099B4EA9CDE900835E
:102440003B4614F055F8DDF84824AA422BDDDDF8B0
:102450003034B71EA3F10208DDF8343440F271299C
:10246000AA465E1E01E0AA421DDD38F9023F37F997
:10247000021F636016F8013F2560A1600135002B43
:10248000F1D001210423614ACDE90031CDE902A256
:10249000CDE904B90322234641200CF0CBFADDF844
:1024A0004824AA42E1DC0A9E099DDDF83424314625
:1024B000284614F097F8824612F032FFDDF83424F3
:1024C00031462846FFF7D0FC0C9B022B00F07881A8
:1024D0004F4B1F78002F40F07381AB1E0D93DDF83A
:1024E0003484B31EDFF830910C9316AD15AECDF8E1
:1024F00048A00D9B0C9933F9022F59F827000D9332
:1025000031F9023F09280C9114922A60336023604C
:102510004FEA870ACDF84C8098F8001040F37E818E
:1025200014AB00223846009611F0D6F859F80A107C
:102530002268149BC1F10A0C02FB0CFE03FB01F0A4
:1025400032682B6802FB01E203FB0C03314808F1FF
:10255000010880FB02CE80FB030CDB17C3EBAC0C45
:102560000D9B18F8010CD217A3F800C00C9BC2EB0E
:10257000AE021A80002800F04681129B022B40F325
:102580004281092902DC013149F80A10002F00F0CC
:1025900043810226099BDDF848A003EB06080A9B4D
:1025A0009F19DDF8343403F1010938F9020F37F9C6
:1025B00002CF19F8011F2B46009400222860C4F8AE
:1025C00000C0304611F088F801362A6823680A2EC8
:1025D000A8F800203B80E8D1BAF1000F40F3D28088
:1025E000002628220021284614F0CBFADDF84824E2
:1025F0002660B24257DDCDF830A03346DDF834A472
:10260000A94610E0246E0100306E01003C6E01000E
:102610004115002067666666E010002023680133DC
:10262000934223603BDA1AF80330002BF6D040F2D5
:10263000D723012700254FF00408CDE904B3844BCC
:102640003A46CDE90253394623466D200197CDF82D
:1026500000800CF0EFF94FF436702368CDE9015596
:102660007C4D0590A8A800EB8303424639466D20B7
:102670000097CDF810B003950CF0DCF92368A8A9F9
:1026800051F82310DDF83C04DDF8482440F823100D
:102690000133934249F8261023603E44C3DB4D4684
:1026A000DDF830A0F6B24FF4387200274FF0010881
:1026B0009DF83C00684BCDE904B29DF840209DF8A0
:1026C00044C0CDE90177414603938DF8542015AB02
:1026D00004228DF85500CDF800806D208DF856C08D
:1026E0008DF857A00CF0A6F940F2E1205B4ACDE945
:1026F0000177DDF874344146059003926D209A22EB
:10270000CDF80080CDF810B00CF094F940F2E32140
:102710000222534BCDE90187CDE904B10092039326
:102720002022DDF840340F216D200CF083F94FF4A6
:1027300039724C4BCDE9017703930592DDF84434AF
:1027400020220F216D20CDF80080CDF810B00CF0C4
:1027500071F939463E220DF1FA0014F012FA82277F
:1027600042F20F0E4FF0200CDDF840343246009359
:1027700021462B460320A4F800E084F802C06771CC
:1027800012F042FFDDE90A52099CDDF83434294693
:1027900000932046DDF8303410F0FCFBDDF83434D3
:1027A0002A4621460A2010F081FB2046DDF8342419
:1027B000294613F00FF80E980DF20C4DBDE8F08F7E
:1027C0000026099B16ADA3F102080A9B9F1EDDF8A7
:1027D000343403F1FF3938F9020F37F902CF19F811
:1027E000011F2B46009400222860C4F800C0304628
:1027F00010F072FF01362A6823680A2EA8F800201C
:102800003B80E8D1E8E6129B002B7FF4BFAE49F88D
:102810000A30002F7FF4BDAE01276AE623462A4620
:10282000384611F003F898F8001000287FF478AECD
:10283000024600942B46384610F04EFF98F80010E0
:102840006EE6002310936DE400231193D5E400BFDE
:102850004C6E0100506E01006C6E0100706E010044
:1028600070790100A485010080222DE9F047C0B0F5
:102870000DEB02040021064668464B9F4A9D14F06A
:1028800080F920468022002114F07BF94FF0000EE1
:10289000DDF820C1023F0CF10F08394600230CE09F
:1028A0005DF823009CF800905044B9F11F0F4DF8DB
:1028B00023004BD00133202B12D031F9022F12F11B
:1028C0000A0F02F1050AA2F10509E9DB0A2AF1DD86
:1028D00054F823204A4444F823200133202BECD120
:1028E0000CF1010CC44507F14007D6D14FF00008A8
:1028F0004FF000406FF00044DFF898901FABADF14F
:1029000004050DF1FC0C53F8042F55F8041F571E55
:10291000622F06D811F1140F03DACE45A8BF08F1D3
:1029200001088C42A8BF0C469042B8BF10469C4597
:10293000E9D1B8F1020F02DD14F5FA7F0ADC0023B9
:102940001846124A136040B0BDE8F087002DC8BF9A
:102950009644AFE7B6F92430EF2BF0DCB6F9263019
:102960009533ECDBB0F5C87FE9DD084A4C99136874
:102970008B4203DA013313600120E4E701230021D5
:10298000034C184623701160DDE700BFD010002013
:102990004115002031F8FFFF10B4B0F92440C3689E
:1029A000132C00DC8BB30024B1F90C00132803DCDA
:1029B000B1F90E00133023DA0021B2F90C0013280C
:1029C00011DCB2F90E0013300DDB12685AB954B1A4
:1029D00049B1134A1368132B0EDD0023114913600C
:1029E0000B7010BC704742F210729342F1DC00226F
:1029F0000B4B10BC1A6070470133136010BC70475A
:102A00000968B1FA81F14909D7E7B0F926401334D2
:102A100004DB4468B4FA84F46409C5E71C46C3E7E0
:102A2000D41000204115002000281DDD2DE9F041C3
:102A30000027DDF818C04FEA410802EB000E00291C
:102A40000CDD6446581E461810F8015F0DB115786C
:102A500005B92780B04204F10204F5D10132724574
:102A6000C444ECD1BDE8F081704700BF2DE9F04FC0
:102A7000C7B2C0F3072883B0474501900C992BDCFF
:102A80009DF806A052000AF100499DF807B009F12F
:102A9000FF390AFB023301EB490901EB4B0C0D999D
:102AA00008F1010801EB470EDA4518D849461C46E3
:102AB0000C4D34F9170031F9026F8542B8BF054655
:102AC0008642B8BF08808C451444F2D12DB201373C
:102AD00047452EF8025BE7D103B0BDE8F08F014D0A
:102AE000F5E700BF0080FFFF2DE9F04F06468DB0EF
:102AF0004FEA410A184608AF88461446002152465C
:102B000075003B60D7F83C9014F03BF82A46B86B50
:102B1000002114F036F8002E63DDBE6B0AF10803C5
:102B2000721923F0070B4FEAA803023C7A60BB60DE
:102B3000C7F80CD0ADEB0B0D08ABA51C1846294609
:102B4000524614F013F8B96802464046FEF700FEFC
:102B5000B8F1000F014648DD00202246034632F955
:102B600002CF8C4508BF184601339845F7D105229E
:102B7000ADEB0B0D152340F23E6C4FF0290E079282
:102B80006FF42472009508ADCDE901530692CDE9AA
:102B900003E3A1F11E02CDF814C03C314346FEF719
:102BA000BFFF3A68023D0AEB040134F9023F35F9F0
:102BB000020F1B1AA3EB0903002B238006DD1088EC
:102BC0009BB2184410803088034433808C4202F159
:102BD0000202EAD17B6802369E42D7F80CD00C463E
:102BE000A6D11437BD46BDE8F08F6FF424724FF0C4
:102BF000050E152340F23E6C2920ADEB0B0DCDE9FF
:102C0000062E08AA0390019204930293A1F11E02DA
:102C100000953C31CDF814C043460020FEF780FFFC
:102C200004EB0A01D6E700BF2DE9F04F87B08A0018
:102C300000AF3A61083222F00702ADEB020DFB60F3
:102C40006B464D0000297B613D6040F3C980AC1E9E
:102C50007C606C467A6CFE6C023A02EB05087D687B
:102C6000A6F1020B023B65199E46DC464FF4004A72
:102C700047F6FF790026144624F8026F444525F8EC
:102C800002AF2CF8026F2EF8029FF5D100283DDD2F
:102C90004FF0000AFA683B6CA2F1040B3A69043B5E
:102CA00003EB0209BB607A687B691344FB6000296F
:102CB0001DDDD7E9025CDE46FB6C9C1E7B699E1E17
:102CC00055F8048F5EF8043F3CF9022FC3EBA813BC
:102CD0009A42B8BFACF8003036F9022F9A4234F865
:102CE000022FC8BF338013444D452380E8D10AF139
:102CF000010A3B6950459B44D9D100296CDDFB6C2E
:102D00007A6CA3F1020B7B69023A023B9E46BC6CD3
:102D10007D68A61E3C6806EB04087C6904EB050C84
:102D20003CF8024F3EF8025F641B26F8024F3BF965
:102D3000024FB04594FBF0F4ABF80040F0D11446DC
:102D400078697D68461933F9020F34F9025F00286B
:102D5000B8BF4042854200DA20809E42F3D17C68B1
:102D60007B69234418463B68144613441E4630F9D9
:102D7000023F34F9025F002BB8BF5B429D42B8BFEF
:102D80002380A642F3D16FF000443B6DA446581E49
:102D90000144034604E0AC42A8BF2C4699420AD045
:102DA00013F8016F32F9025FF607F4D4AC45A8BFFF
:102DB000AC469942F4D17A6C10F8015F118815F095
:102DC000010FA1EB04050ABFA1EB0C0115801180D6
:102DD000984202F10202EFD11C37BD46BDE8F08FE8
:102DE0000028F9DD3B68023B7B6051E72DE9F04F9D
:102DF0009FB08A0008AF7A61083222F00702ADEB7B
:102E0000020DB8614E0008A800297963B860FE6120
:102E100019DD4FF4004E47F6FF7C0025B11ED7F8B0
:102E200084200144D7F88C00023A96190DF11E0453
:102E3000023822F8025FB24221F802EF20F8025F66
:102E400024F802CFF5D1B969786B4A0000FB02F291
:102E5000083222F00702ADEB020D08AA00297A60C1
:102E600040F3E3807A6400223A6300EBD07222F0F0
:102E70000102043B0A32D7F88010BB6322F007033B
:102E80003B617B690439CB18F9603B653B69C7F846
:102E90002CD0ADEB030D08AAADEB030D08ABBB6462
:102EA0007B6BFA64002B40F33981D7F89020002324
:102EB000013A144647F6FF797A629046D7F88C209B
:102EC0009A46951E7A6CC7E90F33CB46FE68D7F851
:102ED00038E0A2F1020C3C620BE0FC6C4A4524F89D
:102EE000130002DA01468146FB633A6D01339642D4
:102EF00021D056F8040F5EF8042F35F8021FC2EBFC
:102F0000A0121144298018F8014F10B2E4072CF8E0
:102F1000020F4946C7F854B0DFD4BC6C5A4524F8B8
:102F20001A0003DA83467865C7F840A03A6D0AF1C3
:102F3000010A9642DDD1C7F828A015254FF0000BF5
:102F400005266FF4247840F23E694FF0290AFA6CA6
:102F50003C6A0092F86B6431CDE9066B0395CDE9CC
:102F6000015A4FF00042CDE90498FEF7CFFECDE9BB
:102F700002A5CDE9066BCDE904980195BE6C4FF032
:102F800000420096796DBB6A6431386CFEF7BEFE74
:102F9000796B7B6AFD6C0B44594618467B6C14F8C0
:102FA000012F0233D2074BBF35F81B2036F8112012
:102FB0000BF1010B0131844223F8022CEFD17A6C22
:102FC000F9693B6B0A447A647969BA6B01330A4444
:102FD000BA63BA693B639A42D7F82CD07FF456AFF4
:102FE000D7E90C897A68FB69A2F1020CBA6800265D
:102FF0009E4692469D1E1544B9F1000F11DD2946EB
:103000006046AAF1020230F9023F31F9024F9C42B8
:10301000B8BF0B8032F9024F9C42C8BF1380AA424E
:10302000F1D101364645F444E6D17B6B002B71DDCE
:10303000BB68D7F888109C1E2646FA69881ED7F808
:103040008C10A2F1020CD7F81880023903EB0C05A2
:1030500000EB020E35F8023F36F8022F9B1A20F8DB
:10306000023F31F9023F704593FBF8F30B80F1D139
:10307000D7F88430991E0A46BB6803EB0C0534F977
:10308000023F32F9020F002BB8BF5B42984200DAD0
:103090001380A542F3D1BB68084663449C46FB6994
:1030A0000B441A463CF9023F30F9024F002BB8BFDF
:1030B0005B429C42B8BF03809042F3D16FF0004462
:1030C000D7F890302646581E7B6B03449C46034637
:1030D00004E09442A8BF14469C450AD013F8015F4F
:1030E00031F9022FED07F4D49642A8BF16469C454D
:1030F000F4D1D7F8842010F8015F118815F0010F82
:10310000A1EB04050ABF891B15801180834202F1DF
:103110000202F0D15C37BD46BDE8F08F00241525D2
:1031200005266FF4247840F23E694FF0290AFB6CC3
:103130002046009307942346CDE90586CDE903593F
:10314000CDE9015A4FF0004248F26301FEF7DEFD7F
:10315000CDE90664CDE90498CDE902A50195BB6CE3
:10316000204600934FF00042234648F26301FEF7E9
:10317000CDFD24E710B4041E4FF000000ADD023933
:1031800001EB440431F9023F9342C4BF9B1AC018BB
:10319000A142F7D110BC7047002824DDF0B400250F
:1031A0008E1EAC464FF0FF3700E01D4636F9024F49
:1031B0006B1C944203DD6445C4BFA4462F4698426D
:1031C000F3D17B1C11D07B0031F917001FB1CA1855
:1031D00032F9022C1044AF4203DA1944B1F902303B
:1031E0001844F0BC7047002070470020F0BC7047C6
:1031F00070B40024061E1C6020460EDD023901EB6F
:10320000460631F9024F944202DD1D6801351D600A
:10321000A042B8BF2046B142F3D170BC704700BF96
:10322000F0B500258BB00228CDE90632DDE9107437
:10323000CDE9085518DDAE46AC462E460B1F03EB14
:10324000400031F9023FDA1B002AC4BF4FF0010CE5
:10325000B6181B1B44BF01259E448142F1D1BCF12D
:10326000000F4FD1002D4AD10124002604256822E9
:10327000254F264B059221462246CDE9033764208F
:1032800008ABCDE9014600950BF0D4FB6920204B3B
:103290002246214605900393642007AB0497CDE9AD
:1032A000014600950BF0C6FB6A201A4B22462146C8
:1032B00005900393642009AB0497CDE9014600957E
:1032C0000BF0B8FB6B20144B224605900393049738
:1032D00006ABCDE901460095214664200BF0AAFB20
:1032E000DDE907329A4207DC0998069CA042ACBF90
:1032F000002001200BB0F0BD20460BB0F0BDCDF892
:1033000024E0B1E70896ADE730710100407101009B
:103310004871010058710100607101002DE9F04F02
:10332000064689B000AFB86088461546B86C720092
:103330000021BC6D99463B6113F023FC002206EB93
:10334000D67323F001030A3323F00703ADEB030D1B
:10335000C7F818D09642ADEB030DC7F814D0226021
:103360006260A260E260226140F3C5803046FE6C7C
:103370009346721E164647F6FF7E7A6092462A1FD3
:1033800002EB8000F860B86CCC467146A8F10408E6
:10339000A0F102093E60C7F81CB0BC650FE07345A0
:1033A000A8BF7346BC690CF1010C24F81B00A8BF30
:1033B00018468646F8680BF1010B904233D0386905
:1033C00052F8043F20B19CF8000000FB0333DB11EE
:1033D00058F8040F3E6DC3EBA01347F6FF7083420D
:1033E000A8BF034646480D468342B8BF034618B2FD
:1033F00029F8020F1AF8014F3457002CCFD18B4215
:10340000A8BF0B46FD697C690CF1010C24F815007E
:10341000A8BF18460146F8691D460130F861F868F2
:1034200073469042CBD1D7E916429342A8BF1346C8
:1034300095421BB2A8BF154652429342B8BF1346ED
:103440002DB29542FB612B46B8BF13464FF0000CDE
:103450003B61D7E901310B449A467B6D3E68BA6CFB
:10346000E146D3E9008E6FF000454FF000402AE0BE
:10347000BB69F96933F8193009F101095B1A1BB20C
:103480001380434509DD2389216801332381B2F983
:103490000030A3EB080B594421609E4509DD638988
:1034A000616801336381B2F90030A3EB0E0B59441C
:1034B00061609842B8BF18469D42A8BF1D46B245FC
:1034C00002F102020FD016F8013F396DCB56002BE6
:1034D000CED17B69396933F81C300CF1010C5B1AD1
:1034E0001BB21380CDE72DB202B22437A281E58151
:1034F000BD46BDE8F08F4FF0FF354FF00040F4E7D8
:103500000080FFFF2DE9F04786B08246DDE9129882
:1035100016461C460D46149F0AF070FF1423159A98
:103520000397CDE90423D0F801300F9815333246C4
:103530002946CDE9010300940E9B5046FFF7EEFEAD
:1035400000254FF02D0C012102271848184E234664
:10355000CDE9030652466920CDF814C0CDE9011526
:1035600000970BF067FAAA4528460FDDA31E03EB70
:103570004A0A33F9021FA1EB0902002AC8BFAD189D
:10358000B1EB080148BF40185345F2D1109BAB4244
:1035900007DB119B8342D4BF0020012006B0BDE8A9
:1035A000F087012006B0BDE8F08700BF7079010008
:1035B00030710100002820DDF0B48E1E06EB4006BD
:1035C000B14218D0571C38460B46B1F9004033F9C8
:1035D000025FAC4207DD0D801C8092F9004090F93B
:1035E000005015700470B34200F10100EDD10231BA
:1035F000B1423A46E6D1F0BC704770472DE9F04F32
:103600008046450005F1080485B000EBD07A24F02F
:10361000070407302AF0010A00AF20F00700ADEBE5
:10362000040D08F1090424F00704EB46ADEB000D8E
:103630000AF10A0020F007006E46ADEB040D6C465F
:10364000ADEB000DE946C7E902210AF1020A08F1D3
:1036500002021F2120467B6013F093FA524648462F
:10366000002113F08EFAB8F1000F7B6807DD3246B7
:1036700006EB0800911B02F8011B8242FAD14FF0C1
:10368000FF3A2A46F96858467B6013F06FFA5946AC
:1036900032464046FFF78EFF023D08F1FF3E7B6851
:1036A00006EB0E01AB44013EB14218D03BF9025982
:1036B00011F901299D4202F1010C10DBA05C2244AA
:1036C0001F28927860D01E2860D81E2A96BF4FF01F
:1036D000FF3204F80C0004F80C20B142E6D1B8F136
:1036E000020F04F1010113DD0B46FF20A64402E0A6
:1036F000013373450CD05A781F2AF9D11A781E2A43
:10370000F6D89A7801331E2A98BF18707345F2D103
:10371000B8F1000F2EDDFB6804EB0806F96004E049
:103720000134A64203F1020323D06278FF2AF7D1C5
:10373000257894F802C039F8150039F81CE0834662
:10374000704528BFF346B3F90020B96B0A4493458E
:10375000E6DA704538BF7046013465458CBF29F8FC
:103760001C0029F81500A6420AF1FF3A03F10203F2
:10377000DBD1F9684246B86813F0F8F90AF10100A4
:103780001437BD46BDE8F08F1F2A06D01E2A88BF19
:103790006FF0690204F80C2086E70AF1010A04F8C8
:1037A0000CA029F81A507FE710B4DDE90134019428
:1037B00010BCFFF723BF00BF38B500240A4A0B48EE
:1037C0000B4B0C4D2146146004704FF420720A48D4
:1037D0002C601C6013F0D5F92146BDE838404FF449
:1037E0009672064813F0CDB9F4100020F0100020B6
:1037F000E8100020EC100020F810002078130020C2
:103800002DE9F04FADB006AFF962011EC7E9022302
:10381000D7F8E880796340F39783BB4BBB4A1C68B9
:10382000BB61D7F8C0304900023B02EB84127961DA
:10383000023A581833F9021F834222F8021FF9D1C5
:10384000FB6A002B16DD0023B14AC4EB0414D7F841
:10385000C41002EB4402FC6A023A023931F9020F49
:1038600001339C4222F8020FF8DC00207B6B83427C
:1038700040F374834FF0000B47F6FF755846DE4661
:103880005E46D7F8E030A14CD3F800C0DFF8849250
:10389000D7F8C0A0C7F828B0C7F830B02246002338
:1038A00004F5207B32F9401B93450B44FAD189FB88
:1038B0000312DB17C3EBA2031BB2002BC8BF9E444D
:1038C0009E42B8BF1E469D42A8BF1D469C452AF891
:1038D00010300DDAB8F80820D8F800300132A8F816
:1038E00008203AF91020A2EB0C021344C8F800306B
:1038F000022840F340837B6B0130834204F10204D1
:10390000CCD1D7F830B05B46BBF1000F40F0E38379
:1039100032B27A622AB23A629EFBF0F23A61002237
:10392000F96AC7E910329142BA6440F31E839646A1
:103930006FF001049446F14647F6FF76D7F8E4307D
:10394000C7F8E880D3F800A0D7F8C4500B19704826
:10395000D7F8EC807A60FA613A63BB6202460023D2
:1039600000F5967B32F91E1B93450B44FAD1694A48
:1039700082FB0312DB17C3EBA2031BB2002BC8BFF1
:1039800099449C45B8BF9C469E42A8BF1E469A4596
:103990002B800DDAB8F80830D8F800200133A8F8E9
:1039A0000830B5F90030A3EB0A010A44C8F800203A
:1039B0000B2C23EAE37340F2F9829E4401233B631C
:1039C000BB6A0134A34205F1020500F10200C5D132
:1039D0003B6BD7F8E880002B40F08C837B68002B92
:1039E00040F07683FB6A0FFA8CFC99FBF3FB7B6C4F
:1039F00036B2FB617D69398C2B46083323F007030F
:103A0000ADEB030DA8F80E106946BB8CFA6AA8F856
:103A10000C30C2F39C03A1EBC3030DF1180A9D46C1
:103A20000020D7F8EC30C7E91300A3F80CC0DE8102
:103A300006AB7B62131FBB627B6BC7E91500834239
:103A4000C7E9170033DD40F24458844681460646F4
:103A50000446D7F8C030C7F820A0991E0D44AE46E2
:103A6000AAF10205D7F810A0386331F9022FA2EBB2
:103A70000A0323EAE3731BB2973A9E4292B225F8F7
:103A8000023F03DA1E464FF001093C6342459CBFEA
:103A9000012084448E4504F10104E6D1D7F820A02A
:103AA000B9F1000F40F01F83002840F01983FB6A32
:103AB000042B1EDD002502222E462C46D7F8C4100A
:103AC000A3F1020C7B6A8818991E30F9023FA3EB20
:103AD0000B0323EAE3731BB2A34221F8023F02DD8A
:103AE0001C461546012601326245EED1002E40F0FB
:103AF000FE827B6B002B18DDBAF90030002B14DD41
:103B000052460023786B0BE0F4100020F8100020E0
:103B1000781300206766666632F9021F002903DD0C
:103B200001338342F8D17B6BFB64FB6901241946A6
:103B3000BB6A00254FF0040891FBF3FC40F23942C8
:103B4000A64EA74B0592CDE90336CDE901452246A5
:103B50002146CDF8008007F14003C7F864C0492032
:103B60000AF068FF40F23A409E4B224621460590FB
:103B70000393492007F164030496CDE90145CDF88C
:103B800000800AF057FF4FF0020940F23C4CCDE9AB
:103B90000145954804967A6B53462146CDF814C0EA
:103BA0000390CDF8009049200AF044FF40F23D4CCC
:103BB000CDE901458D480496CDF80090D7E909324A
:103BC0002146CDF814C0039049200AF033FF40F29B
:103BD0003F40874B2246214605900393492007F139
:103BE00044030496CDE90145CDF800800AF022FF98
:103BF0004FF488607F4B224621460590039349206D
:103C000007F148030496CDE90145CDF800800AF09C
:103C100011FF40F24240784B224621460590039323
:103C2000492007F14C030496CDE90145CDF8008009
:103C30000AF000FF40F24340704B224621460590B7
:103C40000393492007F150030496CDE90145CDF8CF
:103C500000800AF0EFFE40F24540694B22462146C3
:103C600005900393492007F154030496CDE90145DB
:103C7000CDF800800AF0DEFE40F24640614B22465D
:103C8000214605900393492007F15C030496CDE992
:103C90000145CDF800800AF0CDFE4FF489605A4B03
:103CA0002246214605900393492007F158030496C4
:103CB000CDE90145CDF800800AF0BCFE40F2494054
:103CC000524B2246214605900393492007F1600399
:103CD0000496CDE90145CDF800800AF0ABFE4FF027
:103CE000030E4B4A4B4BDFF848C107F17001B7F99F
:103CF0004400C7E91E2387F83E50C7E92055C7E9AD
:103D00002255C7E92455C7E91CEC12F077FDD7E925
:103D10001132A342B8BF2346920192FBF3F323EA88
:103D2000E373984287F83F50C7E91A0304DAFB6D42
:103D3000032BC8BF87F83F4001244FF0000804253B
:103D40004FF48E62344BCDE9046221462246009541
:103D50000393492007F16C03CDE901480AF06AFE9C
:103D600040F271402D4B0095224621460590039369
:103D7000492007F16803CDE9014804960AF05AFE8C
:103D800040F27240264B274D224605900393CDE921
:103D9000018807F13F0300940496214649200AF068
:103DA00049FE2A783B6C002A44D1502B03DD7B6E00
:103DB0001E2B00F3AA804FF49462084B00921A491C
:103DC000002264200AF07EFE97F83E30002B40F07F
:103DD000B0800022154B1A6047E000BF307101002F
:103DE000886E0100946E0100A46E0100B86E01009F
:103DF000CC6E0100DC6E0100EC6E0100FC6E010077
:103E0000106F0100286F0100446F01005C6F01001A
:103E1000E8034000D0074000786F0100886F010080
:103E2000986F0100F01000208C700100EC10002051
:103E3000F4013200462B03DD7B6E1E2B00F3A580C0
:103E40004FF49762AD4B0092AD49002264200AF016
:103E500039FE002387F83E30AA4A13680133282B25
:103E6000136002DD00232B70136001244FF0000863
:103E70004FF004094FF49962A34BCDE90462214647
:103E800022460393CDE90148CDF800909F4B49208D
:103E90000AF0D0FD40F2C9409D4B224621460590D4
:103EA0000393CDE90148CDF800900496954B492045
:103EB0000AF0C0FD40F2CB40964B224621460590C9
:103EC0000393CDE9018807F13E030094049649204D
:103ED0000AF0B0FD40F2CC408F4B22460590039390
:103EE000CDE901880094049621468C4B49200AF0C4
:103EF000A1FDBA69287813689C3723440A2B08BFB0
:103F000043461360BD46BDE8F08F4FF48F6384498C
:103F100000936420794B0AF0D5FD3B6D87F83E4055
:103F2000132B02DCFB68002B46D097F83F30002BA8
:103F300059D1764A136801330A2B136095DD0121AC
:103F400000232970136090E7FB6A002B64DD7A6B15
:103F5000744B5200BB617A611C6874E447F6FF72CF
:103F600003463861C7E90820D9E4934647F6FF764F
:103F7000FA6194463EE501223AF910303A63BA6A92
:103F8000002BA8BFD218BA62B5E44FF496625B4B1F
:103F900000926549424664200AF094FD97F83F205C
:103FA00087F83E4062BB574B1A605EE701227A6099
:103FB000FA691A44FA6103E5FB6D052B3EDC7B6C64
:103FC000B3F57A7F66DBFB6C052BB2DC40F28442F2
:103FD0004A4B00925549002264200AF073FD0023E9
:103FE00087F83E30F5E640F29C42444B009250493F
:103FF000002264200AF066FD002387F83E30E8E6E0
:1040000040F2B4423D4B00924A49424664200AF0D5
:1040100059FD87F83E801FE7002347F6FF763B6196
:10402000C7E91033BB647B629B46FB619C463D4BFA
:104030003E62BB617B6B5B007B61DBE497F83F30EA
:10404000DBB9BB6CB3F57A7F06DDFB6C052B03DCBB
:104050007B6DB3F5FA7F2EDBBB68002B3FF469AFB5
:1040600040F29542254B00923349002264200AF029
:1040700029FD002387F83E30ABE640F28B420092E8
:10408000FC681E4B22462B4964200AF01BFD87F872
:104090003E409EE64FF490620092FC68174B224629
:1040A000264964200AF00EFDFB6C87F83E40052B84
:1040B0003FF78FAE8AE740F29242104B00922049C0
:1040C000002264200AF0FEFC002387F83E3080E6E0
:1040D000FB697B6486E40323BA6A92FBF3F317E47B
:1040E000C7F850C0E3E43B6B7E65FB65DCE4BC6570
:1040F0003D66FEE4C7F848E070E400BF307101009F
:104100008C700100E8100020E4700100EC10002029
:10411000F87001000C71010020710100F010002006
:10412000A46F0100F4100020C0700100EC6F0100CA
:10413000607001000870010048700100C86F010044
:10414000287001000048704700000020014B036008
:104150002020704780710100014B03600F207047E1
:10416000A0710100014B03600F20704770710100C6
:1041700030B44FF0804300220E211F2020250F2451
:1041800083F8082183F80A2183F8090183F80B11C9
:104190001A739A735873D9731D725C72DA7793F835
:1041A000211041F0010183F8211093F8211062F3EE
:1041B000410183F8211030BC704700BF10B44FF0AC
:1041C000804485B00DF1100C0CE90F00BDF80030F3
:1041D0002382BDF802306382BDF90430A382BDF9A9
:1041E0000630E382BDF808302383BDF80A306383CC
:1041F000BDF80C30A38305B010BC70474FF080436E
:10420000988370474FF08043988B70474FF08043FE
:1042100083F82000704700BF0123002110B50A4A2F
:104220000A4C2377917210B94FF08042D3704FF04F
:1042300080430122987000211A700A2000F0BEF914
:104240000022024B1A7710BDA41400200000105069
:1042500001234FF08040102110B4034A034CA37295
:10426000436010BC1160704714000020A4140020AB
:1042700001234FF08040102110B4044A044C6372B3
:10428000C0F8043110BC1160704700BF140000205A
:10429000A4140020E0220021014812F072BC00BFEB
:1042A000800100402DE9F04105461F4B1F4886B0B4
:1042B0006A1E13F8011B834202F8011FF9D1012481
:1042C0002B464FF0A90C002702262868184AC11770
:1042D00082FB00E2DFF8648002441648C1EB222230
:1042E00043F8242B2146CDF814C02246CDE903081B
:1042F000CDE90147009662200AF09CFB4FF0AA0C22
:104300000D48CDF810800390CDE90147009605F1E6
:10431000260322462146CDF814C062200AF08AFB0B
:1043200006B0BDE8F08100BF280000405400004006
:1043300089888888B4710100C8710100B0710100DA
:1043400070B5E022064600210B4812F01AFC00244A
:1043500001234FF08042094D09492B770A208C72C6
:1043600093702146137000F029F92C773046BDE890
:104370007040FFF797BF00BF800100400000105061
:10438000A414002010B50446FFF78CFF2E234FF035
:10439000804004F14E0203F1600150F82110013B0E
:1043A0001F2B22F8021DF6D14FF0804004F1960237
:1043B00003F1600150F82110013B22F8021D591C45
:1043C000F6D110BD4FF0804270B5037909B201FB00
:1043D00003F1948B8B11A342B8BF2346012500241F
:1043E000022106889BB24380A2F80C61A2F80E312C
:1043F000074E084B357709205C7282F8035182F82A
:1044000002112146A2F8005100F0D8F8347770BDAF
:1044100000001050A41400204FF0804393F81401C2
:10442000704700BF4FF0804393F81701704700BFFB
:104430000023094A82F832305064916472B6012335
:1044400082F8403000BFB2F852309BB2002BFAD055
:1044500062B6B2F850007047000010502DE9F047E6
:1044600050221020202130244FF0400A4FF06009E4
:104470004FF001084FF4807E4FF4007C4FF48067CA
:104480004FF400660825104B83F8040383F80813E3
:1044900083F8004383F8034383F805A383F80923D3
:1044A00083F80A2383F80B2383F80F93C3F8008063
:1044B00018601960C3F800E0C3F800C01F601E60F8
:1044C0001D60BDE8F08700BF00E100E04FF400424E
:1044D000014B1A60704700BF00E100E0002201219B
:1044E000034BA3F86E20A3F86A20A3F86810704766
:1044F0000000105030B5134DA1B02B7803B3124C0F
:10450000124B22689A421BD080226846002112F08A
:1045100038FB002223468034186820A9043301EBBD
:104520008201A34241F8800C02F10102F4D1074B51
:104530006A4680210448009300F07AFC00232B7027
:1045400021B030BDDC14002000FC0100DEADDEAD8A
:1045500010B5174C84B094E80300029002A88DF8BF
:104560000C1000F07DF800F085F8FFF777FF62B6D9
:1045700000F00AFAA36804A840F80C3D00F0FEF928
:1045800000F046FA00F06EF900F0AEFA094B1A6935
:1045900022F004021A61BFF34F8F0721064A82F806
:1045A00024105A6942F010025A6104B010BD00BFD5
:1045B000DC71010000ED00E0000010502DE9F04733
:1045C000044682B00F464FF0AC0A124DDFF8489017
:1045D000DFF8488005E000BF30BF62B60CF024F879
:1045E00070B900BF72B62B5D03F0FF06002BF2D04E
:1045F00000232B5507B1B84762B602B0BDE8F0877B
:10460000CDF800A032464B46414664200AF05AFAE3
:10461000E7E700BFA4140020E8710100EC7101007D
:1046200000200A4B0A4913F8012B10448B42C0B2F8
:10463000F9D1064B1A78AA2A01D000207047DB7BFB
:10464000181AB0FA80F04009704700BF800040009F
:104650008F0040004FF0A04301225A74704700BF02
:104660000246034B0068127918601A71704700BF48
:10467000B414002070B5FFF7D3FF01220021334BA3
:10468000D9705A72DA7200285CD0314AD278D2B22C
:104690001A72002201242F492C4B8D789A725A737A
:1046A0001D734D780E781E751D77CD78097983F8C6
:1046B000215083F820105A749A741C749A7018B39D
:1046C000234A51781A78C9B2D2B28A4208D08A42B3
:1046D000B4BF013202F1FF32D0B28A421870F6D173
:1046E0001B4B1A491A794B78D2B2DBB29A420AD0E4
:1046F0009A4203F1010096BF03F1FF33C3B2DBB26C
:104700009A424B70F4D170BD1A78D2B2B02A08D058
:10471000AF2AD4BF013202F1FF32D1B2B02A1970F0
:10472000F6D10A4A5378DBB2082BECD0072B03F101
:1047300001018ABF03F1FF33CBB2DBB2082B537008
:10474000F4D1E0E7E0221A72A3E700BF00001050A6
:1047500080004000B414002007490B78DBB283428C
:1047600008D09842CCBF013303F1FF33DAB2834261
:104770000A70F6D1704700BF00001050014B187846
:10478000704700BF00001050084A5378DBB28342E4
:104790000AD0984203F1010196BF03F1FF33CBB277
:1047A000DBB283425370F4D1704700BF0000105059
:1047B000014B5878704700BF0000105010B50446F8
:1047C000FFF748FF4FF0A04320686168A26807C365
:1047D00010BD00BF38B54FF0A044E37DDBB2042B21
:1047E00028D0082B19D0022B09D00123184A1370A6
:1047F00000BF4FF0A042137300BF537338BD154D77
:104800001549607910F0E6FB6179286810F02AFC00
:1048100062792B6813442B60E7E7104BD0E905124F
:1048200059609A60236A5BBA0A4A1846136010F00E
:104830009BFBDAE7074D0A49207910F0A9FB2179A3
:10484000286810F0E3FB22792B6813442B60CCE737
:10485000A4140020BC14002020000050381C0020AC
:1048600024000050274B0022D3F8801021F00101D2
:10487000C3F88010196C41F001011964196841F006
:1048800001011960D3F8801021F00201C3F88010F3
:10489000196C21F002011964196841F002011960D4
:1048A000D3F8801021F01001C3F88010196C41F08A
:1048B00010011964196841F010011960D3F88010D3
:1048C00021F02001C3F88010196C21F02001196437
:1048D000196841F020011960D3F8801021F04001DF
:1048E000C3F88010196C21F040011964196841F077
:1048F00040011960C3F80821C3F80421C3F800215E
:10490000704700BF00000250034BD3F8C03018427C
:104910000CBF012000207047000002504FF04053B0
:10492000012283F8242083F8812070474FF0405300
:10493000002283F8242083F881207047142001226C
:10494000002130B50A4D89B02D780A4C05900A48EF
:1049500008AB03F8015DCDE90111CDE90304009234
:10496000114664200AF066F89DF81F0009B030BDBA
:10497000B700400000720100087201000268014B9C
:104980001A607047C014002038B5FFF749FE0F23A6
:10499000F0B94FF040524FF00104D9B2013B072B60
:1049A00082F82B1082F8284082F82800F5D10423E1
:1049B00082F82F304FF040530121002283F8281055
:1049C00083F828204FF47A70BDE8384000F022BB0D
:1049D0004FF04051012500240C4806E081F82B20BF
:1049E000013B81F8285081F82840027A0E2A8EBFB8
:1049F0000F22027AD2B29342DAB2EFDA4FF040528B
:104A0000024B5B7ADBB282F82F30D3E780004000A4
:104A1000F8B5FFF705FE4FF0405401250026074684
:104A200084F825604FF47A7084F8205084F8275079
:104A300000F0F0FA84F8256084F8245007BB0623C0
:104A40001C4D84F82730EB7884F826302B7884F8D6
:104A500042304FF0405401230022697840F24C402C
:104A600084F8461084F8442084F8453084F84130B6
:104A700084F8403000F0CEFAAB7884F84430F8BDCA
:104A8000FFF75CFF0C4B9B7A88B94FF04052DBB2CA
:104A9000084D84F82730E978074B82F82610DB7A36
:104AA00029780B440B3BDBB282F84230D1E7053B5F
:104AB000EBE700BFC01400208000400020B9064A88
:104AC000064B10601860704703490548034B054AC0
:104AD00008601A60704700BFC8140020C41400208A
:104AE0001D4900002D4900004FF040530620F0B44E
:104AF00001220A26FF24002583F8D60093F8D71058
:104B00004FF00F0C60F3030183F8D710042183F8F2
:104B1000D860052783F8402183F8D0400324072676
:104B200083F87F5093F88C00104383F88C0093F83F
:104B30008C0040F0020083F88C0093F8910061F340
:104B4000030083F8910083F8901083F88D1083F8A8
:104B5000A02093F8A10065F3010083F8A10083F879
:104B600094C093F88800104383F8880093F8890074
:104B7000104383F8890083F8F12083F8874083F895
:104B80008E4083F8D22083F8D52083F8AB7083F869
:104B9000AD5083F8AC4083F8AE1083F8AF1093F8B3
:104BA0008B1041F0700183F88B1083F8936083F8C9
:104BB000B020F0BC704700BF00220D480D4B0E49DD
:104BC00010B403600B6800EB82047F3323F07F0393
:104BD00041F8043B52B154F8043C51F8084C022A05
:104BE000234440F8223001D110BC70470132E9E77C
:104BF00074200020000240000400002032232DE930
:104C0000F04F514E8BB00093002233464F49642041
:104C100009F058FF002504273323DFF844814C4A6C
:104C2000CDE9046303924346032201216420CDE9C8
:104C30000155009709F0FEFE4FF0640B3423454CFC
:104C4000454A0593039223460322012158460496C0
:104C5000CDE90155009709F0EDFE01223C23A06843
:104C6000D8F808C03D498444ACF50074A4B20BFBED
:104C700004F4A1FB0414DFF8EC80DFF8ECE011464B
:104C8000A40A58460593049607ABCDE90155009751
:104C9000CDF80C80CDE908E4CDF81CC0144609F02D
:104CA000C9FE3D23DFF8C4905846059322462146AD
:104CB00008AB0496029500970194CDF80C9009F08A
:104CC000B9FE3E23DFF8A8A022460593049609AB5F
:104CD000CDE90145009758462146CDF80CA009F0D2
:104CE000A9FEDDE907239A422BD927464FF08C0B0A
:104CF00000240425012207AB1146CDE9046BCDE960
:104D00000248CDE90054642009F094FE01228D236D
:104D100011460593029408AB0095CDE903960197DF
:104D2000642009F087FE8E230122059302940095EA
:104D3000CDE903A60197114609AB642009F07AFE7C
:104D4000D6E70BB0BDE8F08F0C72010028720100AD
:104D50005C7201000400002070720100ABAAAAAAD4
:104D6000742000208472010000084000907201004D
:104D70009C720100034B044AD3E9001310681944E4
:104D8000FFF756BB040000207420002041F23423BA
:104D900010B50D4C226812889A4201D0002010BD37
:104DA000FFF7E8FFA3681B888342F7D123685B887D
:104DB000012BF3D10DF092FC23685B68181AB0FA4E
:104DC00080F0400910BD00BF74200020164B30B4A5
:104DD0001D7BEDB272B60022072491421C7383F84A
:104DE00031200EDD4A1E22F07F0200F180030124F3
:104DF0001A4400E0803340F480109A420460184660
:104E0000F8D10121084B094A83F831101D73D2F8FB
:104E10000001000405D54FF40040A3F86C10C2F85F
:104E2000800162B630BC70470000105000E100E025
:104E3000F0B5A1B006460F461546FFF7C7FF6B4613
:104E40001946C3F1C04000F580200C5C20AA01F88F
:104E5000014B9142F9D11B4A92F80CC05FFA8CFCCD
:104E600072B607240021147382F831103A1EB8BFBD
:104E700003329210002A09DD294605EB8205761AD5
:104E80008A1951F8044BA9421460F9D101240D4A42
:104E90000D4982F8314082F80CC0D1F800512D0440
:104EA00009D462B61A1813F8011B117020AA934294
:104EB000F8D121B0F0BD4FF40045A2F86C40C1F824
:104EC0008051EEE70000105000E100E0034610B40E
:104ED0000448054C0A4650F8230054F8231010BC2F
:104EE000FFF7A6BF74200020040000200022052147
:104EF000034B04481A6058609A601960704700BFFD
:104F000010E000E0FFFF0F000022044B98681A60D9
:104F1000C0F57F2000F6FF70704700BF10E000E092
:104F2000054A0649937CD27801335B00934000FB2D
:104F300003F091FBF0F070470000105000B4C4047F
:104F4000054A937AD27ADBB20AB101339840034B17
:104F500093FBF0F0704700BF0000105040420F007C
:104F6000054A937AD27ADBB22AB10122134402FABB
:104F700003F390FBF3F0704700001050054A00EB7C
:104F80008000937CD27801335B009340000190FB5A
:104F9000F3F0704700001050034B044A5B7C03F0B1
:104FA000010352F82330184700001050BC72010072
:104FB000034B044A5B7C03F0010352F8233018478B
:104FC00000001050B472010070B5012200241D21B0
:104FD000042688B008AB43F8040D0B4D0B48CDE90F
:104FE00001240591CDE9030511460096642009F0DE
:104FF00021FD074B07985C7100F046F8214605201B
:10500000FFF7DCFA08B070BDC4720100CC72010079
:10501000A414002008B5FFF7BFFFBDE80840FFF764
:10502000D3BF00BF08B5FFF7C3FFBDE8084000F0DD
:1050300013B800BF08B5FFF7AFFFBDE8084000F0A8
:1050400023B800BF002000F043B800BF012000F0EB
:105050003FB800BF00F030B8012830B44FF0000274
:105060004FF0020438BF01200121054B054D1A7095
:105070002A719C709860DA605A70197030BC704761
:1050800000000850A414002001284FF000024FF047
:10509000010138BF012010B4054B064C1A70627133
:1050A00099709860DA605A70197010BC704700BF30
:1050B00000000950A4140020012000220249034BE3
:1050C00008711A70704700BFA41400200000085037
:1050D00010B40B4A0B4983B0CDE9001202AB03EBCD
:1050E000800353F8082C9378DBB2012B04D1002104
:1050F000054C04302354117003B010BC704700BF3E
:105100000000095000000850A4140020024A136C4B
:1051100023F001031364704700000250024A136C2D
:1051200043F001031364704700000250024B186CF7
:10513000C04300F0010070470000025070B4DCF87A
:105140000C400028D4F809304FF000021E680DDD35
:10515000DCF80830DB681D18013D013B13F8011F26
:10516000715C9D420A44F9D192FBF0F2DCF8041024
:105170004B88A3B108891B1A1B02121A93FBF2F287
:10518000B2F5DC7FA8BF4FF4DC720A62D4F80D30B0
:1051900070BC198902FB01F212125A8170474FF458
:1051A00080720A62F2E700BF002822DDF0B5DCF869
:1051B0000460002496F80EE00CE0DCF800703F5D1F
:1051C00007FB033305FB03F35B1242F82430013481
:1051D000A0420DD051F8043B356ABEF1000FECD16E
:1051E00003FB05F39B1042F824300134A042F1D1B7
:1051F000F0BD704770B4DCF80C400028D4F80930DA
:105200004FF000021E680DDDDCF80830DB681D1869
:10521000013D013B13F8011F715C9D420A44F9D125
:1052200092FBF0F2DCF80410CB88A3B188881B1A3B
:105230001B02121A93FBF2F2B2F5DC7FA8BF4FF407
:10524000DC720A62D4F80D3070BC198902FB01F2DD
:1052500012125A8170474FF480720A62F2E700BF5F
:10526000002822DDF0B5DCF80460002496F80EE09A
:105270000CE0DCF800703F5D07FB033305FB03F334
:105280005B1242F824300134A0420DD051F8043BA7
:10529000356ABEF1000FECD103FB05F39B1042F819
:1052A00024300134A042F1D1F0BD704770B4DCF875
:1052B0000C400028D4F809304FF000021E680DDDC4
:1052C000DCF80830DB681D18013D013B13F8011FB5
:1052D000715C9D420A44F9D192FBF0F2DCF80410B3
:1052E0004B89A3B188891B1A1B02121A93FBF2F295
:1052F000B2F5DC7FA8BF4FF4DC720A62D4F80D303F
:1053000070BC198902FB01F212125A8170474FF4E6
:1053100080720A62F2E700BF002822DDF0B5DCF8F7
:105320000460002496F80EE00CE0DCF800703F5DAD
:1053300007FB033305FB03F35B1242F8243001340F
:10534000A0420DD051F8043B356ABEF1000FECD1FC
:1053500003FB05F39B1042F824300134A042F1D145
:10536000F0BD704770B4DCF80C400028D4F8093068
:105370004FF000021E680DDDDCF80830DB681D18F8
:10538000013D013B13F8011F715C9D420A44F9D1B4
:1053900092FBF0F2DCF804104B88A3B108891B1AC9
:1053A0001B02121A93FBF2F2B2F5DC7FA8BF4FF496
:1053B000DC720A62D4F80D3070BC198902FB01F26C
:1053C00012125A8170474FF480720A62F2E700BFEE
:1053D000002822DDF0B5DCF80460002496F80EE029
:1053E0000CE0DCF800703F5D07FB033305FB03F3C3
:1053F0005B1242F824300134A0420DD051F8043B36
:10540000356ABEF1000FECD103FB05F39B1042F8A7
:1054100024300134A042F1D1F0BD704770B4DCF803
:105420000C400028D4F809304FF000021E680DDD52
:10543000DCF80830DB681D18013D013B13F8011F43
:10544000715C9D420A44F9D192FBF0F2DCF8041041
:10545000CB88A3B188881B1A1B02121A93FBF2F2A5
:10546000B2F5DC7FA8BF4FF4DC720A62D4F80D30CD
:1054700070BC198902FB01F212125A8170474FF475
:1054800080720A62F2E700BF002822DDF0B5DCF886
:105490000460002496F80EE00CE0DCF800703F5D3C
:1054A00007FB033305FB03F35B1242F8243001349E
:1054B000A0420DD051F8043B356ABEF1000FECD18B
:1054C00003FB05F39B1042F824300134A042F1D1D4
:1054D000F0BD7047F0B40024DCF8083001F5F06549
:1054E000D3F8093001F50067DE68043E56F8041F62
:1054F000A5F5F06252F8803BCB1AAA421C44F9D1C0
:10550000151DAF42F2D1DCF804104A887AB194FB41
:10551000F0F3F0BC8888121A12021B1A92FBF3F304
:10552000B3F5DC7FA8BF4FF4DC730B6270474FF418
:105530008073F0BC0B627047F0B4DCF80450AC7BB5
:105540007CB900280BDD51F8046B2B6A013403FB96
:1055500006F3A0424FEAA30342F8043BF3D1F0BCA8
:1055600070470028FBDDDCF80060013E304416F88F
:10557000017F51F8044B2B6A07FB044403FB04F33F
:10558000B0424FEA632342F8043BF0D1F0BC7047CD
:10559000704700BF00280BDD10B4002451F8043B15
:1055A00001349B01A04242F8043BF7D110BC704784
:1055B000704700BF30B58DB02022002104A811F043
:1055C000E0FA1E4D1E491F4C1F48CDE90054CDE99D
:1055D00002011E4A1E4B069293F881208DF81C2072
:1055E00093F881308DF81D300DF04EF88DF81E00C7
:1055F0000DF050F88DF81F000DF052F88DF82000D6
:105600000DF054F88DF821000DF056F88DF82200B9
:105610000DF058F809900DF05BF80A900DF05EF867
:10562000ADF82C0068460FF0BDFB0DF057F810F0F8
:105630003DF80FF08DFB0DB030BD00BF0D510000E7
:10564000155000001D5100002D5100006E0016780D
:105650000000105070B5002301223F214826082584
:10566000022484B001A8CDE9013303938DF80760CB
:105670008DF808508DF809208DF80F208DF80A401C
:105680008DF80D10FFF79AF804B070BDD0F80D201A
:10569000138901FB03F1091251817047002809DDCC
:1056A000043A02EB8000043952F8043F824241F888
:1056B000043FF9D1704700BF2DE9F042204E92B06F
:1056C000204D0DAC05AF99460691089296E80F0063
:1056D00084E80F0018ABC4E90275204611A91193A4
:1056E000FAF7CEFD96E80F00174E09AD85E80F00DA
:1056F000C5E9027621462846FAF7C2FD089B069ABC
:1057000044F0010445F00105D3F801001269189E28
:10571000CDE903450D490790059202910196D3F812
:1057200009308022DB690021184611F02AFA202274
:10573000034601A948460CF0D7FF12B0BDE8F0823D
:10574000D07201003D510000A9510000351C01003C
:105750002DE9F042204E92B0204D0DAC05AF994698
:105760000691089296E80F0084E80F0018ABC4E990
:105770000275204611A91193FAF782FD96E80F00F1
:10578000174E09AD85E80F00C5E902762146284687
:10579000FAF776FD089B069A44F0010445F00105EE
:1057A000D3F801001269189ECDE903450D49079011
:1057B000059202910196D3F809303C22DB69002161
:1057C000184611F0DEF90F22034601A948460CF0F5
:1057D0008BFF12B0BDE8F082D0720100F5510000DD
:1057E00061520000991C01002DE9F042994692B0E7
:1057F0001C4E1D4D0DAC05AF0691089296E80F00AA
:1058000084E80F0018ABC4E90275204611A9119372
:10581000FAF736FD96E80F00144E09AD85E80F0043
:10582000C5E9027621462846FAF72AFD089B069A22
:1058300044F0010445F00105D3F801001269189EF7
:10584000CDE903450A490790059202910196D3F8E4
:10585000093048469B68002201A90CF045FF12B0B0
:10586000BDE8F082D0720100AD5200001953000073
:10587000C92001002DE9F042204E92B0204D0DAC20
:1058800005AF99460691089296E80F0084E80F004C
:1058900018ABC4E90275204611A91193FAF7F0FC80
:1058A00096E80F00174E09AD85E80F00C5E90276AE
:1058B00021462846FAF7E4FC089B069A44F00104C6
:1058C00045F00105D3F801001269189ECDE90345A2
:1058D0000D490790059202910196D3F80930802274
:1058E000DB690021184611F04CF92022034601A97A
:1058F00048460CF0F9FE12B0BDE8F082D07201000B
:1059000065530000D15300004D1C01002DE9F04209
:10591000204E92B0204D0DAC05AF994606910892ED
:1059200096E80F0084E80F0018ABC4E90275204622
:1059300011A91193FAF7A4FC96E80F00174E09ADD0
:1059400085E80F00C5E9027621462846FAF798FC5B
:10595000089B069A44F0010445F00105D3F80100C4
:105960001269189ECDE903450D49079005920291F1
:105970000196D3F809303C22DB690021184611F06A
:1059800000F90F22034601A948460CF0ADFE12B003
:10599000BDE8F082D07201001D540000895400005F
:1059A000F51C0100D0F80D301A68D38801FB03F113
:1059B00009121181704700BF0269054B0548013A81
:1059C00012F8011F013303F8011C8342F8D170471C
:1059D00000008360E00183602DE9F043894691B0C7
:1059E0001F4E204D0BAC04AF9846CDE9050296E85A
:1059F0000F0084E80F0018ABC4E9027520460FA918
:105A00000F93FAF73DFC96E80F00174E07AD85E8B7
:105A10000F00C5E9027621462846FAF731FCD9F88D
:105A200009304FF4F0621B690021184611F0A9F803
:105A3000059A0E4E12690E4F0346049244F001047B
:105A400045F0010540464FF4F0726946CDE9024544
:105A5000CDE900670CF048FE11B0BDE8F08300BF4F
:105A6000D0720100D554000039550000D90501005D
:105A700075FF0000F0B50F46D0F8093085B0DC683E
:105A80000AF0AAFD0AF06CFA20468022002111F0EB
:105A900078F8084A0849094E094D009201912346B9
:105AA000384620226946CDE902650CF01DFE05B09E
:105AB000F0BD00BFD905010061FF00009155000055
:105AC000955500002DE9F04100264FF00108284FC0
:105AD00082B0FFF76FFDFFF7BDFDFEF733FB0AF065
:105AE00095FAFFF769F8A7F86860FFF74FF90FF02C
:105AF000C1FAA7F86880FEF72BFDFEF739FBDFF847
:105B000080C01C4C6546A7F868600FCC0FC50FCC51
:105B10000FC50FCC0FC5DCF80030226801332A60B6
:105B200005D0A4F130008021FFF750F9FEE7124CB8
:105B3000A7F86880FFF762F80FF0F2FB0CF0D0FADC
:105B4000414632462568334600960220A8470B4D51
:105B500063689847A36898472C68FEF70FFEA0700B
:105B60002C68FEF725FEE07002B0BDE8F08100BFB2
:105B70000000105010FC010038B30100D80C0020C8
:105B8000441C00200246034B51680068926807C31A
:105B9000704700BFD01400202DE9F04F964683B027
:105BA000544E9DF834709DF830C098460097634677
:105BB0000D46B6F90620B6F90410044670469DF865
:105BC000387010F0AFFD3378800290FBF8F0002BB6
:105BD0004BD0A91C96F801904B002A4604EB030E0B
:105BE00003F10208B9F1000F50D13EF8069C05F10F
:105BF000FF3C24F80890A3F108053EF8043C254436
:105C000024F811306189238961802380531ED2B327
:105C10001A4602F1010B4FEA4B0104EB010A06316F
:105C200034F801903AF8028C34F81B30C84407FB72
:105C300008F9BAF8048096F903B043440BFB0398C3
:105C4000BAF8023096F90290624509FB03834FEAE5
:105C5000A31300FB03F34FEA2343635246D0012A08
:105C6000D4D1E38800226380D3E765B1A91C04EB9B
:105C70004101043431F8022D00FB02F28C424FEA5C
:105C800022428A80F6D103B0BDE8F08F0023638002
:105C9000238024F8113024F80830002DF3D07F0041
:105CA00004EB450131F802E996F90350B1F808C058
:105CB0000B88CA889C4538BF9C46964538BF964697
:105CC0000CFB07F36A000EFB02338D8896F9022065
:105CD0008C4205FB02324FEAA21200FB02F24FEAAD
:105CE00022420A81DED103B0BDE8F08F2B88AEF8E6
:105CF00000308BE7D0140020F0B505462C4C4269EB
:105D000094F9033094F90270C3F12003E07AC7EBF1
:105D10004307A37A85B0C7F34707CDE9010700938E
:105D200005F12C0020230E460F21FFF735FF617A85
:105D3000237A05F152046A692046CDE901170093E0
:105D400020210F23FFF728FFFEF7A4FA20462E2379
:105D50004FF0804403F1600230F8021D013B1F2B1D
:105D600044F82210F6D14FF0804405F19A0232F83F
:105D7000020D03F16001013B44F82100591CF6D1EA
:105D80000120FEF749FA2846FEF78CFAB4F84C30A9
:105D90001BB2336094F85030337294F85130737200
:105DA00094F85230B37294F85330F37205B0F0BDEA
:105DB000D014002038B504220125134B134C1D715B
:105DC0002260FFF73FF90FF0ABFA837E43B9104B27
:105DD0001B682BB10F4A126812B90F4A1570984709
:105DE0000E4BD3F80021120708D5002208250C48D5
:105DF0000C49C3F880510270C1F8402101211023E1
:105E0000094AD160236038BDA4140020140000208A
:105E1000C8150020201A0020C515002000E100E070
:105E20001000002000000250000008500520012151
:105E300038B50F4B0F4C104A1B682060517103B1ED
:105E40009847FFF703F90D4BD3F80021120708D547
:105E5000002208250A480B49C3F880510270C1F896
:105E6000402101211023084AD160236038BD00BFC2
:105E7000CC15002014000020A414002000E100E054
:105E800010000020000002500000095001210322F0
:105E900038B50B4B0B4DD9700B4C2B7822601BB1D6
:105EA000FFF732F8094B186001232B70FFF71EF83B
:105EB00000211023064AC2F84011236038BD00BFFC
:105EC000A41400201000002014000020CC14002096
:105ED0000000025001234FF06050102110B4034A1B
:105EE000034CE372836210BC116070471400002001
:105EF000A41400200F200121114A124B10605B6F87
:105F000084B00193019B104A23F4FF6323F007033D
:105F10000293019B117023F07F030393029BB3F55F
:105F2000800F09D00399094B994205D00122054BF6
:105F3000A3F86C2004B0704700231370F6E700BF8D
:105F40001400002000001050DC14002080FF01002D
:105F500008B5FFF7B7FD00F08DFC002008BD00BFBD
:105F6000704700BF08B54FF0CD3203490348FBF737
:105F700005FF002008BD00BF1C3800201C240020A5
:105F8000704700BFD2232DE9F041184A184D194C33
:105F900082B012682146009363202B4608F092FDE0
:105FA00008F078F8804608F027F9074608F026FA46
:105FB00006460AF093F940460AF0E2F838460AF03D
:105FC000DFF830460AF0DCF808F040F908F040FA53
:105FD00008F084F9E920084A2B461268214600900F
:105FE000632008F06FFD02B0BDE8F081AC0B00202B
:105FF0001C73010008730100B00B002056222DE92C
:10600000F04FB34BADF66C0D00921A68B149B24B2C
:10601000632008F057FD08F03DF8D0F8095008F06B
:10602000EBF80027D0F80930B946069308F014F8C9
:1060300008F0E4F9B8464FF0040BD0F809303AAC58
:10604000079308F023F808F02FF94FF470724946CF
:10605000204610F096FD402249461AA810F091FD06
:106060000DF595661E2249460AA810F08AFD4FF4E8
:1060700070724946304610F084FD402249462AA8F5
:1060800010F07FFD12A81E22494610F07AFDEB6841
:106090000DF6280A08937C3309930DF166050AF082
:1060A0009BFA0AF0D1FAB4460998A0F18002614641
:1060B00001E0B1F9007052F8043F3B44824221F8FC
:1060C000023BF6D1D44500F1800002D03CF9407F7C
:1060D000EBE7079B12A99B69043B01E0B1F9009033
:1060E00053F8042F4A4421F8022BA942F6D1069B0B
:1060F0002AAA9B69043B01E0B2F9008053F8040F1F
:10610000404422F8020BA242F6D1BBF1010BBDF9CB
:10611000A880BDF94890B6F90070C0D10DF59D601A
:1061200006F5806CA0F1400301E0B3F90070002F88
:10613000B8BF0337BF1023F8027B9842F5D1403037
:10614000844502D030F9407CECE712AB01E0B3F9B2
:106150000090B9F1000FB8BF09F103094FEAA9098E
:1061600023F8029B8B42F2D12AAB01E0B3F9008005
:10617000B8F1000FB8BF08F103084FEAA80823F8E8
:10618000028B9342F2D10FF0B9F80B28524F40F036
:1061900091800AF021FA0AF057FAAE223B460092AB
:1061A0004E490022602008F08DFC089B06F13E0855
:1061B000A3F104092AAB06F2FE3BA3EB060A48460C
:1061C000A8F140020AEB080132F9023F50F804EF4F
:1061D00031F902CFA3EB0E039C45B8BF0B8090456D
:1061E000F2D108F14008C34509F18009E7D1079BC6
:1061F0000DF1460298690DF1260104380DF1640E87
:1062000032F9023F50F8048F31F902CFA3EB0803B3
:106210009C45B8BF0B809645F2D12946069B0DF1EF
:10622000A60298690DF1E60E043832F9023F50F8E3
:10623000048F31F902CFA3EB08039C45B8BF0B8054
:106240009645F2D14FF001084FF0000A4FF00209D5
:10625000C223234A05930392234620220F2169205B
:106260000497CDE9018ACDF8009008F0E3FBC32242
:106270001C4B4146059203930F220AAB6920CDE9DE
:10628000018ACDF80090049708F0D4FBC722164B82
:106290004146CDE90472039320221AAB6920CDE96F
:1062A000018ACDF8009008F0C5FB0FF027F80B2805
:1062B0003FF46FAFCA220D4B00921A680549064B96
:1062C000632008F0FFFB00200DF66C0DBDE8F08F99
:1062D000AC0B0020F47201001C730100307301004C
:1062E000347301004473010050730100B00B0020AF
:1062F00033222DE9F04F5F4B83B000921A685E495C
:106300005E4B632008F0DEFBFDF71CFF044607F040
:10631000C1FE074607F070FF054608F06FF8064615
:1063200007F0C2FF8046204607F06AFF204608F0CB
:1063300069F807F0BDFF07F08BFEC5F80D0007F008
:10634000A1FEC6F80D0007F08BFEC8F80D0007F09F
:10635000A1FE07F051FF08F051F82146304609F040
:1063600037FF09F05FFF2146284609F031FF09F0A9
:1063700059FF2146384609F02BFF09F053FF07F07B
:1063800089FE044607F038FF064608F037F8054650
:1063900007F062FE07F07AFEFDF7D4FE0746002103
:1063A00020780AF077F82146384609F01BFCD4F82B
:1063B0000130DB7A1BB1207831490AF06BF80AF022
:1063C0000BF90AF041F9002130780AF063F8FDF783
:1063D000B9FE2C4A31460AF063FF30782A490AF0A8
:1063E00059F8002128780AF055F8FDF7ABFE254A48
:1063F00029460BF069FA254928780AF04BF807F08E
:1064000049FE824607F04AFE07F0F6FE804607F096
:10641000F5FF064607F048FF044607F0EDFD83460A
:1064200007F01AFE054607F031FE074607F01CFE8E
:10643000D5F82090DBF82010056A3F6A5046FFF738
:10644000B1FA49464046FFF721F939463046FFF791
:106450001DF929462046FFF719F950220C4B0092EE
:106460001A680549054B632008F02CFB03B0BDE812
:10647000F08F00BFAC0B0020E07201001C73010024
:10648000F1F90000D9050100C9140100AD1A01009D
:10649000B00B00204FF4A87330B50D4A0D4D0E4CD3
:1064A00083B012682146632000932B4608F00AFB54
:1064B00007F068FD08F05CF840F25510074A2B46DB
:1064C000126821460090632008F0FCFA03B030BD4A
:1064D000AC0B0020BC730100AC730100B00B0020BA
:1064E000432330B50C4A0D4D0D4C83B01268214644
:1064F000632000932B4608F0E5FA07F0D9FF07F078
:10650000CBFC4820074A2B461268214600906320A6
:1065100008F0D8FA03B030BDAC0B0020BC7301000A
:106520005C730100B00B00204E2330B5134A144DAC
:10653000144C87B012682146009363202B4608F064
:10654000C1FA114B02930CF0C9F80390FEF716F94B
:106550008DF81000FEF72CF902A98DF8110000202B
:10656000FEF7B4FC5E20094A2B46126821460090D3
:10657000632008F0A7FA07B030BD00BFAC0B0020C5
:10658000BC7301006C73010034120100B00B0020D9
:1065900065222DE9F041444BE2B000921A6843496C
:1065A000434B632008F08EFA07F0B0FD074607F072
:1065B000ADFE804607F048FD064607F05FFD054644
:1065C00007F06CFDD0F8094000200EF053FD0720C5
:1065D00006F072F8E3681BB107F024FD0023E360C6
:1065E000326A2B6A05AECDE90323D7F809301C685F
:1065F00004F1200C354620686168A268E368103415
:10660000644506F110060FC5F4D123784222337099
:10661000D7F809300DF14A00996810F0A7FAD8F8B8
:10662000093023AE1B681A685C689868D968CDF891
:106630003520CDF83940CDF83D00CDF841101A692C
:10664000CDF84520D8F809309C6804F1200C354677
:1066500020686168A268E3681034644506F110069A
:106660000FC5F4D120686168842203C6D7F80930C9
:106670002DA8D96910F07AFAD8F809305022D969D2
:106680004EA810F073FA03A90120FEF71FFC932215
:10669000084B00921A680549054B632008F012FA6E
:1066A00062B0BDE8F08100BFAC0B00207C7301003C
:1066B000BC730100B00B00209A2330B5104A114D75
:1066C000114C85B012682146009363202B4608F0D8
:1066D000F9F9FEF74FFB04A921F8040D0220FEF79B
:1066E000F5FB01200EF0C6FCA120084A2B461268DB
:1066F00021460090632008F0E5F905B030BD00BFE9
:10670000AC0B0020BC73010090730100B00B0020A3
:10671000F0B5B3B0A720514A02AF1268504B5149AF
:106720000090632008F0CEF90EF0B0FC01380B2881
:106730000BD8DFE800F018080808080808068D7272
:10674000491DFFF725FF0EF0E5FC40F24910464ACF
:10675000434B126843490090632008F0B3F90120CD
:10676000C437BD46F0BDFFF7DFFE0EF0D3FCECE70B
:106770003E4A3F4C9168D2E90030034419442068F6
:10678000FEF724FB00200EF075FC41F23420236854
:106790003E221B8800211B1A18BF012307F182002B
:1067A00087F8403010F0EDF9012340F2011207F1B3
:1067B000400107F18000A7F8802087F8823087F831
:1067C00085300EF069FCC0E7284B6D46D3E90042E6
:1067D0009B6814441C44E31D23F00703ADEB030D39
:1067E00002AE22460021304610F0CBF93E220021B5
:1067F00007F1420010F0C5F90123E4B2314607F178
:10680000400087F8414087F8424087F8403087F8D9
:1068100045300EF041FCAD4697E7FFF785FEFFF7E8
:10682000B7FEFFF749FF0EF02BFC3E2287F88000F1
:106830000021B81C10F0A5F9012340F2011207F164
:10684000800138463A80BB707B710EF025FC7CE7F6
:10685000FFF732FF0EF05EFC77E700BFAC0B0020C5
:10686000BC7301009C730100B00B002004000020E9
:10687000742000202DE9F04784B00EF03FFD2D225A
:10688000204E00920446204B00222049642008F04C
:1068900019F90025DFF880A0DFF86C90DFF87C8024
:1068A0001B4F56B3102D28D833689847A54201D006
:1068B0000EF01AFD012439224B4600924146002277
:1068C000602008F0FFF814B17368984704464FF051
:1068D000CD3239460F48FBF7ABFA0EF00FFD85427B
:1068E000E9D0B3680390984710F0ECF803982C4671
:1068F00005465AF82560002ED4D10EF0FFFC05465F
:10690000F7E700BFA00B0020C47301001074010062
:106910001C3800201C240020CC73010030730100BF
:106920004C23F0B5114A124D124C83B01268214627
:10693000009363202B4608F0C5F807F0ABFB074631
:1069400007F0ACFB064609F0C9FC384609F018FC14
:10695000304609F015FC5620074A2B46126821469E
:106960000090632008F0AEF803B0F0BDAC0B00203F
:106970005C74010048740100B00B0020F0B583B0D6
:10698000FDF7E0FB3C23124D124C134A21461268DE
:106990000646009363202B4608F094F807F07AFB34
:1069A000074607F07BFB3946304609F0F5F93946D2
:1069B000304608F0C9F94420084A2B46126821469F
:1069C0000090632008F07EF8002003B0F0BD00BF07
:1069D0005C74010034740100AC0B0020B00B00208B
:1069E00026232DE9F0411A4A1A4D1B4C82B0126839
:1069F0002146009363202B4608F064F807F04AFB19
:106A0000804607F04BFB0746FDF79CFB0646014618
:106A1000404609F0DDFB09F005FC3146384609F037
:106A2000D7FB09F0FFFB07F0E7FA0646807BFDF78E
:106A3000EDFB3046FEF7C0FF3520084A2B461268B2
:106A400021460090632008F03DF802B0BDE8F081D7
:106A5000AC0B00205C7401001C740100B00B002022
:106A60002DE9F04383B000F0CDF8814600F0CEF878
:106A7000804600F0D3FC074600F0D4FC72230646A3
:106A8000134D144C144A21461268632000932B4680
:106A900008F018F809F0EEFD09F020FC484609F06E
:106AA0006FFB404609F06CFB384609F069FB304645
:106AB00009F066FB00F014FD7F20084A2B4612689F
:106AC00021460090632007F0FDFF03B0BDE8F0838E
:106AD000887401007C740100AC0B0020B00B002016
:106AE0002A232DE9F047214A214D224C82B0126819
:106AF0002146009363202B4607F0E4FFFDF722FBBD
:106B000006460EF0FBFD00F07DF8824600F07EF8B0
:106B1000074600F083FC814600F084FC804600F0CC
:106B20007DF8CAF80D0000F075F8C7F80D0000F008
:106B300079F8C7F8090000F061FCC9F80D0000F011
:106B400061FCC8F80D00304600F08EFC304600F0C5
:106B5000A9FC3D20084A2B4612682146009063207C
:106B600007F0B0FF02B0BDE8F08700BFAC0B00201B
:106B70008874010070740100B00B002008B50EF09D
:106B8000BDFD431E1D2B15D8DFE803F01A1A1A1499
:106B90000F1E141414141414141414141A1A142593
:106BA00014142525141425251A160D4A136C23F0E8
:106BB00001031364012008BD00F030FA012008BD74
:106BC00000F034F8012008BD054A0120136C43F0A1
:106BD0000103136408BD00F0B3FC012008BD00BF31
:106BE0000000025010B5064C04F11000FDF7AEFA9B
:106BF000207504F11800FDF7AFFA2077204610BD8C
:106C0000C0000020004870476C000020004870471A
:106C10005400002000487047E800002000487047FA
:106C2000A800002000487047E0140020C9222DE988
:106C3000F04FADF5B55D83B08D4B00921A688D496C
:106C40008D4B06460890632007F03CFFFFF7CAFF14
:106C500005460990FDF776FA0446024629460120CA
:106C600009F030FA22462946022009F02BFA214683
:106C7000824809F0ADFA09F0D5FA2146804809F0BA
:106C8000A7FA09F0CFFA4FF480620021AAA80FF00A
:106C900078FF4FF4006200210DF5D5600FF071FF11
:106CA0004FF40062FF210DF6A8600FF06AFF2AA8DA
:106CB0004FF400727F210FF064FF1D2E00F0D3808F
:106CC0004FF01D094D46089B03F1FF3B5FFA8BF324
:106CD000079309F081FC4FF0040809F0B5FC00248B
:106CE0004FF48572654B6748D3F80910644BCF6841
:106CF000D3F8093060499E683B46049103900592A1
:106D0000CDF8008020220F217220CDE9014407F048
:106D100091FE40F20B1258495B4BCDF80080049174
:106D2000039305923346CDE90144202201217220CC
:106D300007F080FEAAAB9946A7F1040A0DF1A80856
:106D40000DF5D56C0DF6A86E5746002457F8040FC4
:106D50000346BBF11C0F1CD8DFE80BF00F14601BBF
:106D60001B1B1B1B1B1B1B1B1B1B1B1B0F0F1B1B8B
:106D70001B1B1B1B1B1B1B1B490056F82430C31A73
:106D800023EAE3735CF8242013444CF82430002DEC
:106D90005CD00134202CD9D14B46403308F1200877
:106DA0009946A2AB98450AF1800A0CF1800C0EF1CD
:106DB000800EC9D115F1FF358BD20BA83A220021E4
:106DC0000FF0DFFE089B033B1A2B00F2B480DFE8D4
:106DD00003F05FB2B2B2B2B2B2B2B2B2B2B2B2B257
:106DE000B9B9B2B2B2B2B2B2B2B2B2B2AA0056F845
:106DF00024105CF82420411A0029A8BF52184CF82E
:106E00002420002DC5D1214BA3FB02321209312AC7
:106E10004CF82420BDD8ADF8A852BAE75CF824207D
:106E20005EF82430824238BF0246834228BF0346C0
:106E3000D11AB1F57E7F2CBF7F2141F3C7014CF8F9
:106E400024204EF8243008F80410A2E70F4AA2FBD1
:106E50000323079A1B09012A96BF4A464CF824309F
:106E600022F8143095E70123ADF8A83228E700BFD7
:106E7000AC0B002094740100887601006C000020A7
:106E80005400002094760100A0760100898888884B
:106E900020260F2701230DF1A80C1AAD002243F084
:106EA00080032F70AC700DF12C0E6B716E7017AFEC
:106EB000EA702A71AC1D76460FCEBE42206061603A
:106EC000A260E3600EF1100E04F11004F3D17346DA
:106ED00003CB206061601B886146238128460EF049
:106EE00013FC09F0C7FB09F0F9F9474809F048F924
:106EF000464809F045F9099C0120214609F030F97E
:106F00002146022009F02CF94FF4D572404B009233
:106F10001A684049404B632007F0D4FD0DF5B55D7C
:106F200003B0BDE8F08F01240DF52A7C26462746E4
:106F300002231AADB2E70DF52A7C20260F27022383
:106F40001AADABE7089B112B52D04FF00E080DF194
:106F5000280C4746E2462026012100231AAD0E22C6
:106F60009646114403EB41110DF5D56303EB810106
:106F7000CCF800200DF6A8590DF5C56B1F2007941D
:106F8000286017E059F8202051F8204051F82030AF
:106F90001344A21A4FF47A745B10012BB8BF01237B
:106FA00004FB02F292FBF3F32BF810300138431C80
:106FB00028600BD0DAF800304345E3DB4FF00003E4
:106FC0002BF810300138431C2860F3D10EF1FF3E3E
:106FD000BEF1FF3F079CCCF800E0A1F18001A9F1D0
:106FE0008009ABF1400BC9D10DF52A7C022355E78E
:106FF0004FF01F081AAD4646AA46002101230F276D
:107000000DF1280CABE700BF6C00002054000020FD
:10701000B00B0020947401008876010009222DE94C
:10702000F04F0026ADF65C1DD24B00921A68D24993
:10703000D24B63200DF1740B07F044FD3146E22280
:1070400058460FF09EFDADF83460FFF7DBFD81463A
:107050000790FFF7C7FD0746FFF7D8FD8046089069
:10706000FDF770F8054631464FF4006256A80FF060
:1070700088FD2A463946012009F024F82A46394677
:10708000022009F01FF82946484609F0A1F809F046
:10709000C9F82946404609F09BF809F0C3F80123D6
:1070A0003446B2461D26DFF8F482ABF8003009F012
:1070B00093FA09F0C9FA3F22079B0027D3F8091079
:1070C000089BCD68D3F80930AC49D3F808900592F5
:1070D0000422AB482B460491039000920F212022FA
:1070E0007220CDE9017707F0A5FC0423402200932C
:1070F000A249A44B0491039305924B46CDE9017735
:1071000020220121722007F095FC7C35A9F1040EA4
:107110000DF5AC79A5F18000F4464946234603E01D
:10712000854226D051F8043F50F8044F5CF8042FF4
:10713000A41A002CACBF1C191C1C0C60002EEFD133
:10714000A8FB04342409312C0C60E9D8BAF10E0FE5
:10715000ABF8006005D80AF1010A5FFA8AFA2BF849
:107160001A7001370F2F05F180050CD059F8804FA8
:10717000D0E701370F2F05F18005F7D116F1FF3663
:1071800001D3569C93E709F0A9F8079808F0F8FF97
:10719000089808F0F5FFFCF7D5FFBC220021064651
:1071A00056A80FF0EEFC00F039F9054600F03AF968
:1071B000044600F02BF9C5F80D0000F02BF9C4F8D7
:1071C0000D0000F033F9C5F8010000F03DF9C4F8F6
:1071D0000100D5F801103246052008F073FF324651
:1071E000D4F80110062008F06DFF3146204608F063
:1071F000EFFF09F017F83146284608F0E9FF09F0DB
:1072000011F829463046604A0AF04AF821465E4A9B
:1072100030460AF059FB0F2320224FF00308D5F81F
:1072200009100891D4F80910CDE90E230AF10103E1
:10723000099107930021287809F02CF9524A294630
:1072400030460AF02DF85149287809F023F9002139
:10725000207809F01FF94C4A214630460AF034FBE9
:1072600020784B4909F016F94FF0010200274FF042
:10727000200C089B5868079B2BF81320002255AB65
:1072800003EBC711434B043803EB471E0B944C68C8
:1072900050F8043F234441F8043FB8F1000F00F0D8
:1072A000858001326245F2DB0B9C002F78D018F10B
:1072B000FF38BFD209F012F8284608F061FF2046D7
:1072C00008F05EFF3A2200210EA80FF05AFC0023BE
:1072D00007220A254FF4024E4FF0050C09260B2019
:1072E0000C21ADF858318DF85A318DF85B31ADF87D
:1072F0003A209DF835309DF83420ADF83C70ADF85B
:107300004470ADF842500EACADF840A0ADF85CE171
:107310008DF838C0ADF83E60ADF84600ADF84A10C3
:10732000ADF84820ADF84C300DF5AF751AAF2646D4
:107330000FCEBE4228606960AA60EB6004F11004C1
:1073400005F11005F3D1234603CB286069601B8843
:10735000594656A82B810EF0D7F9D7220E4B009232
:107360001A680549054B632007F0ACFB0DF65C1D60
:10737000BDE8F08FAC0B0020A4760100B8760100C8
:1073800094760100A0760100D9050100C91401001E
:10739000AD1A010038770100B00B00208988888879
:1073A000099BDDF83CC00127586867E71EF802908A
:1073B00042F20F74B9F1000F08BF4FF07F099B082C
:1073C00003FB09F3DB09A3420B603FF66AAF4FF002
:1073D00000090DABDB5D079C0A930A9B2BF8149008
:1073E00001330DF1340909F807309DF834309DF868
:1073F000359023444B442BF8132052E70048704744
:10740000F0000020004870475001002000487047FD
:107410006801002000487047800100200048704744
:1074200020010020004870473801002010B5054CAD
:1074300004F10C00FCF78AFEE36820752361204606
:1074400010BD00BFB402002010B5064C04F10C00C2
:10745000FCF782FE207504F11000FCF783FE204645
:1074600010BD00BF2C03002038B50A4C41780A4AF1
:107470008D0020460FF026FA2946201D074A0FF0FE
:1074800021FA294604F10800054ABDE838400FF00A
:1074900019BA00BFB001002078770100947701008D
:1074A000B077010038B50A4C01780A4A8D002046B1
:1074B0000FF008FA2946201D074A0FF003FA294663
:1074C00004F10800054ABDE838400FF0FBB900BFE1
:1074D00014020020D8770100F47701001078010031
:1074E00038B50F4D0F4928460FF078FA0E4C281D7D
:1074F0000E490FF073FA05F108000D490FF06EFA0E
:1075000020460C490FF06AFA201D0B490FF066FA6D
:1075100004F108000949BDE838400FF05FBA00BF28
:10752000B001002078770100140200209477010058
:10753000B0770100D8770100F477010010780100DE
:1075400040F2B9222DE9F04FBB4BADF5397D0092E9
:107550001A68BA49BA4B04460790632007F0B2FA9A
:10756000FCF7F0FDBC220B9000215AA80FF009FB9C
:107570005E22FF2142A80FF004FB89A8BC22002153
:107580000FF0FFFA1B2C00F01082079B1C2B00F061
:107590006982079B142B17AB0E9300F03F811846AE
:1075A0002F2200210FF0EDFAA64CDFF8ACB2A64A6C
:1075B000DFF8A8A2A54B04F10C00CBF80D20CAF807
:1075C0000D30FCF7C3FDA24DE368207505F10C00FA
:1075D0002361CBF80140FCF7BFFD287505F11000D1
:1075E000FCF7C0FD0B9CDBF8011022460520CAF811
:1075F000015008F067FD2246DAF80110062008F075
:1076000061FD2146504608F0E3FD08F00BFE2146DF
:10761000584608F0DDFD08F005FEDBF809300F9351
:10762000DAF809301093079B172B00F09C81042394
:107630000D93012320210F2240F29110D846079C80
:10764000CDE91512143CE4B2A3401840DDF83490A3
:1076500003F0080306940890099319F1FF3968D3E1
:10766000069B082BF9D8089B002B40F0FD80099B56
:10767000002BF2D008F0B0FF089C0A9408F0E4FF59
:107680000C940AF0CDFA2123CDE91198834698464F
:10769000CDF84CA00C9B15AA52F82340002C3AD0F0
:1076A00040F24D3A4FF000090A9BE718E518BF0079
:1076B0005AABDE1989AB1F4442AB03EB45050BEB1C
:1076C00084045F4A04230492624A0121CDE90292B4
:1076D0000122CDF814A0CDE9003272205B4642466B
:1076E00007F0A8F954F8043D56F8041D35F8022DAA
:1076F0008B4238BF0B46336021688A42A8BF0A46D6
:1077000091B25B1AFD2B8CBF7F235B085C452A80FE
:1077100047F8043DD5D10A9B20330A930C9B002BDC
:1077200000F01681DDE9119819F1FF39DDF84CA060
:1077300096D2079BC346172B00F012811C2B00F03A
:10774000F08100245AAF3A22002123A80FF019FA41
:10775000042100224FF0020C4FF005084FF0010900
:107760004FF0200E0F2503209DF8CD30ADF892C0CC
:1077700061F3060364F3C71323AE8DF88C80ADF874
:107780008E90ADF890E0ADF89450ADF896008DF87D
:10779000CD30ADF89A10ADF8C8208DF8CA208DF81C
:1077A000CB208DF8CC200DF1CE040DF1BC0C35466C
:1077B0000FCD654520606160A260E36006F11006B0
:1077C00004F11004F3D103CE2060616033883946A0
:1077D000238132A80DF098FF08F04CFF08F07EFDE1
:1077E0001D4808F0CDFC1D4808F0CAFCDBF801106C
:1077F000052008F0B5FCDAF80110062008F0B0FC0E
:1078000040F28F32164B00921A680C490C4B6320E1
:1078100007F058F90DF5397DBDE8F08F1C46114D84
:107820000FCD0FC40FCD0FC495E80F0007C41A0C7D
:1078300024F8023B2270B7E6AC0B0020C8760100AA
:1078400068770100D8010020F000002050010020DE
:107850003C02002074770100200100203801002044
:10786000B00B0020D8760100002198F8000008F045
:1078700011FE00219AF8000008F00CFE079B1C2B5B
:1078800000F0E4800B9CAF4AAF49204609F008FDA8
:10789000AC4AAE4920460AF017F84D46AC4998F874
:1078A000000008F0F7FDAB499AF8000008F0F2FD7F
:1078B000159C0F9B04F180410139586889000B1D0C
:1078C0005AAA1144184414F1FF3417D30B6850F826
:1078D000042D134441F80439002DF4D10E9A0D9E65
:1078E000125DB3FBF6F3002A08BF7F2203FB02F30D
:1078F00014F1FF344FEAD3134B60E7D2169C109B70
:1079000004F11F0059688000A0F17C035AAA1044BA
:10791000194414F1FF3419D3036851F8042D1344AA
:1079200040F80439002DF4D10E9A0D9E224492F8AD
:107930002020B3FBF6F3002A08BF7F2203FB02F3EB
:1079400014F1FF344FEAD3134360E5D2A94684E62D
:107950000AF098F9012383460C934FF0140899E636
:1079600089AF0124EFE600219BF8000008F092FDAA
:1079700000219AF8000008F08DFD0B9C714A5946D1
:10798000204609F08DFC6F4A5146204609F09CFFC5
:107990006F499BF8000008F07DFD6E499AF80000E1
:1079A00008F078FD1E230D9343E617AB1C466A4D85
:1079B0000E930FCD0FC40FCD0FC495E80F0007C471
:1079C000664EDFF884B16649DFF880A1654A24F885
:1079D000023B1B0C237006F10C00CBF80D10CAF80B
:1079E0000D20FCF7B3FB604CF368307504F10C001C
:1079F0003361CBF80160FCF7AFFB207504F1100098
:107A0000FCF7B0FB0B9DDBF801102A460520CAF8F5
:107A1000014008F057FB2A46DAF80110062008F06A
:107A200051FB2946504608F0D3FB08F0FBFB2946E2
:107A3000584608F0CDFB08F0F5FB04230D93DBF866
:107A400009300F93DAF809301093F2E50B9C474A9E
:107A500020463D4909F024FC444A3C49204609F0AF
:107A600033FF1AE717AB1C46414D0E930FCD0FC4E1
:107A70000FCD0FC495E80F0007C43E4EDFF8C8B025
:107A8000DFF8C8A03C493D4A24F8023B1B0C237098
:107A900006F10C00CBF80D10CAF80D20FCF756FBD0
:107AA000374CF368307504F10C003361CBF801609A
:107AB000FCF752FB207504F11000FCF753FB0B9D03
:107AC000DBF801102A460520CAF8014008F0FAFA4E
:107AD0002A46DAF80110062008F0F4FA2946504642
:107AE00008F076FB08F09EFB2946584608F070FB2C
:107AF00008F098FB00224FF04053DBF809100F917B
:107B0000DAF80910109183F84020FCF70FFF0120EC
:107B1000FCF7D4FF04230D9308F042FD08F094FD18
:107B200087E54FF04053012240F24C4083F840205B
:107B3000FDF770FA00205AAFFCF7C0FF0024FCF7F5
:107B4000EDFE00E6D90501002001002038010020EB
:107B5000C9140100AD1A010038770100B4020020F9
:107B600068010020800100202C030020A1050100F5
:107B70000877010078020020980100200801002009
:107B8000F00200200048704768030020004870475A
:107B9000AC03002000487047B8030020024A80214F
:107BA00002480EF08FBE00BF38780100FC140020A0
:107BB000014902480EF012BF38780100FC14002081
:107BC000014B1868704700BFFC1400200048704744
:107BD000C003002000487047F403002010B506F0F1
:107BE00059FA06F05BFA044606F006FB06F006FCBE
:107BF000D4F80940FFF7DCFF0023E360BDE8104044
:107C0000F9F782BD38B506F045FA054606F046FAA2
:107C1000044606F0F1FA06F0F1FB08F05FFB284697
:107C200008F0AEFA2046BDE8384008F0A9BA00BF17
:107C300040F20E53F0B5144A144D154C83B012683F
:107C40002146632000932B4606F03CFF08F012FD0E
:107C5000FFF7D8FF06F01EFA06F020FA06460027C6
:107C600006F0CAFA06F0CAFB40F21350D6F80960D3
:107C7000084BF7601A68214600902B46632006F0F7
:107C800021FF03B0F0BD00BFAC0B0020687A0100FB
:107C9000B4780100B00B00202DE9F04FADF22C6D4F
:107CA00000260127F9F74EFD4FF0040B40F2232286
:107CB000C94CCA4DCDE901763946209020AB0592DA
:107CC000CDF800B03A46CDE90354642006F0B2FE88
:107CD0004FF40971C24A2346126863200091C149DA
:107CE00006F0F0FEFCF72EFA21960DF019FB037F4B
:107CF0001D9006F0CFF9D0F80930394602201B93C9
:107D000008F0B8FAD0F80950804608F0DDFC1020E1
:107D1000FCF7FAFD40F25129DFF8F0E280EA070CA7
:107D2000CDF81490CDF80CE03A463946CDE901661D
:107D300000970DF17F03642004948DF87FC006F056
:107D400079FE40F253220221A74BCDE9016605924C
:107D5000009103932022A54B0F216220049406F08A
:107D600069FE4FF415711B9A7220D368A04ACDE9C1
:107D70000176CDF800B0059103920F2120220494E2
:107D800006F058FE31463E220DF272200EF0F9FE4A
:107D90004FF0200A42F20F0E4FF0840C1B9A022083
:107DA000D3689CA9324600933346ADF870E28DF853
:107DB00075C28DF872A20DF027FC31469A220DF59E
:107DC0009E600EF0DEFE31469A220DF28C500EF0CF
:107DD000D8FECDE935663796FFF7D4FE31461C90C4
:107DE0004022ACA80EF0CDFE0DF1940931461E22C2
:107DF00054A80EF0C6FEC9F80060A9F804608DA86A
:107E0000FCF7A4F9CCA8FCF7A7F9D8F80D308D9AA7
:107E10005B6851461878AB6804920DF58E62039248
:107E2000FCAA02922A680192EA6800921A22FAF7E2
:107E3000DDFF4FF4437C6F48EB685246CDE9017695
:107E40003946CDF800B0CDF814C0039004946220F8
:107E500006F0F0FD4FF4447CD8F80D2066485268D7
:107E6000AB681178CDF814C05246CDE90166CDF863
:107E700000B003900494722006F0DCFD40F2113053
:107E800002222B6805905D48CDE9017639460092C3
:107E9000039052466620049406F0CCFD29685046B3
:107EA0000A22FBF779F940F2163CDFF86481CDF83D
:107EB00014C0CDE900B73A4639460296229022AB6B
:107EC0006E200494CDF80C8006F0B4FD504629686D
:107ED000DCAB1E22FBF78CF9229BEC90B342B8BFBF
:107EE0001F335B1186B29FB228826B823E22F31B46
:107EF00000210DF2F220A9F80270A9F80430A9F8C7
:107F000000600EF03EFE002340F201304FF0020A06
:107F10004FF0030B1A46BCA9ADF8F002CDF8009063
:107F20001220012600278DF8F5A28DF8F2B20DF08F
:107F30006BFB40F2353231492B686E20CDF800A042
:107F400003910592314620220494CDE9016706F0A1
:107F500071FD4FF0040A40F2363332463146059344
:107F60006E2022ABCDE90167CDE90384CDF800A0F6
:107F700006F060FD40F23730214B32460590039306
:107F8000CDE90167ECABCDF800A0049431466E203A
:107F900006F050FD229B1B4A462B44DD13683344F8
:107FA0005B45136002DD8DF884B0176040F2075224
:107FB000154B00921A680B49074B632006F082FDAF
:107FC0000020219BDAB262F30700C3F3072262F3B9
:107FD0000F20C3F307421DE0687A0100C878010052
:107FE000AC0B0020A4780100E07801000000846060
:107FF0001C790100307901004879010060790100A5
:108000007879010004150020B00B0020D47801001D
:108010007C79010062F317401B0E63F31F600DF2C1
:108020002C6DBDE8F08F0F2B176040F32F830020DD
:108030000025FCF7F1F80126022740F27733DFF83C
:1080400008A4CDE90443CDE901654FF0C1432022E6
:108050000F2169200097CDF80CA006F0EBFC0DF580
:10806000A463CDE900354FF0C1420DF24653202103
:108070000F20FAF739FD0DF59E60FCF761F940F22B
:108080008233CDE9025ACDE9044320224FF0C143A7
:108090000F216920CDE9007606F0CCFCBDF916C5AC
:1080A000BDF91435BCF1000FB8BFCCF1000C002BAA
:1080B000B8BF5B429C4540F28B32B8BF9C46D9F8B2
:1080C0000000CF49B9F804E00DF1A408CDE901554D
:1080D000CDF8A600434605920391324631466E2004
:1080E00000970494ADF8AAE0ADF8A4C0ADF8AC5088
:1080F00006F0A0FC4FF4637CC248CDF814C0CDE973
:1081000001550DF1A60332463146039000976E20CB
:10811000049406F08FFC40F28D30BB4BCDE9015545
:1081200032463146059003936E202AAB00970494A3
:1081300006F080FC40F28E30B44BCDE9015532465A
:108140003146059003936E200DF1AA030097049425
:1081500006F070FC29463E220DF232300EF011FD81
:1081600040F2014E4FF0040C2B462A46CCA91D20AC
:10817000CDF80080ADF830E38DF832C38DF835735B
:108180000DF042FA2946202264A80EF0FAFC294696
:108190008022FCA83A95CDE93855CDF8EB500EF089
:1081A000F0FC29463C227EA80EF0EBFC9A220DF54D
:1081B0009E610DF28C500EF0D9FC35A90DF28C5059
:1081C000FDF79AFD4FF47073CDE9025ACDE90443EF
:1081D000CDE900764FF0C14320220F21662006F042
:1081E00029FC1C9B93F83250002D00F02F825CAFCD
:1081F00040220021DCA80EF0C4FC38461E220021DB
:108200000EF0BFFC00209DF8DF209DF8DE309DF8C9
:10821000DD1062F3070063F30F209DF8DC201B9B49
:1082200061F3174062F31F60DCAA9B690F2100977E
:1082300001922022FAF71AFC012500264FF0020ACB
:108240004FF47D72724BCDE904422946CDF800A06F
:1082500003932022DCAB5320CDE9015606F0EAFB64
:1082600040F2F5304FF050094FF02808694A3B467C
:10827000CDF800A029460590039253200F22CDE9A6
:108280000156049406F0D6FB0DF58E63DCA96CAAAA
:10829000CDE900892020FBF787FA82464FF47F70F2
:1082A0005D4A6CAB2946059003924C202022CDE913
:1082B00001660095049406F0BDFB39468DAB3CAADF
:1082C000CDE900890F20FBF76FFA07464FF4806075
:1082D000524A3CABCDE904400392CDE901660F223E
:1082E000009529464C2006F0A5FB4D4B1A68002A44
:1082F00000F09D81642A06D1BAF1010F40F3E581B7
:1083000000210A46196047490B680133062BC2BF9A
:108310000020034608604FF00000D8BF0B604249C0
:1083200041F823200B1F183153F8042F002AC8BF2F
:1083300001308B42F8D10428D4BF3C4E3C4EECAD0A
:108340000FCE0FC53368ECA82B60D4BF4FF0000AE6
:108350004FF0640A0BF020FF3E2200210DF2B230F4
:108360000EF00FFC00234FF0C14242F20F008221B9
:1083700020271D464FF001080F260092ADF8B003EC
:108380001A468DF8B5130320ECA98DF8B2730DF0E1
:108390003BF927A8BDF8B015CDF89E50ADF89C80EC
:1083A0008DF8A060FCF70EF840F25240214B3A469F
:1083B0003146CDE9044003936C201F4BCDF800807B
:1083C000CDE9015506F036FBFCF726F81D28239071
:1083D00003DCFCF727F800285FD040F25642174B29
:1083E000009217490022642006F06CFB0025012250
:1083F00040F257410420134BCDE9044126E000BF71
:10840000887901009C790100B0790100C4790100EC
:10841000EC790100FC7901000C7A01001C7A010062
:10842000081500203C04002080200020487801002E
:108430005C780100A485010000008160687A010079
:108440002C7A0100306E010070790100CDE9012520
:10845000114600900393642023AB06F0EBFAFBF780
:10846000D1FE064602E0062D00F0DD80013506FA59
:1084700005F080B2FBF7C2FEBDF8B01527A8FBF7E8
:10848000A1FFFBF7C9FF1D282390ECDCFBF7CAFF17
:108490000028E8D13046FBF7B1FE002774AE4FAD9F
:1084A00039460DF1B0080DF1BC092822304640973D
:1084B00041974297439744974597469747974897E0
:1084C00049974A974B974C974D974E97C5E9007738
:1084D000C5E902772F61C8E90077A8F80870C9E9F3
:1084E0000077A9F808700EF04CFB4FF0C143CDE9BE
:1084F0001677CDE914770E970C9707970DF59E67C1
:1085000012970DF28C5711971C9F239910977EAFED
:108510000F97FCAF0D9738AF704A0B9764AFDFF839
:10852000D4C10A9754AF0691049305924AAB45AA69
:1085300040A90997CDE90296ACAFCDE900580A20D1
:108540000897CDF860A0CDF84CC0F9F7A7FD9DF8CD
:108550007F10229A002914BF20231E230746F9F713
:1085600041FD002840F0AD801D9BDB7B002B40F0DF
:10857000A88038460521F9F7B7F810B102238DF825
:1085800084304FF0000A32AFCDE900872B464AAA6B
:1085900045A940A8C7E900AAA7F808A00AF074FFF7
:1085A0002B464AAA45A940A8CDE9008909F0B4FDA7
:1085B000CDE90168CDE905AACDE9039748480095C2
:1085C00005684AAB45AA40A90A20A847012540F200
:1085D000F94240F2FA46434BCDE9044229462A4685
:1085E000039365204346CDE901AA009506F022FADF
:1085F0003D482A460390CDE901AA009504943B46E4
:1086000029460596652006F015FA0DF1D20217F8F5
:10861000013B0BB188F800A0BA4208F10108F6D17D
:10862000F9F788F8C2E43046FBF7E8FDBEE4BAF19A
:10863000010F7FF468AE012F7FF465AEBDF9B01570
:1086400095293FF760AE64221A605CE61E46DDF8AD
:10865000FC141A464942DDF8F404F9F773FC96F865
:108660003030002B3FF4C3AD40F2CA321F4B0092B2
:108670001F492A46642006F025FA1C9B284683F8E9
:1086800030500CF057FE8DF88670B0E5F9F75AF8C7
:10869000EB680DF58E62CDE904231C9D0146B5F90A
:1086A0001A300393B5F918203B460292B5F916002B
:1086B00013220190B5F91450202000950AF068F8B3
:1086C000B5E401238DF8853053E7012F3FF718AE4D
:1086D000BDF9B015C8297FF716AE11E6000081601C
:1086E00014240020547A01005C7A0100687A0100A9
:1086F000D8790100707A010038B505F0CBFC054649
:1087000005F0CCFC044605F077FD05F077FE05F09A
:10871000CBFDFFF73BFAC5F80D00FFF73BFAC4F8B5
:108720000D0038BD70B505F0B5FC064605F0B6FC89
:10873000054605F061FD05F061FEFBF703FD04460B
:108740000146304607F044FD07F06CFD21462846FF
:1087500007F03EFDBDE8704007F064BD4FF4FF73C5
:10876000F0B52A4A2A4D2B4C83B01268214600935B
:1087700063202B4606F0A6F905F08CFCFFF7BCFF42
:1087800005F088FC05F08AFC064605F035FD05F08D
:1087900035FED6F80960FFF713FAF06005F07AFCB1
:1087A000074605F07BFC05F027FD05F027FEFFF7E7
:1087B000E9F90646FFF70AFAFFF70CFA4FF4807161
:1087C00038463162FDF7EEF8FFF7ACFF124B134E5F
:1087D0000FCBFBF7F3FC1248FDF7D4F93046F8F75E
:1087E0003DFF06F5DC700AF08FFB642007F0A2FE67
:1087F000F8F79AFF4FF407700A4A2B461268214691
:108800000090632006F05EF903B0F0BDAC0B0020D1
:10881000687A010094780100A07C0100707A010060
:10882000B07C0100B00B00204FF4F073F0B5194A92
:10883000194D1A4C83B012682146064600936320F6
:108840002B4606F03FF9FFF757FF05F023FC05F034
:1088500025FC074605F0D0FC05F0D0FDD7F80970DF
:10886000FFF79CF9FFF7ACF9F860FFF75BFF05F045
:1088700015FCF1B2FDF7FEF8FFF7C4F94FF4F47000
:10888000074A2B46126821460090632006F01AF929
:1088900003B0F0BDAC0B0020687A010070780100D5
:1088A000B00B00204FF4F77330B50F4A0F4D104C4A
:1088B00083B012682146009363202B4606F002F92C
:1088C0000220FFF7B1FF0B48F8F7C8FEF8F71CFFCE
:1088D0004FF4FC70084A2B46126821460090632032
:1088E00006F0F0F803B030BDAC0B0020687A010050
:1088F00084780100707A0100B00B002000487047B6
:10890000400400200048704784040020004870475D
:1089100090040020024A802102480DF0D3BF00BF1E
:10892000387801000C150020014902480EF056B8B5
:10893000387801000C150020014B1868704700BF03
:108940000C1500200048704798040020004870472C
:10895000CC04002010B5F8F7D7FE05F09BFB05F01E
:108960009DFB044605F048FC05F048FDD4F809409D
:10897000FFF7DAFF0023E36010BD00BF38B505F054
:1089800089FB054605F08AFB044605F035FC05F039
:1089900035FD07F0A3FC284607F0F2FB2046BDE8B2
:1089A000384007F0EDBB00BF40F2DA43F0B5144A9F
:1089B000144D154C83B012682146632000932B465A
:1089C00006F080F807F056FEFFF7D8FF05F062FBCF
:1089D00005F064FB0646002705F00EFC05F00EFDD1
:1089E00040F2DF40D6F80960084BF7601A6821466C
:1089F00000902B46632006F065F803B0F0BD00BF81
:108A0000AC0B0020147D0100007D0100B00B0020A4
:108A10002DE9F04FADF2D45DF8F794FE0024012665
:108A200004271D90FBF78EFB40F23522CF4DD04836
:108A3000CDE9016431461DAB059200973246CDE980
:108A40000305642005F0F6FF40F23621C94A2B46A3
:108A5000126863200091C84906F034F81E940CF0A7
:108A60005FFC037F05F016FB3146D0F809B0022009
:108A700007F000FCD0F80970824607F025FE1020B0
:108A8000FBF742FF40F26228DFF810E380EA060CB1
:108A9000CDF80CE032463146CDE9014400960DF1A7
:108AA0007303CDF81480642004958DF873C005F02D
:108AB000C1FF4FF4197205920222B04BCDE9014477
:108AC000009203932022AE4B0F216220049505F003
:108AD000B1FF40F265210420AA4ADBF80C30CDE951
:108AE00001640090059103920F21202272200495C9
:108AF00005F0A0FF21463E220DF25A200EF041F86B
:108B00004FF0200842F20F0E4FF0840CDBF80C30CF
:108B1000224600930220234696A9ADF858E28DF82C
:108B20005DC28DF85A820CF06FFD21469A220DF538
:108B300093600EF026F821469A220DF234500EF082
:108B400020F8CDE92F443194FFF7D8FE21461B9041
:108B50004022A6A80EF015F80DF1880921461E2224
:108B60004EA80EF00EF8C9F80040A9F8044078A805
:108B7000FBF7ECFA87A8FBF7EFFADAF80D30789AF2
:108B80005B6841461878BB6804920DF583620392D6
:108B9000E6AA02923A680192FA6800921A22FAF75B
:108BA00025F94FF4467C04227748FB683146CDE92D
:108BB00001640092CDF814C04246039004956220EF
:108BC00005F038FFDAF80D204FF4477C52686F4803
:108BD00011780422BB68CDF814C0CDE9014400929D
:108BE000039042467220049505F024FF40F21D30A8
:108BF0000222DFF8ACA13B683146CDE90164009266
:108C000005904246CDF80CA06620049505F012FFB1
:108C1000396840460A22FAF7BFFA40F2223C0423A0
:108C20001F905B48CDF814C032463146029401963D
:108C3000009303901FAB6E20049505F0FBFE4046A9
:108C40003968C6AB1E22FAF7D3FA1F9A83B2A24242
:108C5000B8BF1F32521194B21E1BD6900021388229
:108C60007A820DF2DA203E22A9F80240A9F80460C7
:108C7000A9F800300DF085FF002340F201340226F0
:108C80004FF003081A46CDF80090B6A91220994675
:108C9000ADF8D8428DF8DA8201248DF8DD620CF04F
:108CA000B3FC40F241323B682146CDE903A5059271
:108CB0006E2020220096CDE9014905F0BBFE4FF061
:108CC000040A40F24233324A214603920593224677
:108CD0001FAB6E20CDE901490495CDF800A005F049
:108CE000A9FE40F243302B4B05900393CDE9014997
:108CF000D6ABCDF800A00495224621466E2005F0A3
:108D000099FE1F9B322B00F3B4821E2B40F3298166
:108D1000214B1E6000200024FBF77EFA012702266B
:108D200040F27733DFF87C80CDE90453CDE901745C
:108D30004FF0C14320220F2169200096CDF80C800E
:108D400005F078FE0DF59963CDE900344FF0C1428E
:108D50000DF2EE4320210F20F9F7C6FE0DF59360CA
:108D6000FBF7EEFA40F282331EE000BF147D0100F3
:108D7000C8780100AC0B0020F07C0100E078010015
:108D8000000084601C7901003079010048790100FD
:108D90007C7901007879010000050020D478010079
:108DA0006079010070790100CDE90248CDE90453F2
:108DB00020224FF0C1430F216920CDE9006705F063
:108DC00039FE214620225EA80DF0DBFE21468022DE
:108DD000E6A83494CDE93244CDF8D3400DF0D1FE6D
:108DE00021463C2278A80DF0CCFE9A220DF5936125
:108DF0000DF234500DF0BAFE2FA90DF23450FCF7ED
:108E00007BFF40F2A233CDE90248CDE90453CDE91E
:108E100000674FF0C14320220F21662005F00AFEB3
:108E20001B9B93F83240002C00F0478256AF402243
:108E30000021C6A80DF0A5FE38461E2200210DF027
:108E4000A0FE00209DF8C7209DF8C6309DF8C510F3
:108E500062F3070063F30F209DF8C42061F317400D
:108E600062F31F60C6AADBF818300F210097019249
:108E70002022F9F7FBFD012400264FF0020A40F200
:108E8000D6324B4BCDE904522146CDF800A00393D6
:108E90002022C6AB5320CDE9014605F0CBFD40F2C0
:108EA000D7304FF050094FF03208424A3B46CDF8D8
:108EB00000A021460590039253200F22CDE90146E0
:108EC000049505F0B7FD0DF58363C6A966AACDE943
:108ED00000892020FAF768FC824640F2DE30364AEC
:108EE00066AB2146059003924C202022CDE9016615
:108EF0000094049505F09EFD394687AB36AACDE96E
:108F000000890F20FAF750FC074640F2E2302B4A66
:108F100036ABCDE904500392CDE901660F220094EF
:108F200021464C2005F086FD254A1368002B4BD0C6
:108F3000642B54D1BAF1010F40F3DF810023136099
:108F400064204623002401214FF46172D890D6A8F2
:108F5000D994D693D7938DF86413DA920BF01CF959
:108F60004EE018490A68002AC6BF02F1FF320A60C3
:108F7000C1F800900F2B3FF7CDAEF8F7E3FBFB688D
:108F80000DF58362CDE904231B9C0146B4F91A3028
:108F90000393B4F9182000230292B4F916001322A7
:108FA0000190B4F914402020009409F0F1FBB1E6DF
:108FB000EC790100FC7901000C7A01001C7A0100B7
:108FC0001415002000050020BAF1010FB8D1012FBF
:108FD000B6D1BDF95835952BB2DC642313600A2055
:108FE00000260F243C21012240F6C413D790D6A8B6
:108FF000D996D694D8918DF86423DA930BF0CCF8F7
:109000003E2200210DF25A300DF0BBFD00234FF03F
:10901000C14242F20F00822120261C460127009205
:10902000ADF858031A468DF85D130320D6A98DF8C4
:109030005A630CF0E9FA24A8BDF85815CDF892400F
:10904000ADF89070FBF7BEF940F21E41AF4B3246CF
:10905000CDE9045103930F21AD4B6C200097CDE96E
:10906000014405F0E7FCFBF7D7F91D28209000F339
:10907000C880FBF7D7F9002840F0C38000276EAE08
:1090800049AC39460DF198080DF1A4092822304663
:10909000CDE93A77CDE93C77CDE93E7740974197E6
:1090A0004297439744974597469747974897C4E90F
:1090B0000077C4E902772761C8E90077A8F808704B
:1090C000C9E90077A9F808700DF05BFD4FF0C143C6
:1090D000CDE91777CDE9157714970E970C97079779
:1090E0000DF5936712970DF2345711971B9F209936
:1090F000109778AF0F97E6AF0D9732AF844A0B9772
:109100005EAFDFF834C20A974EAF06910493059222
:1091100044AB3FAA3AA90997CDE90296A6AFCDE99B
:1091200000480A200897CDF84CC0F8F7B7FF9DF823
:1091300073101F9A002914BF202303230746F8F752
:1091400051FF10B101238DF8793038460521F8F729
:10915000CBFA10B102238DF878304FF0000A2CAF13
:10916000234644AA3FA9CDE900873AA8CDE92CAA15
:10917000ADF8B8A00AF088F9234644AA3FA93AA856
:10918000CDE9008908F0C8FFCDE90168CDE905AA5D
:10919000CDE903975F480094046844AB3FAA3AA91D
:1091A0000A20A047012440F2C54240F2C6465A4B6D
:1091B000CDE9045221462246039365204346CDE97A
:1091C00001AA009405F036FC54483B462246039021
:1091D000CDE901AA6520009404952146059605F085
:1091E00029FC3B4642460DF1BA0013F8011B09B1B8
:1091F00082F800A0984202F10102F6D1F8F79AFA3B
:1092000039E040F22242464B009246490022642057
:1092100005F058FC0024012240F223410420424B77
:10922000CDE90451CDE90124114600900393642057
:1092300020AB05F0FFFBFAF7E5FF064601E0062C40
:1092400037D0013406FA04F080B2FAF7D7FFBDF840
:10925000581524A8FBF7B6F8FBF7DEF81D28209078
:10926000EDDCFBF7DFF80028E9D13046FAF7C6FF5E
:1092700004E78DF8788040F2D3422C4B00921A68B4
:109280002B49274B632005F01DFC00201E9BDAB202
:1092900062F30700C3F3072262F30F20C3F3074210
:1092A00062F317401B0E63F31F600DF2D45DBDE83F
:1092B000F08F3046FAF7A2FFDDE71F46DDF8A41471
:1092C0001A464942DDF89C04F8F73CFE97F8303026
:1092D000002B3FF4ABAD4FF46B72114B009215496C
:1092E0002246642005F0EEFB1B9B204683F83040AD
:1092F0000CF020F88DF87A6098E5012F3FF71EAE4C
:10930000BDF95835B42B7FF76AAE17E6A485010086
:109310000000816014240020547A01005C7A01006E
:10932000147D01002C7A0100306E0100B00B00208A
:10933000F07C0100D87901001C7D010038B504F0F3
:10934000A9FE054604F0AAFE044604F055FF05F008
:1093500055F8FFF7D7FAC5F80D00FFF7D7FAC4F8AC
:109360000D0038BD70B5FAF7EDFE044604F092FE2C
:10937000064604F093FE054604F03EFF05F03EF875
:109380002146304606F024FF06F04CFF21462846D1
:1093900006F01EFFBDE8704006F044BF40F20F2308
:1093A000F0B52A4A2A4D2B4C83B01268214600930F
:1093B00063202B4605F086FB04F06CFEFFF7BEFF32
:1093C00004F068FE04F06AFE064604F015FF05F09E
:1093D00015F8D6F80960FFF7AFFAF06004F05AFE0E
:1093E000074604F05BFE04F007FF05F007F8FFF7FF
:1093F00085FA0646FFF7A6FAFFF7A8FA4FF4807140
:1094000038463162FCF7CEFAFFF7ACFF124B134E31
:109410000FCBFAF7D3FE1248FCF7B4FB3046F8F74F
:109420001DF906F5DC7009F06FFD642007F082F885
:10943000F8F77AF940F22D200A4A2B4612682146A5
:109440000090632005F03EFB03B0F0BDAC0B0020A4
:10945000147D0100E07C01004C7F01001C7D0100B7
:109460005C7F0100B00B0020004870471C7D0100AC
:1094700040F2F113F0B51B4A1B4D1C4C83B012682F
:1094800021460746009363202B4605F01BFBFFF7A0
:1094900055FF04F0FFFD04F001FE064604F0ACFEAB
:1094A00004F0ACFFD6F80960FFF734FAFFF744FA8E
:1094B000F060FFF757FF04F0F1FD064604F0EAFD07
:1094C000F9B23046FCF7D6FAFFF758FA40F2F91035
:1094D000074A2B46126821460090632005F0F2FAF5
:1094E00003B0F0BDAC0B0020147D0100BC7C01007A
:1094F000B00B002040F2FF1330B50F4A0F4D104C57
:1095000083B012682146009363202B4605F0DAFAF7
:109510000220FFF7ADFF0B48F8F7A0F8F8F7F4F8D2
:1095200040F20920084A2B46126821460090632029
:1095300005F0C8FA03B030BDAC0B0020147D01006B
:10954000D07C01001C7D0100B00B0020004870475A
:1095500018050020004870475C050020004870474F
:1095600068050020024A802102480DF0ABB900BF17
:109570003878010018150020014902480DF02EBA74
:109580003878010018150020014B1868704700BF9B
:1095900018150020002301488373704770050020D0
:1095A0000023014883737047A405002010B5F8F725
:1095B000ABF804F06FFD04F071FD044604F01CFEEE
:1095C00004F01CFFD4F80940FFF7D6FF0023E36046
:1095D00010BD00BF38B504F05DFD054604F05EFD2A
:1095E000044604F009FE04F009FF06F077FE284661
:1095F00006F0C6FD2046BDE8384006F0C1BD00BFFC
:1096000040F22D43F0B5144A144D154C83B0126846
:109610002146632000932B4605F054FA07F02AF800
:10962000FFF7D8FF04F036FD04F038FD06460027AA
:1096300004F0E2FD04F0E2FE40F23240D6F80960A8
:10964000084BF7601A68214600902B46632005F00E
:1096500039FA03B0F0BD00BFAC0B0020C07F0100A1
:10966000AC7F0100B00B00202DE9F04FADF2945D0E
:10967000F8F768F8002401264FF0040B1D90FAF764
:1096800061FD4FF4C772D24DD248CDE90164314635
:109690001DAB0592CDF800B03246CDE9030564203C
:1096A00005F0C8F940F28F11CB4A2B4612686320AF
:1096B0000091CA4905F006FA1E940BF031FE037FB3
:1096C00004F0E8FCD0F80930314602201A9306F085
:1096D000D1FDD0F80970824606F0F6FF1020FBF7A6
:1096E00013F940F2B918DFF814E30DF17302CDF865
:1096F0000CE080EA060CCDF8148013463146324661
:10970000CDE901440096642004958DF873C04FF0B4
:10971000020905F08FF940F2BB12B14BCDE90144CB
:109720000592CDF8009003932022AE4B0F216220CA
:10973000049505F07FF94FF4DE711A9BAA4ADB68A5
:109740007220CDE90164CDF800B0059103920F219C
:109750002022049505F06EF921469A220DF58B60C2
:109760000DF00FFA21469A220DF2F4400DF009FA9D
:10977000CDE92F443194FFF7E9FE21461B904022AA
:1097800096A80DF0FEF90DF1880821461E224EA87C
:109790000DF0F7F9C8F80040A8F8044078A8FAF7E7
:1097A000D5FC87A8FAF7D8FCDAF80D30789A5B6810
:1097B00020211878BB680492F6AA0392D6AA0292D6
:1097C0003A680192FA6800921A22F9F70FFB40F208
:1097D0006D20864AFB683146CDE90164CDF800B0C2
:1097E0000590039262202022049505F023F940F2AF
:1097F0007120DAF80D20BB6851687D4A0978CDE9FF
:109800000144CDF800B00590039272202022049507
:1098100005F010F940F27222DFF8E4A13B6831460E
:10982000CDE90164CDF800900592CDF80CA020227E
:109830006620049505F0FEF839680A222020F9F721
:10984000ABFC40F2772CDFF8BC91CDF814C0CDE929
:1098500000B63246314602941F901FAB6E2004952D
:10986000CDF80C9005F0E6F83968B6AB1E22202042
:10987000F9F7BEFC1F9A83B2A242B8BF1F32521141
:1098800094B21E1BC690002138827A820DF29A2073
:109890003E22A8F80240A8F80460A8F800300DF0B5
:1098A00070F9002340F2013402264FF0030B1A46F0
:1098B000CDF80080A6A912209846ADF898428DF800
:1098C0009AB201248DF89D620BF09EFE40F2962222
:1098D0003B682146CDE903A505926E202022009623
:1098E000CDE9014805F0A6F84FF0040A40F29723AD
:1098F0002246214605936E201FABCDE90148CDE9F4
:109900000395CDF800A005F095F84FF42670394B7B
:1099100005900393CDE90148C6ABCDF800A00495AE
:10992000224621466E2005F085F81F9B322B00F35E
:10993000B3821E2B40F328812F4B1E600020002491
:10994000FAF76AFC012702264FF43373DFF8B88078
:10995000CDE90453CDE901744FF0C14320220F211A
:1099600069200096CDF80C8005F064F80DF5916340
:10997000CDE900344FF0C1420DF2AE4320210F205B
:10998000F9F7B2F80DF58B60FAF7DAFC40F2D7235D
:10999000CDE90248CDE9045320224FF0C1430F2105
:1099A0006920CDE9006705F045F8214620225EA830
:1099B0000DF0E7F821468022D6A83494CDE9324450
:1099C000CDF8D3400DF0DDF821463C221EE000BF6B
:1099D000C07F0100C8780100AC0B00209C7F010013
:1099E000E0780100000084601C79010030790100FA
:1099F0004879010078790100D8050020D478010069
:109A0000607901007C7901007079010078A80DF07F
:109A1000B8F89A220DF58B610DF2F4400DF0A6F81E
:109A20002FA90DF2F440FCF767F940F2F723CDE9D6
:109A30000248CDE90453CDE900674FF0C14320222D
:109A40000F21662004F0F6FF1B9B93F83240002C98
:109A500000F0468256AF40220021B6A80DF091F8E2
:109A600038461E2200210DF08CF800209DF8C720FA
:109A70009DF8C6309DF8C51062F3070063F30F2010
:109A80009DF8C4201A9B61F3174062F31F60B6AAC9
:109A90009B690F21009701922022F8F7E7FF01242C
:109AA00000264FF0020A40F22B324A4BCDE9045215
:109AB0002146CDF800A003932022B6AB5320CDE978
:109AC000014604F0B7FF4FF44B704FF050094FF0D0
:109AD0003208414A3B46CDF800A02146059003924A
:109AE00053200F22CDE90146049504F0A3FFF6AB05
:109AF000B6A966AACDE900892020F9F755FE82466D
:109B000040F23330354A66AB2146059003924C2033
:109B10002022CDE901660094049504F08BFF3946BC
:109B200087AB36AACDE900890F20F9F73DFE07463D
:109B300040F237302A4A36ABCDE904500392CDE9E2
:109B400001660F22009421464C2004F073FF254A41
:109B50001368002B4AD0642B53D1BAF1010F40F3A4
:109B6000DF810023136064204623002401214FF489
:109B70006172C890C6A8C994C693C7938DF8241380
:109B8000CA920AF009FB4DE017490A68002AC6BFCD
:109B900002F1FF320A60C1F800800F2B3FF7CEAE12
:109BA000F7F7D0FDFB68F6AACDE904231B9C01461C
:109BB000B4F91A300393B4F9182000230292B4F9CF
:109BC000160013220190B4F914402020009408F0EC
:109BD000DFFDB3E6EC790100FC7901000C7A0100AD
:109BE0001C7A010024150020D8050020BAF1010FCD
:109BF000B9D1012FB7D1BDF91835B32BB3DC64232C
:109C000013600A2000260F243C21012240F6C413D1
:109C1000C790C6A8C996C694C8918DF82423CA9344
:109C20000AF0BAFA3E2200210DF21A300CF0A9FF18
:109C300000234FF0C14242F20F00822120261C4631
:109C400001270092ADF818031A468DF81D13032062
:109C5000C6A98DF81A630BF0D7FC24A8BDF8181517
:109C6000CDF89240ADF89070FAF7ACFB40F272314B
:109C7000B04B3246CDE9045103930F21AE4B6C201B
:109C80000097CDE9014404F0D5FEFAF7C5FB1D2885
:109C9000209000F3C980FAF7C5FB002840F0C4808B
:109CA00000276EAE49AC39460DF198080DF1A409B4
:109CB00028223046CDE93A77CDE93C77CDE93E77A9
:109CC00040974197429743974497459746974797C0
:109CD0004897C4E90077C4E902772761C8E90077AB
:109CE000A8F80870C9E90077A9F808700CF049FFD6
:109CF0004FF0C143914A20981268CDE91777CDE91A
:109D0000157714970E970C9707970DF58B67129799
:109D10000DF2F44711971B9FDFF81CC2109778AF24
:109D20000F97D6AF0D9732AF0B975EAF0A974EAF36
:109D3000139204933FAA44AB3AA906900997CDE940
:109D4000029696AFCDE900480A200897CDF814C0D6
:109D5000F8F7A4F99DF873101F9A002914BF202367
:109D600003230746F8F73EF910B101238DF8793047
:109D700038460521F7F7B8FC10B102238DF878308A
:109D80004FF0000A2CAF234644AA3FA9CDE9008733
:109D90003AA8CDE92CAAADF8B8A009F075FB234686
:109DA00044AA3FA93AA8CDE9008908F0B5F9CDE960
:109DB0000168CDE905AACDE90397614800940468DC
:109DC00044AB3FAA3AA90A20A04701244FF483627A
:109DD00040F219465B4BCDE90452214622460393DB
:109DE00065204346CDE901AA009404F023FE5648BD
:109DF0003B4622460390CDE901AA652000940495D4
:109E00002146059604F016FE3B4642460DF1BA0087
:109E100013F8011B09B182F800A0984202F1010277
:109E2000F6D1F7F787FC39E040F27632474B0092E3
:109E300047490022642004F045FE0024012240F23C
:109E400077310420434BCDE90451CDE9012411467B
:109E500000900393642020AB04F0ECFDFAF7D2F9F4
:109E6000064601E0062C37D0013406FA04F080B231
:109E7000FAF7C4F9BDF8181524A8FAF7A3FAFAF707
:109E8000CBFA1D282090EDDCFAF7CCFA0028E9D1B6
:109E90003046FAF7B3F903E78DF878B040F226427E
:109EA0002D4B00921A682D49284B632004F00AFEBE
:109EB00000201E9BDAB262F30700C3F3072262F3AD
:109EC0000F20C3F3074262F317401B0E63F31F60BA
:109ED0000DF2945DBDE8F08F3046FAF78FF9DDE7BB
:109EE0001F46DDF864141A464942DDF85C04F8F7B1
:109EF00029F897F83030002B3FF4ACAD40F2013236
:109F0000124B009216492246642004F0DBFD1B9B95
:109F1000204683F830400BF00DFA8DF87A6099E511
:109F2000012F3FF71EAEBDF91835C82B7FF769AE7C
:109F300017E600BFA4850100000081602015002005
:109F400014240020547A01005C7A0100C07F0100D3
:109F50002C7A0100306E0100B00B00209C7F0100C4
:109F6000D879010038B504F095F8054604F096F864
:109F7000044604F041F904F041FAFFF7EBFAC5F8A2
:109F80000D00FFF7EBFAC4F80D0038BD70B5FAF715
:109F9000D9F8044604F07EF8064604F07FF805463A
:109FA00004F02AF904F02AFA2146304606F010F9A6
:109FB00006F038F92146284606F00AF9BDE8704057
:109FC00006F030B94FF4B473F0B52B4A2B4D2C4C3E
:109FD00083B012682146009363202B4604F072FD83
:109FE00004F058F8FFF7BEFF04F054F804F056F8F8
:109FF000064604F001F904F001FAD6F80960FFF70B
:10A00000C3FAF06004F046F8074604F047F804F09D
:10A01000F3F804F0F3F9FFF799FA0646FFF7BAFAF6
:10A02000FFF7BEFA4FF4807138463162FBF7BAFC95
:10A03000FFF7ACFF134B144E0FCBFAF7BFF81348E2
:10A04000FBF7A0FD3068F7F709FB306800F5DC701E
:10A0500008F05AFF502006F06DFAF7F765FB4FF451
:10A06000C3700B4A2B46126821460090632004F00F
:10A0700029FD03B0F0BD00BFAC0B0020C07F010084
:10A080008C7F0100C87F010020150020D87F0100CF
:10A09000B00B002040F24913F0B51B4A1B4D1C4C7D
:10A0A00083B0126821460746009363202B4604F0D4
:10A0B00009FDFFF757FF03F0EDFF03F0EFFF064642
:10A0C00004F09AF804F09AF9D6F80960FFF74AFA12
:10A0D000FFF75AFAF060FFF759FF03F0DFFF06467B
:10A0E00003F0D8FFF9B23046FBF7C4FCFFF772FA71
:10A0F00040F25110074A2B46126821460090632017
:10A1000004F0E0FC03B0F0BDAC0B0020C07F010008
:10A11000687F0100B00B002040F2571370B5114A60
:10A12000114D124C82B012682146009363202B46D9
:10A1300004F0C8FCFFF798F90D4E30600220FFF7DD
:10A14000A9FF3068F7F78AFAF7F7DEFA4FF4B17033
:10A15000084A2B46126821460090632004F0B2FCA6
:10A1600002B070BDAC0B0020C07F01007C7F0100FD
:10A1700020150020B00B002038B5054C04F1100567
:10A1800054F8043B1B689847AC42F9D138BD00BF76
:10A1900004060020034A044B127853F822305B680F
:10A1A000184700BF2815002004060020034A044B6E
:10A1B000127853F82230DB68184700BF28150020BA
:10A1C0000406002038B5054C04F1100554F8043B92
:10A1D0001B699847AC42F9D138BD00BF0406002086
:10A1E0002DE9F043394EDFF8FC80337885B058F81C
:10A1F00023309B68984710F0FF05029043D1DFF8A9
:10A20000E8903478D9F800301A78A24226D0392163
:10A210002F4A1F7812682F4B009163202E49FFB2FE
:10A2200004F050FC3378BB4218BF3C46A34209D02F
:10A2300058F82330DB68984758F8243034705B684E
:10A24000984733785021D9F80000244A12680370E7
:10A250000091204B2049632004F034FC08F06CF896
:10A260000020029BDAB262F30700C3F3072262F315
:10A270000F20C3F3074262F317401B0E63F31F6006
:10A2800005B0BDE8F0833923DFF85C90104AD9F8B7
:10A29000001012680F78632000930F490D4B34783B
:10A2A00004F010FC032DFFB208D10D4B621CA3FB80
:10A2B0000234640804EB4404141BB3E7022D01D1FB
:10A2C0000324AFE7012D08BF0024ABE728150020C9
:10A2D000AC0B002000800100E47F0100B00B0020E7
:10A2E000ABAAAAAA04060020D80C002040F27A23C8
:10A2F00030B50C4A0C4D0D4C83B0126821460093CA
:10A3000063202B4604F0DEFBF7F7FEF94FF41F70D5
:10A31000074A2B46126821460090632004F0D2FBC6
:10A3200003B030BDAC0B00207C8001006C800100CC
:10A33000B00B002040F26F2370B5104A104D114C45
:10A3400082B012682146009363202B4604F0BAFBCA
:10A3500006F090F903F09EFE064605F0BFFF30467A
:10A3600005F00EFF4FF41D70074A2B461268214678
:10A370000090632004F0A6FB02B070BDAC0B00207F
:10A380007C80010058800100B00B00204FF4BD73A9
:10A390002DE9F04FD64AD74EADF55F7D1268D6490C
:10A3A00000936320334604F08DFBF7F7CBF90024CC
:10A3B00001254FF0040A1D90F9F7C4FE40F27D120A
:10A3C000CE4829461DABCDE90154059203902A469B
:10A3D00064200496CDF800A004F02CFB1E9403F03A
:10A3E00059FED0F809704FF002083B691B9303F047
:10A3F00003FE814606F068F940F28D12C04BCDE9AC
:10A400000144059203932022BE4B0F216220049643
:10A41000CDF8008004F00EFB4FF4C771BA4AFB6818
:10A42000722001950294059103920F212022049637
:10A43000CDF800A004F0FEFA21463E220DF5A170F1
:10A440000CF09FFB842542F20F0E4FF0200CFB68AE
:10A45000224600934046234650A9ADF840E18DF8CE
:10A4600042C18DF845510BF0CFF821469A2290A8B1
:10A470000CF087FB21469A22B7A80CF082FB2046FD
:10A48000CDE92F443194F9F7C7FE90A8F9F77AFF88
:10A4900099F8324054B993994A4649429198F7F74E
:10A4A00051FD99F83030002B40F004820024012740
:10A4B0004FF0020A40F2AF13DFF858B2CDE904635F
:10A4C000CDF800A04FF0C14320220F216920CDE933
:10A4D0000174CDF80CB004F0ADFA21463E220DF522
:10A4E000C1700CF04EFB4FF0C14542F20F014FF02E
:10A4F000820C4FF02008234622463846ADF88011E2
:10A50000009560A98DF885C18DF882810BF07CF8EB
:10A510002946B7A804F098F94FF4DA712B46CDE933
:10A5200000A74246CDE9046166200F21CDE9024B28
:10A5300004F080FADFF8E0A19A2290A9B7A80CF005
:10A5400015FB2FA9B7A8FBF7D7FBDAF80030002BD3
:10A5500000F0A881642B00F0568100250824052016
:10A560000A21012240F6C4130DF50078C8F80C50FA
:10A57000C8E90040C8F81030C8F8081088F80C2066
:10A58000404609F009FE3E2200210DF5E1700CF075
:10A59000F8FA00234FF0C14242F20F008221202737
:10A5A0001C464FF0010B0F250092ADF8C0011A4672
:10A5B0008DF8C511032070A98DF8C2710BF024F835
:10A5C00021A8BDF8BC10CDF88640ADF884B08DF858
:10A5D0008850F9F7F7FE4FF4F8704C4B3A4629468D
:10A5E000CDE9046003936C20494BCDF800B0CDE970
:10A5F000014404F01FFAF9F70FFF1D281F9000F324
:10A600001181F9F70FFF002840F00C81002446ABC0
:10A6100023AD214618462822CDE93244CDE9344401
:10A62000CDE93644CDE93844CDE93A44CDE93C445E
:10A63000CDE93E44409441944294439444944594DB
:10A64000C5E900442C81CDE92644ADF8A0400CF0CA
:10A6500098FA03464FF0C142DAF800001F99DFF87C
:10A66000BCE0DFF8ACC00DF5827B039390AF26AB66
:10A670000691CDE9015304923CAB37AA32A9189058
:10A680001297CDF800B00A20B7AFCDF84CE0CDF866
:10A6900014C0CDE91097CDE91644CDE91444CDE9B5
:10A6A0000E44CDE90C44CDE90A44CDE908440794B1
:10A6B000F7F7F4FC214681463E220DF202200CF011
:10A6C00060FA42F20F0A4FF0200E4FF0840C1B9BF1
:10A6D00041460093224688F802E088F805C02346E8
:10A6E000A8F800A009200AF08FFF0DF1A40817E0D8
:10A6F000AC0B00207C80010048800100C87801007C
:10A70000E0780100000084601C790100A48501004C
:10A7100000008160707901002C150020B8800100D4
:10A7200048460221F6F7E0FF0095CDF804805B462D
:10A730003CAA37A932A8C8E90044A8F8084008F0A4
:10A74000A3FE4FF0010940F257224FF0013C62484E
:10A750002B46059249464A460390CDE901446520BF
:10A760000496CDF80090CDE92CCCADF8B8C004F03B
:10A7700061F94FF4167C594843464A464946CDF89C
:10A7800014C00390CDE901446520CDF800900496F3
:10A7900004F050F926ABCDE9005337A95B463CAA3B
:10A7A00032A88DF8789007F0B7FC43460DF1AE0162
:10A7B00013F8012B02B12C70994205F10105F7D174
:10A7C000474808F0A1FBF6F7B5FF4FF41A72454B66
:10A7D00000921A684449454B632004F073F9002045
:10A7E0001E9BDAB262F30700C3F3072262F30F2065
:10A7F000C3F3074262F317401B0E63F31F600DF5AE
:10A800005F7DBDE8F08FBDF90033BE2B7FF7A5AEAD
:10A81000CAF8004000255F245A206421012240F23A
:10A820004C43A1E64FF4FA72304B009230490022BB
:10A83000642004F047F940F2F514012200210420BD
:10A840002C4BCDE90121CDE904641146009003931E
:10A8500064201FAB04F0EEF82A25F9F7D3FC05FBC2
:10A8600000F507460624AB4601E0013C16D0CBF3C9
:10A870008F10F9F7C3FCBDF8BC1021A8F9F7A2FDB1
:10A88000F9F7CAFD1D281F90AB44EEDCF9F7CAFDAD
:10A890000028EAD13846F9F7B1FCB7E63846F9F7AF
:10A8A000ADFC92E7BDF90033952BB3DC6423CAF805
:10A8B000003052E64FF4D372334600920E492246DE
:10A8C000642004F0FFF889F8304020460AF032FD99
:10A8D0008DF87A8079E700BF547A01005C7A010034
:10A8E00070820100B00B0020488001007C800100D4
:10A8F0002C7A0100306E0100D879010040F25D131E
:10A9000070B5264A264C274D82B01268294600931E
:10A910006320234604F0D6F803F0BCFB064603F0A0
:10A920006FFBC6F80D0003F0B5FB03F0B3FB064662
:10A93000F9F708FC0146304605F04AFC05F072FCC8
:10A9400003F0A8FB064603F057FB016A3046FBF70D
:10A9500029F81548F6F782FE3C2005F003FEF6F7CD
:10A96000E3FE40F26B12234600921049002264205D
:10A9700004F0A8F800230E4900931A4618460E6802
:10A980000821B0474FF4BA700A4A23461268294694
:10A990000090632004F096F802B070BDAC0B00206C
:10A9A0007C80010034800100B880010088800100B3
:10A9B00038B30100B00B00204FF4A17330B50B4A3F
:10A9C0000B4D0C4C83B012682146009363202B463C
:10A9D00004F078F84FF4A270074A2B46126821461B
:10A9E0000090632004F06EF803B030BDAC0B002083
:10A9F0007C8001000C800100B00B00204FF4A57397
:10AA000070B5124A124D134C82B012682146009361
:10AA1000114E2B46632004F055F80220FFF7CCFFBF
:10AA20003046F6F71BFEF6F76FFE06F5DC7008F011
:10AA30006BFA40F24F10094A2B46126821460090EB
:10AA4000632004F03FF802B070BD00BFAC0B0020E3
:10AA50007C80010024800100B8800100B00B002040
:10AA60009D2370B50F4A104D104C82B063201268C0
:10AA7000214600932B4604F025F800210C4E0D4A88
:10AA8000336811701B69984773681B699847A52044
:10AA9000094A2B46126821460090632004F012F800
:10AAA00002B070BDAC0B00202C8301002483010098
:10AAB0003C06002030150020B00B00205F23F0B5CD
:10AAC0000F4A104D104C83B0104E1268214663207F
:10AAD00000932B4603F0F6FF336800271B68984766
:10AAE00073680B4E1B68984766200A4B21461A680C
:10AAF00000902B466320377003F0E4FF03B0F0BDF5
:10AB0000AC0B00202C830100048301003C060020D4
:10AB100031150020B00B00208D2330B5154A164D9D
:10AB2000164C83B021461268632000932B4603F035
:10AB3000C9FF134A134B127853F82230DB68984749
:10AB40004FF04053012240F24C4083F84020FAF786
:10AB500061FA0020F9F7B2FFF9F7E0FE97200A4A00
:10AB60002B46126821460090632003F0ABFF03B030
:10AB700030BD00BFAC0B00202C8301001883010006
:10AB8000311500203C060020B00B002079232DE970
:10AB9000F041DFF860814D4D8AB04D4ED8F800206D
:10ABA0004C49009363202B4603F08CFF4A4F3378C7
:10ABB00057F823309B68984710F0FF0408901DD188
:10ABC000464C07F0B9FB8623226842490093632074
:10ABD0003E4B03F077FF0020089BDAB262F30700D8
:10ABE000C3F3072262F30F20C3F3074262F3174057
:10ABF0001B0E63F31F600AB0BDE8F0813B23D8F859
:10AC000000203749009363202B468DF81F4003F046
:10AC100059FF9DF81F303278012B099253D0022B37
:10AC200001D10123099301244FF000084A222D4B42
:10AC3000CDE904522146224603936420244BCDE9FA
:10AC40000188009403F0F6FE4B20274B2246214654
:10AC50000590039364200DF11F03CDE90188009452
:10AC6000049503F0E7FE4FF04C0C04201F4B0090BE
:10AC70000393CDE9014809AB049522462146CDF85E
:10AC800014C0642003F0D6FE194B1B78C3B9099A8F
:10AC9000337893420AD057F82330DB689847099BF2
:10ACA000DAB257F8222033705368984759230B4C77
:10ACB00000932268054B0A49632003F003FF80E7F5
:10ACC00022460994E4E700230993ACE72C830100B2
:10ACD00031150020108301003C060020B00B00203D
:10ACE000E8820100388301004083010044830100B1
:10ACF00030150020AC0B002010B5F9F717FE01202D
:10AD0000F9F7DCFEBDE81040034A044B127853F813
:10AD100022305B68184700BF311500203C06002038
:10AD200040F61B1370B5164A164D174C82B01268C8
:10AD30002146009363202B4603F0C4FE03F0AAF9DA
:10AD400003F0ACF9064603F057FA03F057FBD6F8C8
:10AD5000096003F067F90023F36003F0D7F903F00B
:10AD6000D5FAF6F7D1FC40F62310084A2B461268B4
:10AD700021460090632003F0A5FE02B070BD00BF25
:10AD8000AC0B002000840100F0830100B00B002018
:10AD90002DE9F04103F07EF9804603F07FF9074684
:10ADA00003F02AFA064603F029FB054603F07CFA75
:10ADB000044605F093FA404605F0E2F9384605F0FE
:10ADC000DFF9304605F0DCF9284605F0D9F92046D0
:10ADD00005F0D6F903F09AF9054603F097FA044610
:10ADE000284605F0CDF92046BDE8F04105F0C8B988
:10ADF0004FF4116370B5164A164D174C82B02146B8
:10AE00001268632000932B4603F05CFE05F032FCD1
:10AE1000FFF7BEFF03F03EF903F040F9064603F0EA
:10AE2000EBF903F0EBFA0022D6F80930DA6003F010
:10AE30006DF903F06BFA40F61510084A2B461268BC
:10AE400021460090632003F03DFE02B070BD00BFBC
:10AE5000AC0B002000840100DC830100B00B00205B
:10AE60002DE9F04FADF6D41DF6F76CFC012400255A
:10AE70002F900426F9F766F940F21142B348DFF843
:10AE80000CB30592CDE9030B2FABCDE9014522466A
:10AE900021460096642003F0CDFD30950AF0F0F8CD
:10AEA000002840F03A860AF03BFA034604461B7F2E
:10AEB000279003F0EFF80121D0F809A0022005F057
:10AEC000D9F91C90D0F8096003F096F92090D0F8D9
:10AED000099003F0C1F8219003F090FA2290074600
:10AEE000D0F8098003F0D2F8239003F0DDF903F0E5
:10AEF000BBF803F00BF91E90D0F809301A9303F059
:10AF0000A3F8269003F002FA1F90D0F809501D957F
:10AF100003F0B4F8E37B2890DAB21B9205F0C8FB8B
:10AF200038788B4905F0B6FA1F9C8A49207805F0DD
:10AF3000B1FA1E9901240878874905F0ABFA102070
:10AF4000F9F7E2FC002540F28342DFF844C280EAD0
:10AF50000407CDF80CC021460DF1B703059200940B
:10AF600022466420CDF810B0CDE901558DF8B770B8
:10AF700003F060FD022740F28542784BCDE904B230
:10AF8000009703932022764B0F216220CDE90155D3
:10AF900003F050FD042740F28641724ADAF80C3083
:10AFA0007220CDE90145CDE904B1009703920F214C
:10AFB000202203F03FFD40F287416B4ADAF800306F
:10AFC00065200094CDE904B103920F212022CDE940
:10AFD000015503F02FFD40F28C40D8F81C3005904D
:10AFE0000620624ACDE900742146CDE90202CDF87F
:10AFF00010B00F22622003F01DFD4FF49260062175
:10B000005B4AD9F81C30CDE90141009721460590F3
:10B01000039262202022CDF810B003F00BFD4FF018
:10B02000060C40F29B401D99524ACB69CDE9014C78
:10B03000214600970590039262200F22CDF810B0B0
:10B0400003F0F8FC4FF0060C40F29F401A9A21469C
:10B05000D369494ACDE9014C0097059003926220DB
:10B060002022CDF810B003F0E5FC40F2A240434AA4
:10B07000D8F818302146CDE9014500970590039294
:10B0800072200F22CDF810B003F0D4FC40F2A340A0
:10B090003B4AD9F818302146CDE901450097059083
:10B0A000039272202022CDF810B003F0C3FC40F2CE
:10B0B000A5401D99334A8B692146CDE9014500978A
:10B0C0000590039272200F22CDF810B003F0B2FC6D
:10B0D00040F2A6401A9A214693692B4ACDE90145D0
:10B0E0000097CDE904B003927220202203F0A2FC65
:10B0F00029463E220DF29A200BF043FD202742F212
:10B100000F0C8424DAF80C30022000932A462B46D8
:10B11000A6A9ADF898C28DF89A728DF89D420AF0F2
:10B1200073FAD9F818200DF20C63043A0DF28C6012
:10B1300052F8041F43F8041F8342F9D1D8F81820AD
:10B140000DF5D263043A0DF2CC6023E0C87801001B
:10B15000AD1A0100CD1A0100E9140100E0780100E8
:10B16000000084601C790100BC840100D8840100C7
:10B17000EC84010000850100188501003085010084
:10B18000448501005885010070850100008401009C
:10B19000D478010052F8041F43F8041B8342F9D10C
:10B1A0003E2200210DF2DA200BF0EBFC002342F6E8
:10B1B00001772F2504240DF5C2620092B6A91A4624
:10B1C0000620ADF8D8728DF8DA528DF8DD420AF01B
:10B1D0001BFA9A2200210DF59B600BF0D2FC9A22FB
:10B1E00000210DF274500BF0CCFC0023DAF8102093
:10B1F000419342934393489349934A934B934C937F
:10B200004D934E934F9350935193299202F0F4FE35
:10B21000219B1A909F7B07B11F69239B9D7B05B1E2
:10B220001D6931A8F8F792FF044632A8F8F794FF99
:10B23000D9E906214FF0140A1D90CB4848ABCDE95F
:10B240000303209BCDF814A0D3F80100319BE4B296
:10B2500025931530249402902046259C3B4601946A
:10B26000C6AC0094F8F75AF801244FF0000940F2F8
:10B2700002510227BD4AC6AB059103922146202206
:10B280006920CDF810B0CDE90149009703F0D2FB59
:10B29000D8E90621B64B4DA8CDE90330229BCDF865
:10B2A00014A0D3F80100329B153025939DF874301B
:10B2B00002901D932B46259D1D98019574AD009518
:10B2C000F8F72CF840F20E50AA4A74AB059003929E
:10B2D00069200F22CDE9014900972146CDF810B031
:10B2E00003F0A8FB0DF216330DF20E620DF256308C
:10B2F00033F8021F834222F8021FF9D10DF5E773DC
:10B300000DF5CA627BA833F8021F984222F8021B8F
:10B31000F9D13E2200210DF25A300BF032FC00230D
:10B3200042F6017582240DF5C2620092D6A91A4632
:10B330000720ADF858538DF85D430AF065F91C9B62
:10B34000319AD3F80D3024995B6801241878B368DA
:10B3500004920DF5C26203920DF58B62029232687F
:10B3600004270192F268002500921A22F7F73EFDA9
:10B3700040F246500621804AF368CDE904B0CDE999
:10B3800001410392214620226220009703F052FBE4
:10B3900040F24A501C9B4FF00208D3F80D20B368CE
:10B3A0005168764A0978CDE904B0039272202022D0
:10B3B0000097CDE9015503F03DFB40F24B52DFF819
:10B3C000D09133682146059266202022CDE90145BF
:10B3D000CDF810B0CDF80080CDF80C9003F02AFB2A
:10B3E00031680A22CD842020F7F7D6FEE6AB3390F1
:10B3F0001E2231682020F7F7FBFE0DF58B61F690D9
:10B400000DF583631E222020F7F7F2FE40F25B5217
:10B4100033682146CDE904B26E202022CDE90259DD
:10B42000CDE9008403F006FB40F25C5C544833AB8A
:10B4300022462146CDF814C00390CDE901456E2087
:10B440000097CDF810B003F0F5FA40F25D5C4D487E
:10B45000F6AB22460390CDE901450097CDF810B038
:10B460002146CDF814C06E2003F0E4FA9DF8B72011
:10B47000339BAA4214BF64225A229A4280F2F2827B
:10B48000279BDB7B002B00F02A830020F8F7C4FE0B
:10B490000DF59B60F8F776FF1A9B93F83240002C6D
:10B4A00000F086834FF470724FF0C1410DF5C26019
:10B4B0000BF05CFBBDF9FC440AF0FEF840B91E2C11
:10B4C000D4BF00240124304D2B78A34240F03884AF
:10B4D000002401254FF0020840F2BA53DFF8B4907F
:10B4E000CDE904B3CDF800804FF0C14320220F21F5
:10B4F0006920CDE90154CDF80C9003F09BFA4FF090
:10B50000C14721463E220DF29A300BF03AFB20262D
:10B5100042F20F0E4FF0820C234622462846E6A93F
:10B520000097ADF898E38DF89DC34FF0120A8DF89F
:10B530009A630AF069F8112384AACDE900A3C6A989
:10B540000DF58B633046F8F72FF940F2D35C1C9071
:10B550000E48CDF814C084AB324629460390CDE99D
:10B5600001444C2018E000BF6489010050730100C1
:10B570009C89010044730100307901004879010081
:10B580007C79010078790100401500208885010050
:10B5900060790100707901000095CDF810B003F0DA
:10B5A00049FA0A2344AACDE900A374A997AB0F2056
:10B5B000F8F7FAF8824640F2D750954A44AB29464C
:10B5C000059003924C200F22CDE901440095CDF85F
:10B5D00010B003F02FFA14232CAACDE900332BA9C5
:10B5E0002DAB2046F8F7E0F840F2DB5C89482CAB45
:10B5F000CDF814C0224629460390CDE901444C20E1
:10B600000095CDF810B003F015FA9A220DF59B6164
:10B610000DF274500BF0AAFA41A90DF27450FAF72A
:10B620006BFB39460DF2745003F00EF940F2E45111
:10B63000CDE900853B46CDE904B1CDE9024932466A
:10B640000F21662003F0F6F91B9BDFF8F881002B31
:10B6500040F0268298F80030002B00F0238240F260
:10B66000EE521B9C6C4B00926C492246642003F006
:10B6700029FA1A9B48A91A460DF59B6082F83140B9
:10B6800083F830404DAAF7F787F998F80030002B7F
:10B6900000F0218200232EA88DF8B8308DF8B93043
:10B6A00007F0C8FB98F8003073B3012400250DF5AE
:10B6B00083620DF20F230DF22F2013F8011F0132C8
:10B6C0001F290CBF02F8015C02F8014C9842F4D12A
:10B6D00001240025F6AB0DF20F120DF58F7012F854
:10B6E000011F01331F290CBF03F8015C03F8014C53
:10B6F0009042F4D14FF0C1420DF5836300922021B6
:10B70000F6AA0F20F7F790F91C9B012B00F090820E
:10B7100043490B6840F39182002201334148012BD9
:10B720000B600260404E40F3098314463260642B84
:10B73000326805DD64230B60642C01DD6423036043
:10B74000002A40F0EF82394B1A78012A40F09182AA
:10B750001C9A012A40F3858300221A70344C0DF59F
:10B7600083650FCC0FC523680DF583602B6008F04F
:10B7700013FD98F80030002B40F08682002401274A
:10B780000F2536A8BDF80411CDF8DA40ADF8D87011
:10B790008DF8DC50F8F716FE40F2DE62254B2946A4
:10B7A000CDE904B203932022234B6C200097CDE90E
:10B7B000014403F03FF9F8F72FFE1D28349003DC15
:10B7C000F8F730FE002858D040F2E262124B0092A7
:10B7D0001A490022642003F075F940F2E364012263
:10B7E00000210420164BCDE90121CDE904B4114616
:10B7F00000900393642034AB03F01CF92A25F8F77A
:10B8000001FD05FB00F507460624A9461FE000BF21
:10B8100094850100A085010000840100AC85010031
:10B82000381500203C15002034150020321500206A
:10B8300050830100A4850100000081602C7A010082
:10B84000306E010041150020013C00F06181C9F318
:10B850008F10F8F7D3FCBDF8041136A8F8F7B2FD45
:10B86000F8F7DAFD1D283490A944EDDCF8F7DAFD8D
:10B870000028E9D13846F8F7C1FC00246EAF0DF17D
:10B88000E00921462C228CA8C9E90044CDE93B44BB
:10B89000C9F80740CDF8F3405C945D945E945F94E2
:10B8A0006094ADF884416294639464946594669462
:10B8B000ADF89C41689469946A946B946C94ADF86B
:10B8C000B441C7E90044C7E902443C61BC820BF0C3
:10B8D00058F94FF0C1430DF59B65316812950DF293
:10B8E000745511951A9D3498109597ADCDE90EA514
:10B8F0000DF58B650D951C9D8CAA0C9544AD0B9593
:10B9000084ADDFF828C303920A953BAA74ADBC4E00
:10B91000CDE901920493189168AB069009950097C0
:10B9200062AA5CA90A20C6ADCDE91644CDE914444B
:10B93000079408951396CDF814C0F6F7AFFB98F866
:10B9400000308246002B40F097821B9B002B40F07A
:10B950000C821B9D3E2229460DF2DA300BF011F9C4
:10B9600042F20F0220208424299BF6A90093ADF80F
:10B97000D8238DF8DA032B4609202A468DF8DD43BB
:10B9800009F042FE02215046F5F7AEFE002840F0D5
:10B99000BF821A9500243EAECDE900963B46C6E92B
:10B9A000004468AA62A9C6F807405CA807F06CFDCD
:10B9B0003BABCDE9009368AA3B4662A95CA806F0C0
:10B9C000ABFB1E9B2698D3F809201F9B9469D3F8E4
:10B9D0000930D269817B1C929A69DB692194229299
:10B9E0002093002900F0738203692393289A937BA4
:10B9F000002B00F06A821369259300241B9B52944C
:10BA000053945494559456945794589459945A94E2
:10BA10005B94002B40F0208335AD00241B9B7948BC
:10BA200006933BABCDE902938CABCDE90073049652
:10BA30000594076862AA5CA968AB0A20B84721464A
:10BA400037460DF5817217F8013B0BB189F80010EC
:10BA5000BA4209F10109F6D16B4807F055FAF5F73A
:10BA600069FE40E00F2B3FF710ADF5F76BFEF36872
:10BA70000DF5C262CDE904231A9C0146B4F91A30CF
:10BA80000393B4F918202B460292B4F9160013223E
:10BA90000190B4F914402020009406F079FEF4E4FB
:10BAA00088F800401A9B48A993F831200DF59B6057
:10BAB000013204920DF5C262CDE902A21C9A84AB58
:10BAC000019244AA00924DAAF6F7CEFE98F80030F3
:10BAD000002B7FF4DFAD4D4807F0ACF9E2E503231E
:10BAE00035AD8DF8C1300020309BDAB262F307002B
:10BAF000C3F3072262F30F20C3F3074262F3174038
:10BB00001A0E62F31F602B600DF6D41DBDE8F08F96
:10BB10003846F8F773FB35ADE5E740F219413C4F85
:10BB20003C4A7B686520059103922146CDF810B010
:10BB3000CDE9015500940833212202F07BFF4FF03C
:10BB4000060840F21D417B68334A0591CDE9028227
:10BB50002146CDF810B0CDE90064A833212265203C
:10BB600002F068FF40F21E417B682C4A0591039267
:10BB70002146CDF810B0CDE90155009429331422A7
:10BB8000652002F057FF40F222407B68244A05906E
:10BB9000039203F59673CDF80880CDF810B0CDE987
:10BBA000006421461422652002F044FFFFF77BB9B0
:10BBB000DDF8E4141A464942DDF8DC041D46F6F7C8
:10BBC000C1F9BDF9FE34313380F2C9801A9D95F870
:10BBD0003030002B3FF466AC40F29652114B00928D
:10BBE00011492246642002F06DFF85F8304020465E
:10BBF00009F0A0FB022335AD8DF8C23073E700BF1A
:10BC00003487010014240020EC88010058880100CA
:10BC1000742000203C840100588401007C840100D1
:10BC20009884010000840100D8790100000081603F
:10BC3000BAF1010F61D0BF490B68BAF1010F3FF7AC
:10BC40006BADBDF99825DC2A3FF766AD012BC8BF67
:10BC50000022B948C8BFB94E0468D4BFB74E32609D
:10BC6000012C7FF764AD6422934232603FF762ADEE
:10BC700062E5BDF99825EF2A3FF770AD01221A70F1
:10BC80000DF58365AE4C6CE5AE4FF6AD0FCF0FC52D
:10BC90003B68F6A82B6008F07FFA00230A22642490
:10BCA00002274625A849CDF82434CDF82834CDF80C
:10BCB0002C34CDF83034CDF83434CDF83834CDF8D8
:10BCC0003C34A24B0DF58360CDF84824CDF84C24CC
:10BCD000CDF81C14CDF82034CDF81874CDF84044BC
:10BCE000CDF844540AF048F840F203338CA8ADF87C
:10BCF000303207F009F9346040E5BDF99825BD2AD6
:10BD000000F30F8100218C488A4A036811600133D7
:10BD1000012B036040F366836422884E93423260B5
:10BD20003FF70CAD8A4D0DF583640FCD0FC42B6822
:10BD30000DF58360236008F02FFA1AE53268FFE4FE
:10BD400004F064FC1A9B93F91C001B9B13B1269B07
:10BD500093F91C0004F0EEFB2C70FFF7B9BB85F8DB
:10BD6000314085F83040FFF79DBBBAF1000F40F03D
:10BD7000B0801A99BDF9FC24B1F918309A4280F2CA
:10BD8000D380BDF9FE24B1F91A309A4240F3CC8039
:10BD900040F279726F4B00926F495246642002F074
:10BDA00091FE4FF0C1431A99BDF8F2040D4691F986
:10BDB0001D200493299B0593B1F91A300393B1F91F
:10BDC0001810BDF8F6340291B5F9164003440194F9
:10BDD000B5F914402F9900944FF4F07006F0D8FC98
:10BDE000209BC6A9D3F8093095F91D20DB69219E57
:10BDF000CDE90413B6F91A30BDF928010393B6F959
:10BE00001810BDF92A310291B6F916400344019485
:10BE1000B6F914402F990094202006F0B9FC229B1B
:10BE200074A9D3F8093095F91D20DB69239DCDE96C
:10BE30000413B5F91A30BDF93C010393B5F9183074
:10BE40002F990293B5F91640BDF93E310194B5F929
:10BE50001440034400940F2006F09AFC01231A9327
:10BE600039E0BAF1010F3FF777ACBDF99825B2F58B
:10BE7000827F7FF705AF6FE44FF00046322548AB75
:10BE8000CDE901630A226FF00903C6A900952020BD
:10BE9000F7F7C6F94DAB1C900293CDE900566FF051
:10BEA00009030A2274A90F20F7F7BAF91C9B002B8B
:10BEB00056D0002854D040F26C7322460093274994
:10BEC000244B642002F0FEFD3FE5259395E5239188
:10BED0008CE500231A933E2200210DF2DA300AF09D
:10BEE00050FE002342F20F0120208424299AADF84D
:10BEF000D8130092F6A98DF8DA031A4609208DF8B6
:10BF0000DD4309F081FB02215046F5F7EDFB41E5E9
:10BF100098F800305BB902238DF8C0301B9B1A9350
:10BF200038E504490B688EE6CDF868A0D3E71B9B83
:10BF30001A932FE5381500203C15002034150020F9
:10BF40008C83010078830100050090010A009001B4
:10BF500064830100008401000C8701002086010039
:10BF600040F23F7200920022BDF8F634BDF8F24470
:10BF700036491C446420364BCDF81844144602F070
:10BF8000A1FD01224FF4E8610420324BCDE90124E8
:10BF9000CDE904B100901146039364200DF583634D
:10BFA00002F048FD1A98299B054605930DF5C263DA
:10BFB0000493B0F91A2006460392B0F91810DDF880
:10BFC00018340291B0F9160022460190B5F9140018
:10BFD000214600904FF4F07006F0DAFB209BC6A9D2
:10BFE000D3F809202198D269DDF81834CDE904127C
:10BFF000B0F91A1022460391B0F9180021460290B8
:10C00000B5F916000190B5F914502020009506F0FE
:10C01000BFFB229B74A9D3F809202398D269DDF8CD
:10C020001834CDE90412B0F91A1022460391B0F980
:10C03000180021460290B6F916000190B6F9144096
:10C040000F20009406F0A4FB7FE400BFEC85010004
:10C05000008401000C8601000A2552ABCDE90435AD
:10C06000BD4B1E990393D1F80130319A15330DF56C
:10C070008361CDE901230091239B219A1C99249887
:10C08000F7F74CF902204FF0010840F62403009026
:10C09000B2480593414603900DF583632022692041
:10C0A000CDF810B00294CDF8048002F0C3FC57A97B
:10C0B0000491AB4905951F9D0391D5F80130329A43
:10C0C0007CAD153300950225CDE901232099259BF0
:10C0D000229A1D98F7F722F94FF403620095A14DBB
:10C0E0007CAB03954146059269200F22CDF8048070
:10C0F000CDF810B0029402F09DFC09F0EBFB40F685
:10C10000910EDFF878C235ADCDF80080CDF810B0D3
:10C11000CDE901442B4628704246CDF814E0CDF815
:10C120000CC04146642002F085FC8B4A2B780892B3
:10C130007CAA019257AA0B9252AA0A92259A884980
:10C140000792239A09910692209A0F2105921C9A30
:10C1500020200492229A0392219A02920DF5836282
:10C1600000925246F7F74CFBBDF8B411BDF81834F5
:10C170001B90BDF81A040B44BDF81C1403440B4477
:10C18000DFF8FCC11BB28CFB031C40F6AA020221A3
:10C190007248ACEBE37C03900091059241460DF5AB
:10C1A000836320224920CDF80480CDF810B002949A
:10C1B000ADF8B4C102F03EFC6A4B40F6AB0203930B
:10C1C00002234146009305927CAB0F22CDF80480F8
:10C1D000CDF810B00294492002F02CFC2699BDF94C
:10C1E0005421B1F918309A4261DABDF95621B1F9FA
:10C1F0001A309A425BDD2899BDF96821B1F91830EF
:10C200009A4254DABDF96A21B1F91A309A424EDDE8
:10C210001A9B002B4BD040F6B5032246524900939F
:10C220006420524B02F04EFCBDF95231BDF9504131
:10C230001C44F5F787FA269B1C9993F91D2005915C
:10C240000DF583610491B3F91A10234603912699E1
:10C25000B1F9184001460294269CB4F916000190E9
:10C26000B4F914402020009406F092FABDF966312A
:10C27000BDF964411C44F5F765FA289B209993F9B0
:10C280001D2005917CA90491B3F91A10234603914E
:10C290002899B1F9184001460294289CB4F9160077
:10C2A0000190B4F914400F20009406F071FA269B17
:10C2B00093F83280B8F1000F7FF4AFAB40F6D702AD
:10C2C0000424059201225799294B1A910393589BF4
:10C2D000529800941A9C1C93DDF84CC120441C9C7D
:10C2E0001146CDF80880019252AB1A90CDF810B0EB
:10C2F0004920644402F09EFB0422012140F6D8004C
:10C30000CDE9002101221B4B1146CDF80880059094
:10C310000393492053ABCDF810B002F08BFB40F6ED
:10C32000D90C4FF0010E012204231348CDE9003E41
:10C330001146CDF814C0CDF8088057AB0390CDF866
:10C3400010B0492002F076FB0422012140F6DA0009
:10C35000CDE90021012215E0808901004486010019
:10C36000B889010050860100648601000084010044
:10C3700088860100A4860100C08601005C86010059
:10C3800056555555194B1146CDF808800590039325
:10C39000492058ABCDF810B002F04CFBDDF8988086
:10C3A000214642461A98F5F7CDFD98F83030002B1B
:10C3B0003FF433ABBAF1000F7FF42FAB4FF40E62B2
:10C3C0000B4B00920B495246642002F07BFB269BEC
:10C3D000504683F830A008F0ADFF02238DF8C2303C
:10C3E000FFF781BB044E3268FFF7AAB9DC86010073
:10C3F00000840100F8860100341500202DE9F04189
:10C4000001F048FE804601F049FE074601F0F4FEC7
:10C41000064601F0F3FF054601F046FF044601F031
:10C42000EFFDC8F80D0001F0EFFDC7F80D0001F0B9
:10C430000FFEC6F80D0001F025FEC5F80D0001F055
:10C440000FFEC4F80D0001F061FE054601F05EFF2D
:10C45000044601F0F5FDC5F80D0001F00BFEC4F82F
:10C460000D00BDE8F08100BF2DE9F84301F012FE98
:10C47000064601F013FE054601F0BEFE074601F038
:10C48000BDFF8046F7F75EFE194B04461B789BB94B
:10C490002146384603F09CFE03F0C4FE2146304698
:10C4A00003F096FE03F0BEFE2146284603F090FE00
:10C4B000BDE8F84303F0B6BE08F032FFC37B33B9E2
:10C4C0002146404603F084FE03F0ACFEE0E701F0B5
:10C4D0001DFE814601F01AFF214603F079FE03F0AC
:10C4E000A1FE2146484603F073FE03F09BFEE7E7FA
:10C4F0005806002040F2C7322DE9F04F614B85B05D
:10C5000000921A686049614B632002F0DBFAF7F78A
:10C5100053F904F091F85E4C2070FFF76FFF01F0C3
:10C52000B9FD01F0BBFD054601F066FE01F066FFB6
:10C53000D5F8095001F07EFDE86001F0E7FD01F05B
:10C54000E5FE01F0A7FD834601F0A8FD01F054FED1
:10C55000814601F053FF074601F0A6FE054601F0B3
:10C560004BFD824601F078FD064601F08FFD8046C6
:10C5700001F07AFD336ADAF82010066A5846D8F8D6
:10C5800020800393F9F70EFA039B48461946F9F702
:10C590007DF841463846F9F779F831462846F9F7EB
:10C5A00075F801F0B3FD074601F0B0FE054601F055
:10C5B0004BFD804601F062FD064608F061FD002853
:10C5C00047D1D8F82010366A3846F9F75FF8314677
:10C5D0002846F9F75BF8FFF747FF2E4B0FCBF7F72D
:10C5E000EDFD2D48F9F7CEFA2C48F5F737F801F0B4
:10C5F00005FF2378002B38D001F0FEFC90F91C5089
:10C6000008F08EFEC37B4BBB284603F093FF012549
:10C61000F5F78AF84FF480630022009320492570D3
:10C620001A4B642002F04EFA00231E4900931A466A
:10C6300018460C680221A04740F209421A4B0092AA
:10C640001A681149114B632002F03CFA05B0BDE8AD
:10C65000F08F164B5B68D3E90016B5E701F056FD85
:10C6600001F0F2FC90F91C00CFE701F0C7FE104981
:10C67000007803F00FFF052003F032FF0D4806F0AD
:10C6800043FCB9E7AC0B0020C88301000084010023
:10C6900058060020088A0100D8890100348701006B
:10C6A0000C84010038B30100B00B0020742000207E
:10C6B000BD1C0100D48901004FF460732DE9F04FD7
:10C6C000D14A8DB01268D14900930446D04B632003
:10C6D00002F0F8F9FFF792FE01F0DCFC01F0DEFC5D
:10C6E000054601F089FD01F089FED5F80950EB6897
:10C6F000002B00F0028201F009FD01F007FE01F0BD
:10C70000ABFC01F0C3FC01F0C5FC054601F0C6FC22
:10C71000074601F071FC8046F7F714FD0646014616
:10C72000284603F055FD03F07DFD3146384603F001
:10C730004FFD03F077FD2878002103F0ABFE29467A
:10C74000304603F04FFA98F80E00F7F75FFD4046C9
:10C75000F9F732F9D5F80130DB7A1BB1AD49287809
:10C7600003F098FE03F0BAFD284603F009FD3846B1
:10C7700003F006FD01F0CAFC064601F0C7FD0546C0
:10C78000F7F7E0FC074608F07BFC002840F05681F4
:10C790003946284603F01CFD03F044FD3946304677
:10C7A00003F016FD03F03EFD03F016FF03F04CFF0F
:10C7B00001F04AFC01F062FC9749307803F06AFE10
:10C7C000964A3146384604F06BFD9549287803F0C7
:10C7D00061FE3846914A294605F076F803F07EFD61
:10C7E000304603F0CDFC284603F0CAFC30788D4972
:10C7F00003F050FE8C49287803F04CFE01F0FCFC5D
:10C80000074601F0FBFD0646F7F79CFC8046014613
:10C81000304603F0DDFC03F005FD4146384603F0E9
:10C82000D7FC7E4D03F0FEFC03F0D6FE03F00CFFB8
:10C830003878002103F02EFE2A463946404604F09F
:10C840002FFD3878794903F025FE3078002103F078
:10C8500021FE2A463146404605F036F874493078C4
:10C8600003F018FE03F03AFD384603F089FC304629
:10C8700003F086FCFEF78CFAFFF7F6FD01F00AFCE8
:10C88000074601F00BFC804601F0B6FC069001F073
:10C89000B5FD079001F008FD834601F0ADFB814630
:10C8A00001F0DAFB089001F0F1FB099001F0DCFBEC
:10C8B0008246F7F747FCE4B2214606464046F9F7C0
:10C8C000D9F84246234639464846F9F785F801F03B
:10C8D0001DFC0A9001F01AFD814601F0B5FB0B909A
:10C8E00001F0CCFB804608F0CBFB002840F0E9804B
:10C8F000DDE90A21234630460095F8F7BBFF009595
:10C900004A46414623463046F9F700F80095069A14
:10C91000089923463046F8F7CFFE0095079A099903
:10C9200023463046F8F714FF009523465A465146F1
:10C930003046F8F759FF40F2F52600250120022184
:10C94000D7F80930324C3B4A5B69CDE901050596C1
:10C950000091CDE903240F212022642002F06AF81F
:10C9600001F098FB834601F099FB01F045FC8146FC
:10C9700001F044FD074601F097FC054601F03CFB41
:10C98000824601F069FB064601F080FB804601F01B
:10C990006BFB336ADAF82010066A58460693D8F81B
:10C9A0002080F8F7FFFF069B48461946F8F76EFE11
:10C9B00041463846F8F76AFE31462846F8F766FEE3
:10C9C00001F0A4FB074601F0A1FC054601F03CFB89
:10C9D000064601F053FB316A066A3846F8F756FE00
:10C9E00031462846F8F752FEFEF7D2F940F28A3176
:10C9F000114A2346126863200091044902F062F84C
:10CA00000DB0BDE8F08F00BFAC0B0020A08301008B
:10CA100000840100F1F9000015150100D90501009D
:10CA2000191B0100E9140100CD1A0100C91401000D
:10CA3000AD1A0100E4890100B00B002001F066FB93
:10CA4000074601F063FCD7F80930DFF8BCC01A686C
:10CA5000DCF80410013ACB1D01F1280E13F8011F78
:10CA6000734502F8011FF9D1D0F80930DCF8041041
:10CA70001A6801F13C0E01F12803013A13F8011F75
:10CA8000734502F8011FF9D1D7F80930DCF804C06A
:10CA90009A680CF17E070CF13C03023A33F8021F4E
:10CAA000BB4222F8021FF9D1D0F809200CF1A600F0
:10CAB0009268023A33F8021F834222F8021FF9D12A
:10CAC00094E601F023FB814601F020FCDFF838807A
:10CAD000D9F80930D8F80420D0F80990D969A832DB
:10CAE0002020F8F7DBFDD8F80420D9F81C1002F557
:10CAF00096720F20F8F7D2FD08E701F089FA01F0ED
:10CB000099FAE860F7E500BF742000204FF46E73D7
:10CB100070B5124A124D134C82B012682146009330
:10CB2000114E2B46632001F0CDFF0120FFF7C4FD1D
:10CB30003046F4F793FDF4F7E7FD06F5DC7006F0F8
:10CB4000E3F940F2C130094A2B46126821460090B1
:10CB5000632001F0B7FF02B070BD00BFAC0B002036
:10CB600000840100B883010034870100B00B00206D
:10CB7000F8B501F045FA094D4FF0180C2C46662720
:10CB800002260368186859689A68DB680FC4044B6A
:10CB900085F802C06B602F81AE72F8BD441500208D
:10CBA0000215660001F028BA08B5FFF7E1FF014859
:10CBB00008BD00BF5C06002008B5FFF7D9FF01F0F3
:10CBC00023FA024B426818465A6008BD64060020EA
:10CBD00001F030BA40F26D3330B5104A104D114CAF
:10CBE00083B021461268632000932B4601F06AFF50
:10CBF00001F050FA01F052FA0022D0F80930DA6060
:10CC0000F4F782FD40F27530074A2B461268214640
:10CC10000090632001F056FF03B030BDAC0B002044
:10CC20009C8A0100888A0100B00B002038B501F011
:10CC300031FA054601F032FA044603F04FFB28466C
:10CC400003F09EFA2046BDE8384003F099BA00BFD1
:10CC500040F26233F0B5114A114D124C83B01268A4
:10CC60002146632000932B4601F02CFF03F002FDC8
:10CC7000FFF7DCFF01F00EFA01F010FA002740F296
:10CC80006736D0F80900084BC7601A6821462B4662
:10CC90000096632001F016FF03B0F0BDAC0B00203E
:10CCA0009C8A0100708A0100B00B00202DE9F04F32
:10CCB000ADF54B7DF4F746FD012500244FF0040946
:10CCC0001C90F7F73FFA40F2D112C54EC5481CAB95
:10CCD000059229462A46CDE90306CDE90154642090
:10CCE000CDF8009001F0A6FE4FF4E971BE4A33463C
:10CCF000126863200091BD4901F0E4FE1D9408F024
:10CD00000FFB037F01F0C6F929460746022003F016
:10CD1000B1FAD7F809B08246D0F8097003F0D4FC14
:10CD200040F2E71205920222B14B009203932022B7
:10CD3000B04B0F2162200496CDE9014401F07AFE48
:10CD40004FF4F471AC4ADBF80C3072200591039279
:10CD50000F2120220496CDE90154CDF8009001F076
:10CD600069FE21463E220DF5997009F00AFF4FF049
:10CD7000200842F20F0E4FF0840CDBF80C302246F4
:10CD80000093022023464CA9ADF830E18DF835C15F
:10CD90008DF8328108F038FC21469A227CA809F0EF
:10CDA000F0FE21469A22A3A809F0EBFECDE92B4420
:10CDB0002D94FFF7F7FE1A9028A8F7F7C7F91B90F4
:10CDC0002EA8F7F7C9F9DAF80D30289A5B680DF547
:10CDD000B87B1878BB6804926CAACDE902B23A68B5
:10CDE0001B990192FA68C9B200921A22F5F71CFF4A
:10CDF0004FF4067C8148FB6842462946CDF814C0B2
:10CE0000039004966220CDE90154CDF8009001F022
:10CE100011FE4FF4077CDAF80D2079485268BB68A0
:10CE200011784246CDF814C0039004967220CDE9E3
:10CE30000144CDF8009001F0FDFD40F21D2C0222CE
:10CE400070483B682946CDF814C0009203904246D2
:10CE500066200496CDE9015401F0ECFD39680A2200
:10CE60004046F6F787F93968824633AB1E224046C2
:10CE7000F6F7BEF9594638903DAB1E224046F6F70C
:10CE8000B7F94FF40A7EDFF88CC1CDF814E0429078
:10CE90003DAB2A462946CDF80CC06E200496CDE95C
:10CEA0000154CDF8009001F0C5FD40F2292C564800
:10CEB00042AB2A462946CDF814C0039004966E2052
:10CEC000CDE90154CDF8009001F0B4FD40F22A2CD8
:10CED0004E4804960390CDE90154CDF8009038AB4C
:10CEE0002A462946CDF814C06E2001F0A3FDBAF100
:10CEF0000F0F40F318820020F7F78EF97CA8F7F7A0
:10CF000041FA1A9B93F83240002C00F0ED81BDF9F4
:10CF1000144208F0D1FB78B9142CD4BF00240124AA
:10CF20003B4D2B78A34207D003F070FB1A9B93F97B
:10CF30001C0003F0FFFA2C70002401254FF41B7332
:10CF40004FF00209DFF8D0A0CDE9046320224FF0B2
:10CF5000C1430F216920CDE90154CDF80090CDF8EF
:10CF60000CA001F067FD21463E220DF5B97009F0D5
:10CF700008FE4FF0C1484FF0820C202742F20F010B
:10CF80002346CDF8008022468BF805C0ABF8001090
:10CF9000284659468BF8027008F036FB9A227CA985
:10CFA000A3A809F0E3FD2BA9A3A8F8F7A5FE40F27A
:10CFB0008121DFF868B04346CDE90461CDE9024A3A
:10CFC000CDE900953A460F21662001F033FDDBF8EC
:10CFD0000030002B00F0C381642B00F03A811FE089
:10CFE0009C8A0100C8780100AC0B00205C8A01001B
:10CFF000E0780100000084601C79010030790100B4
:10D000004879010060790100B88A0100787901004F
:10D010005C150020A88A01007079010058150020D5
:10D020000025082405200A21012240F6C4136D9032
:10D030006CA86F9570936C946E918DF8BC2107F07D
:10D04000ABF83E2200210DF5D97009F09AFD0023BE
:10D050004FF0C14242F20F00822120271C464FF0C0
:10D0600001080F250092ADF8B0011A468DF8B511F0
:10D0700003206CA98DF8B27108F0C6FA20A8BDF89B
:10D08000B012CDF88240ADF880808DF88450F7F76B
:10D0900099F94FF42F70B84B3A462946CDE9046010
:10D0A00003936C20B54BCDF80080CDE9014401F02D
:10D0B000C1FCF7F7B1F91D281E9000F3D980F7F7EE
:10D0C000B1F9002840F0D48000270DF188083946D6
:10D0D00025AC282242A8CDE92E77CDE93077CDE9DD
:10D0E0003277CDE93477CDE93677CDE93877CDE9B8
:10D0F0003A77CDE93C77CDE93E7740974197C8E94B
:10D100000077A8F80870C4E90077278109F039FD95
:10D110004FF0C1431E9ADBF80000CDE91677CDE948
:10D120001477CDE90E77CDE90C77CDE90A77CDE913
:10D13000087707977CAF0692129742AAA3AFDFF851
:10D1400068E2039211973DAA1A9F8C4D00920493B6
:10D150002EA91890CDE9018438AB33AA0A20109784
:10D16000CDF84CE00595F4F799FF0221F4F7BCFAED
:10D17000002840F0FD80002528ABCDE9008338AAC7
:10D180003DAB33A92EA8CDE92855ADF8A85006F03F
:10D190007BF928ABCDE90343CDE9055542AB0193BB
:10D1A00077483DAB0093CDF80880046838AB33AACC
:10D1B0002EA90A20A047012440F24B32714BCDE941
:10D1C000046221462246039365204346CDE901557A
:10D1D000009401F02FFC4FF453706B4B22460590E6
:10D1E0000393652028ABCDE90155009404962146B0
:10D1F00001F020FC434628AA0DF1AA0012F8011BF9
:10D2000001B11D70904203F10103F7D15F4805F0B1
:10D210007BFEF4F78FFA40F25B325D4B00921A68A6
:10D220005C495D4B632001F04DFC00201D9BDAB290
:10D2300062F30700C3F3072262F30F20C3F3074230
:10D2400062F317401B0E63F31F600DF54B7DBDE8C5
:10D25000F08FBDF9B032BE2B7FF7E2AECBF80040C5
:10D2600000255F245A206421012240F24C43DEE66F
:10D270004FF43072484B009248490022642001F07C
:10D2800021FC0024012240F2C1210420444BCDE9BD
:10D290000461CDE9012411460090039364201EAB84
:10D2A00001F0C8FBF6F7AEFF054601E0062C17D0EB
:10D2B000013405FA04F080B2F6F7A0FFBDF8B01211
:10D2C00020A8F7F77FF8F7F7A7F81D281E90EDDCE8
:10D2D000F7F7A8F80028E9D12846F6F78FFFF3E61C
:10D2E0002846F6F78BFF96E71D467F991A46494276
:10D2F0007D98F4F727FE95F83030002B3FF407AE09
:10D3000040F25322244B009226492246642001F029
:10D31000D9FB1A9B204683F8304008F00BF8022313
:10D320008DF8763077E7F4F70DFAFB686CAACDE953
:10D3300004231A9A01461046B2F91A300393234681
:10D340000446B2F918200292B0F916204046019224
:10D35000B4F914401322009405F01AFACBE5BDF994
:10D36000B032952B3FF77CAF6423CBF8003057E603
:10D3700002238DF87430FEE6A48501000000816070
:10D3800014240020547A01005C7A0100808C010092
:10D39000B00B00205C8A01009C8A01002C7A0100FD
:10D3A000306E0100F8860100C88A010038B500F02F
:10D3B00071FE054600F072FE0446FFF7F5FBC5F866
:10D3C0000D00FFF7F9FBC4F80D0038BD10B500F0F3
:10D3D00061FE00F063FED0F80940FFF7F9FBE06062
:10D3E00010BD00BF10B500F055FE044600F056FE1B
:10D3F000FFF7D8FB016A2046BDE81040F8F7D2BA23
:10D4000070B500F047FE064600F048FE0546F6F708
:10D4100099FE04460146304602F0DAFE02F002FFB1
:10D420002146284602F0D4FEBDE8704002F0FABE64
:10D4300040F2AF1330B5184A184D194C83B012683A
:10D440002146632000932B4601F03CFBFFF7AEFF23
:10D45000FFF7BCFFFFF7C6FFFFF7D2FF114B0FCB63
:10D46000F6F7ACFE1048F8F78DFB1048F4F7F6F825
:10D47000FFF798FB90F91C0003F05CF8F4F754F9FF
:10D4800040F2C9100A4A2B461268214600906320D8
:10D4900001F018FB03B030BDAC0B00209C8A0100EA
:10D4A000488A0100F88C0100088D0100C88A01003B
:10D4B000B00B002040F2911330B5104A104D114CC2
:10D4C00083B012682146632000932B4601F0FAFADC
:10D4D000FFF76CFFFFF77AFFFFF792FFFFF782FF7E
:10D4E000FFF7A4FB40F29910074A2B461268214629
:10D4F0000090632001F0E6FA03B030BDAC0B0020D1
:10D500009C8A0100188A0100B00B002040F29F1392
:10D5100070B5124A124D134C82B012682146009326
:10D52000114E2B46632001F0CDFA0220FFF7C2FF17
:10D530003046F4F793F8F4F7E7F806F5DC7005F0F9
:10D54000E3FC40F2A910094A2B46126821460090DC
:10D55000632001F0B7FA02B070BD00BFAC0B002031
:10D560009C8A0100348A0100C88A0100B00B0020A7
:10D57000704700BF08B502F0B1FE00F03FFFBDE804
:10D58000084002F0FDBD00BF08B503F073F84FF08E
:10D590004053012283F8402040F24C40BDE808404F
:10D5A000F7F738BD08B503F065F84FF04053012296
:10D5B00040F24C4083F84020F7F72CFDBDE80840CE
:10D5C000FFF7D8BFFFF7EEBF704700BF38B50022A6
:10D5D0004FF0405383F84020F6F7B4FD054600F0C5
:10D5E0000DFF044600F04EFD2946C4F80D0020460C
:10D5F00002F0EEFD02F016FE00F048FD0A4B1B782B
:10D60000012B08D090F91C30084A18461360BDE879
:10D61000384002F08FBF2823044A18461360BDE843
:10D62000384002F09FBF00BFAE15002094060020D6
:10D63000C32230B5204B85B000921A681F49204B99
:10D64000632001F03FFAFFF7C1FFF4F76DF81D4BBF
:10D650001D4A1B781268012B039219D0CB22184B5C
:10D6600000921A490022642001F02CFA00230121C3
:10D6700000931A461846039CA047DE22144B0092E2
:10D680001A680E490E4B632001F01CFA05B030BD3C
:10D690000024D5230F4D224600930F49084B6420E8
:10D6A0002C7001F00FFA00942346224620460421F4
:10D6B000039CA047E1E700BFAC0B0020148D0100E4
:10D6C000348D0100AE15002038B301003C8D0100FF
:10D6D000B00B0020301500206C8D010008B502F061
:10D6E000C9FF4FF04053012240F24C4083F84020E4
:10D6F000F7F790FC02F0F2FD00F080FEBDE8084074
:10D7000002F03EBD70B500F077FD064600F0C2FCA9
:10D710000546F6F717FD04460146304602F058FD6F
:10D7200002F080FD2146284602F052FDBDE870401F
:10D7300002F078BD38B500F05FFD054600F0AAFCA8
:10D74000044602F0CBFD284602F01AFD2046BDE853
:10D75000384002F015BD00BF2DE9F04FCFB0F6F70D
:10D76000F1FC0127F3F7EEFF4FF00009EE224FF036
:10D77000040B654C654D4EAB43F8F80D39460592E8
:10D78000CDE903543A466420CDE90179CDF800B0E3
:10D7900001F050F9F0215E4A23461268632000919F
:10D7A0005C4901F08FF9CDF8449000F027FE8046E7
:10D7B00000F06CFC054600F04FFC824602F084FF4E
:10D7C00004F060FA002800F09B804FF48472D8F8CF
:10D7D0000910514BD1F81C8006460592039304941E
:10D7E0000346CDE90179CDF800B039460F22722009
:10D7F00001F020F9AB7B002B7AD19B469AF80E30D2
:10D80000002B7BD0DAF810300A934FF0000A12A8F0
:10D81000CDF854A0CDF868A0CDE916AACDE918AA94
:10D82000CDE91BAACDE91DAAF6F790FC099013A833
:10D83000F6F792FC18236FF009010A221AAF079736
:10D840000293364F139BDFF8E490CDE90421039750
:10D850000193C0B2CDF800B0CDF818901FAB32469E
:10D860004146F5F74FFE07468DF83F0000285FD090
:10D8700040F23512244B009229495246642001F0AF
:10D8800021F901254FF49B72264B059203930494D2
:10D89000CDE901AA00952A4629460DF13F036420EF
:10D8A00001F0C8F88DF84450F3F744FF9DF8443078
:10D8B000012B00F0238140F213221B4B00921A68C7
:10D8C0001449114B632001F0FDF80020119BDAB2DE
:10D8D00062F30700C3F3072262F30F20C3F307428A
:10D8E00062F317401B0E63F31F604FB0BDE8F08F6B
:10D8F0009AF80E30D5F810B0002B83D10A9384E744
:10D900008DF84470D7E700BF348D0100C87801005E
:10D91000AC0B0020248D01009C8D01000080FFFFD6
:10D92000A48D0100CC8D0100B00B0020708E010091
:10D9300000F062FB1FAB95F91D20CDF81480049315
:10D94000B5F91A300B900393B5F91810BDF97000B2
:10D950000291B5F916C0BDF97230CDF804C0B5F921
:10D9600014C00344CDF800C010990F2004F010FF3C
:10D9700040F249114FF0010B059104200621B84AED
:10D980004346CDE901B100905946039262200F222F
:10D99000049401F04FF800F07DFBDFF8F0A2804620
:10D9A00000F074FBDAF80020109BB3EB420FFFF697
:10D9B0007BAF00F021FC0C9000F04EFBDAF8003059
:10D9C000109A03FA0BFA92FBFAF30AFB132A0C9B48
:10D9D0000D90D3F80930D8F80920D3F81C80BAF19B
:10D9E000000F00F09380BAF1040F7FF45DAF4FF4A5
:10D9F000E870DFF888929B4915694B4605900391C2
:10DA00005A46594664200494CDE901B7CDF800A0E8
:10DA100001F010F84FF0C1430B9805950493B0F94D
:10DA20001A20D9F800300392B0F918201099029208
:10DA3000B0F9162002250192B0F914204FF4F070CD
:10DA400000923A4604F0A4FE40F2DD11864A4FF0FF
:10DA5000C143059103920F21202262200494CDE955
:10DA600001B7009500F0E6FF40F2DF137F4A05930F
:10DA700003927F4B20225946422000950494CDE921
:10DA800001B700F0D7FF4FF4F0717A4A1FAB059150
:10DA9000039259460F22422000950494CDE901B724
:10DAA00000F0C8FF724B0D99CDE90438B1F91A2086
:10DAB000D9F800300392B1F918200B980292B0F90E
:10DAC000162010990192B0F91420202000923A46B5
:10DAD00004F05EFE40F2F1100623674ACDE901B37F
:10DAE000059003920494CDF800A0434659462022A5
:10DAF000622000F09FFFC9F80070D5E600225F4B5E
:10DB000031460F201A6004F0D3F8D4E69B69D76839
:10DB10000B93FFF7E3FDFFF7F5FD0C9A107802F089
:10DB2000DFFC02F091FDFFF705FE4FF4C071042009
:10DB3000534A3B460090059103920F212022722008
:10DB40000494CDE901BA00F075FF40F28111042080
:10DB50004C4A0B9B0090059103925946202272205B
:10DB60000494CDE901BA00F065FF9A22514627A836
:10DB700009F007F85046F6F74FFB27A8F6F792FB97
:10DB80004FF4C97205920222BDF8BA10BDF8B6C0B2
:10DB90003A4F354B8C44009203930494CDE901BA7B
:10DBA0004FF0C143C7F800C020220F21692000F0C8
:10DBB00041FF40F2931104202A4A3B460090059110
:10DBC00003920494CDE901BA5A465946692000F0FF
:10DBD00031FF95F83270002F5AD0002515ABCDE9F2
:10DBE00003930C9B0595D3F801C0DFF88490129F36
:10DBF0000CF1150CCDF808C0DDE90A3241469DF85C
:10DC00002400CDE90097F5F789FB4FF0010840F2B9
:10DC1000B5110220154A4B46CDE90441009041461A
:10DC20006920039202952022CDF8048000F002FFC3
:10DC3000FFF7CCFC4FF4E570134B05900393CDE94F
:10DC4000015511ABCDF80080049442464146642052
:10DC500000F0F0FE9DF84430002B3FF425AE2AE69C
:10DC6000D88D01000C860100F08D01005073010079
:10DC70006415002044730100688E010060150020C7
:10DC8000E08D0100E88D0100588E0100940600200F
:10DC90002A992A4649422898F4F754F995F830A071
:10DCA000BAF1000F1FD1BDF9C0301E2B95DD40F237
:10DCB000A512164B009216495246642000F002FF4E
:10DCC0004FF4D3720221134B0091059203930494F5
:10DCD000CDE901BA30AB5A465946642000F0AAFE9D
:10DCE0008DF844B079E740F29D12084B00920A4942
:10DCF0003A46642000F0E6FE85F83070384607F0BA
:10DD000019FB4FF002038DF8463066E7348D0100B1
:10DD1000148E01003C8E0100F88D0100D42330B533
:10DD20000E4A0F4D0F4C83B02146126863200093BA
:10DD30002B4600F0C7FE0C4A0C4B127853F82230E9
:10DD4000DB689847D6200A4A2B4612682146009085
:10DD5000632000F0B7FE03B030BD00BFAC0B002065
:10DD6000B88E0100A48E0100A4150020D406002066
:10DD7000B00B0020AB2330B50E4A0F4D0F4C83B0D3
:10DD800021461268632000932B4600F09BFE0C4A4C
:10DD90000C4B127853F822305B689847AD200A4A42
:10DDA0002B46126821460090632000F08BFE03B0E2
:10DDB00030BD00BFAC0B0020B88E0100988E010072
:10DDC000A4150020D4060020B00B00202DE9F0415E
:10DDD0002F4E304F337882B057F823309B689847E6
:10DDE000C4B2009007F09CFA027E437E002A0546EA
:10DDF00018BF012493BBAB7973B1337863B90225A3
:10DE00000424A84657F82330DB68984757F8283091
:10DE100035705B68984704E0AB7903F0FF05BBB150
:10DE200014BB04F089FA00208DF80040009BDAB2A0
:10DE300062F30700C3F3072262F30F20C3F3074224
:10DE400062F317401B0E63F31F6002B0BDE8F08160
:10DE50003378022BE4D1A8460124D3E700F0CCF8B4
:10DE6000012380F83230C6E7022C0BD0042C0CD0F2
:10DE7000012CD6D14FF0000833784345D1D05FFA5A
:10DE800088F5BFE74FF00108F6E74FF00208F3E727
:10DE9000A4150020D40600202DE9F84300F0ACF9C9
:10DEA000074600F0ABFA064600F0FEF9054600F022
:10DEB000F1F8814600F0F2F88046F6F743F904469F
:10DEC00000F09EF9204600F09DFA00F0F1F900F014
:10DED00097F8C9F80D0000F097F8C8F80D0000F0A9
:10DEE000B7F8C7F80D0000F0CDF8C6F80D0000F047
:10DEF000B7F8C5F80D0000F009F9064600F006FA7B
:10DF00000546204600F006F9204600F003FA00F02E
:10DF100097F8C6F80D0000F0ADF8C5F80D00BDE8A3
:10DF2000F88300BF30B583B0FFF7B6FF9D220F4BDB
:10DF300000921A680E490F4B632000F0C3FD0E4C8F
:10DF400004F10C0554F8043B1B689847AC42F9D126
:10DF5000A5230025094C0A4A05491268632000934D
:10DF6000044B257000F0AEFD03B030BDAC0B0020BB
:10DF70008C8E0100B88E0100D4060020A41500206C
:10DF8000B00B002008B500F061F900F061FA00F074
:10DF9000A5F900F0F5F8BDE8084000F0F1B900BFC0
:10DFA000DC2230B50F4B83B000921A680E490F4B3C
:10DFB000632000F087FD0E4C04F10C0554F8043B7F
:10DFC0001B699847AC42F9D1FFF7DCFFE022094B0F
:10DFD00000921A680449054B632000F073FD03B0FA
:10DFE00030BD00BFAC0B0020B08E0100B88E010028
:10DFF000D4060020B00B002000487047E006002047
:10E000000048704724070020004870473007002070
:10E01000024A8021024808F055BC00BF3878010050
:10E02000A81500200149024808F0D8BC3878010042
:10E03000A8150020014B1868704700BFA8150020E4
:10E0400000487047380700200048704750070020FC
:10E050000048704784070020004870479C07002054
:10E0600000487047D00700200023014883737047A1
:10E07000E8070020004870471C080020004870474F
:10E0800034080020004870476808002000487047A6
:10E090008008002000487047B408002000487047FE
:10E0A000CC08002010B5064C04F11000F6F74EF82D
:10E0B000207504F11800F6F74FF82077204610BDC0
:10E0C00008090020024A4FF4F071024808F0FABB38
:10E0D000A8940100E40800200149024808F07EBC31
:10E0E000A8940100E4080020024A4021024808F0F8
:10E0F000E9BB00BFBC9401002C0900200149024883
:10E1000008F06CBCBC9401002C090020004870474A
:10E110004409002070B54678124CB500294604F138
:10E120000C00114A08F0CEFB294604F118000F4AF2
:10E1300008F0C8FB294604F11C000D4A08F0C2FB98
:10E14000314620460B4A08F0BDFB2946201D0A4AED
:10E1500008F0B8FB294604F10800084ABDE8704001
:10E1600008F0B0BB5C09002018A2010034A2010035
:10E170004CA2010064A2010080A201009CA2010047
:10E1800010B50F4C0F4904F10C0008F027FC04F106
:10E1900018000D4908F022FC04F11C000B4908F09E
:10E1A0001DFC20460A4908F019FC201D094908F009
:10E1B00015FC04F108000849BDE8104008F00EBC49
:10E1C0005C09002018A2010034A201004CA2010049
:10E1D00064A2010080A201009CA2010010B5054CC0
:10E1E00004F10C00F5F7B2FFE368207523612046C7
:10E1F00010BD00BF8409002000487047C0090020FE
:10E2000070B546780C4CB500294604F11C000B4A49
:10E2100008F058FB31462046094A08F053FB2946CE
:10E22000201D084A08F04EFB294604F10800064A62
:10E23000BDE8704008F046BBD809002058A3010093
:10E240006CA3010088A30100A4A3010010B50A4C2F
:10E250000A4904F11C0008F0C1FB2046084908F0F7
:10E26000BDFB201D074908F0B9FB04F10800064971
:10E27000BDE8104008F0B2BBD809002058A3010047
:10E2800004A301001CA3010034A3010010B5054C38
:10E2900004F10C00F5F75AFFE3682075236120466E
:10E2A00010BD00BF000A0020004870473C0A002053
:10E2B00010B5074C074A04F108000C2108F002FBD6
:10E2C0002046BDE81040044A062108F0FBBA00BF12
:10E2D000540A0020D0A30100E8A3010010B5064CA9
:10E2E000064904F1080008F079FB2046BDE810401B
:10E2F000034908F073BB00BF540A0020D0A30100FB
:10E30000E8A30100004870476C0A002000487047ED
:10E31000A80A002070B50678124CB500294604F111
:10E320000C00114A08F0CEFA294604F118000F4AF1
:10E3300008F0C8FA294604F11C000D4A08F0C2FA98
:10E34000314620460B4A08F0BDFA2946201D0A4AEC
:10E3500008F0B8FA294604F10800084ABDE8704000
:10E3600008F0B0BAC00A002044A4010060A4010073
:10E3700078A4010090A40100ACA40100C8A401008D
:10E3800010B50F4C0F4904F10C0008F027FB04F105
:10E3900018000D4908F022FB04F11C000B4908F09D
:10E3A0001DFB20460A4908F019FB201D094908F009
:10E3B00015FB04F108000849BDE8104008F00EBB49
:10E3C000C00A002044A4010060A4010078A4010058
:10E3D00090A40100ACA40100C8A4010010B5064C33
:10E3E00004F10C00F5F7B8FE207504F11000F5F704
:10E3F000B9FE204610BD00BFE80A00200048704763
:10E40000240B002070B506780C4CB500294604F1A9
:10E410001C000B4A08F056FA31462046094A08F01B
:10E4200051FA2946201D084A08F04CFA294604F101
:10E430000800064ABDE8704008F044BA3C0B0020D2
:10E4400090AB0100A4AB0100BCAB0100D4AB010058
:10E4500010B50A4C0A4904F11C0008F0BFFA204626
:10E46000084908F0BBFA201D074908F0B7FA04F183
:10E4700008000649BDE8104008F0B0BA3C0B002087
:10E4800090AB0100A4AB0100BCAB0100D4AB010018
:10E4900010B5064C04F10C00F5F75EFE207504F192
:10E4A0001000F5F75FFE204610BD00BF640B002092
:10E4B0002DE9F843F5F746FE0446FFF7F3FD054660
:10E4C000FFF7E4FE8046FFF7E3FF0746FFF71AFF7A
:10E4D000224606462946012001F0F4FD224629463F
:10E4E000022001F0EFFDFFF779FE8146FFF776FF8E
:10E4F000054622464946092001F0E4FD2246294608
:10E500000A2001F0DFFD22464146052001F0DAFD38
:10E5100022463946062001F0D5FD22463146072025
:10E5200001F0D0FDFFF7CEFDBDE8F843FFF7DCBDFD
:10E5300010B5FFF7BDFF094B1B689847084B1B68D8
:10E540009847084B1B689847BDE81040064A074BA0
:10E55000127853F822305B68184700BFC0060020CD
:10E5600028060020F0050020AE15002030AC010088
:10E57000F8B5FFF797FD0446FFF788FE0746FFF75B
:10E5800087FF0646FFF7BEFE0546FFF7A5FDFFF72E
:10E59000B5FD2146012001F0E3FD2146022001F0F6
:10E5A000DFFD3946052001F0DBFD3146062001F094
:10E5B000D7FD2946072001F0D3FDFFF70FFE0546E2
:10E5C000FFF70CFF04462946092001F0C9FD21464A
:10E5D000BDE8F8400A2001F0C3BD00BF70B50024BB
:10E5E0009AB010AE2146304628220BADCDE90B443F
:10E5F000CDE90D440F9408F0C4FA08ABCDE903331C
:10E60000CDE90544CDE900560648029308940994E3
:10E61000ADF828402B4604682A4629460A20A04720
:10E620001AB070BD142400200C4A0D4B127810B59E
:10E6300053F82230DB689847FFF7D0FFFFF798FFC9
:10E64000F5F758FF074B1B699847074B1B6998471D
:10E65000BDE81040054B1B69184700BFAE150020F0
:10E6600030AC0100C006002028060020F005002084
:10E6700070B5064606F048FE174D012804462B7873
:10E680001CD09EB99C421BD0012B1AD0134E56F8B9
:10E690002330DB68984720462C7006F03BFE2B7831
:10E6A00056F82330BDE870405B681847012E0FD044
:10E6B000032EE7D1022B03D00224E5E7012B00D182
:10E6C00070BDFFF7B1FF2C70BDE87040FFF730BFA1
:10E6D000002BF5D00024D7E7AE15002030AC0100A8
:10E6E0004E4A2DE9F04112784D4B88B053F8223054
:10E6F0004C4E9B6898470790C0F30728C0F3074427
:10E7000006F00EFE054606F00FFE474BEA7B197831
:10E71000914216BFEA7B07461A70444B18BF012787
:10E72000986804F099FDF6F729F833688DF81A0017
:10E730009B78834215D00122D3210023DFF800C14A
:10E740003B480591CDE90133CDE9030C0DF11A03E6
:10E7500064200092114600F06DF933689878F5F75F
:10E76000FBFFF6F725F833688DF81B00DB78834252
:10E770000CD11FBB002C43D12B7E002B47D1404630
:10E78000FFF776FF012008B0BDE8F0810122D92112
:10E790000023DFF8ACC027480591CDE90133CDE96E
:10E7A000030C0DF11B0364200092114600F042F9A6
:10E7B0003368D878F5F7E8FF002FDBD0002006F0AB
:10E7C000B9FD2B7E13B1002006F0A4FD64221A4B84
:10E7D00000921A6819491A4B632000F073F9FFF789
:10E7E00023FFFFF7A5FE6722164B00921A68134914
:10E7F000134B632000F066F9012008B0BDE8F081FA
:10E800006B7E002BB8D12B7E002BDCD1DEE7002005
:10E8100006F080FD4FF00108B1E700BFAE15002003
:10E8200030AC0100D80C0020AD150020B40C002045
:10E830001CAC010024AC0100AC0B0020F8AB0100C3
:10E840000CAC0100B00B00202DE9F04792B004465B
:10E85000884606F065FD00233F4FC27DC7E90033BF
:10E860003B81002A56D094F82B0094F82AA094F803
:10E870002990504594F8281038D8A0F1160EC21FE0
:10E88000A0F10F065FFA8EFED2B2F6B2894521D80A
:10E890004B4612E0A3F10A04022C4ED800EB4314BD
:10E8A00038F91450002437F914C0AC45B8BF27F824
:10E8B00014500133DBB299420CD3022AEAD9022E5A
:10E8C0002BD89C1F022C28D800EB4315022438F9C2
:10E8D0001550E8E70130C0B20EF1010E01320136E9
:10E8E00082455FFA8EFED2B2F6B2CFD23E2200212E
:10E8F0000DF10A0008F045F9002340F20155822489
:10E9000000971A4602A91E20ADF808508DF80D4058
:10E9100006F07AFE12B0BDE8F087BEF1020FC8D84B
:10E92000A3F10A04022C11D99C1E022CC1D800EBC1
:10E93000431438F914500424B5E79C1E022CB8D8AF
:10E9400000EB431438F914500124ACE700EB4314F6
:10E9500038F914500324A6E7B0150020F0B5204E76
:10E9600083B0054601F1200014461F467160F1F79F
:10E9700089FC1C4B1C4A99682130376048609460C0
:10E9800060782278E37802FB00F203F07F0303FB58
:10E9900002F3164C22790B60D3B2012B01D003B0E5
:10E9A000F0BD7721FF221E46114F39702271237965
:10E9B000FF2B10D120222946684608F0B3F8009BAF
:10E9C000032B04EB830206DC019BD2F8052006FA38
:10E9D00003F31342EBD105233B7003B0F0BD00BF3E
:10E9E000201C0020040D0020440F00205C1D00208E
:10E9F000D40D002070B504460E461546049A1946FB
:10EA000020F8022B20341E2208F07AF920463146E5
:10EA1000DF2208F075F945B13046F1F733FC29469D
:10EA2000C0F1DF02204408F06BF92046BDE87040D9
:10EA3000F1F728BCF0B5C5B004460E4615460146B0
:10EA4000202204A81F4608F06DF8049B032B0EDC5F
:10EA500001221B48059900EB8303D3F805C002FA95
:10EA600001F313EA0C0F02D00379934201D045B0B1
:10EA7000F0BD4F9B4D99009300224E9B04A8FFF7D9
:10EA8000B9FF4FF0000E9DF80BC04A9B4B9A63F301
:10EA9000060C8DF80F0020464C9C62F3C71C3B46C9
:10EAA00004A902AA8DF808608DF809508DF80E406F
:10EAB0008DF80BC08DF80CE0FFF750FFD7E700BFD3
:10EAC0005C1D0020F0B5C5B004460D461646014653
:10EAD000202204A81F4608F025F8049B032B0EDC17
:10EAE00001221548059900EB8303D3F805C002FA0B
:10EAF00001F313EA0C0F02D00379934201D045B021
:10EB0000F0BD4A9B3246009329463B4604A8FFF7D6
:10EB100071FF00258DF80F0004A902AA20462B469C
:10EB2000ADF808508DF80B508DF80C508DF80E5044
:10EB3000FFF714FFE3E700BF5C1D0020F0B564465B
:10EB400087B001F049FD002601F07EFD012504207B
:10EB500040F21D372369A268DB68E168CDE9015600
:10EB60000090064D06480597CDE903057220FFF792
:10EB700061FF2369D86807B0F0BD00BF34AD010064
:10EB80009CAC01002DE9F04F91F81CE090F802C018
:10EB90000F460EFB0CF5097D85B00191DDF838803C
:10EBA0004DB34446002605EB450C08EB0C1C2262D5
:10EBB00094F8245084F8246094F8255084F8256053
:10EBC00094F8265084F8266094F8275084F827603B
:10EBD00094F8285084F8286094F8295084F8296023
:10EBE00094F82A5084F82A6094F82B5084F82B600B
:10EBF0003034A445DBD1BEF1000F32D03D460026B3
:10EC0000074603F1FF3921B3CB4600242B690622C6
:10EC100013F804A002A84FEA6A01013107F082FF4D
:10EC2000BA780AF0010306FB0233029A03EB4303AE
:10EC3000920002EB0313039943441BF8012F186A57
:10EC400001EB81018A4002431A622B7D0134A34209
:10EC5000DCDC2B7F0136019AB342914401DD297D32
:10EC6000D1E705B0BDE8F08F2DE9F041002482B076
:10EC7000089D2A622A6595F8242085F8244095F895
:10EC8000252085F8254095F8262085F8264095F81A
:10EC9000272085F8274095F8542085F8544095F8AA
:10ECA000552085F8554095F8562085F8564095F83A
:10ECB000572085F8574095F8282085F8284095F882
:10ECC000292085F8294095F82A2085F82A4095F8CA
:10ECD0002B2085F82B4095F8582085F8584095F85A
:10ECE000592085F8594095F85A2085F85A4095F8EA
:10ECF0005B2085F85B400A7D12B30F465E1E3B69C0
:10ED0000062213F8048068464FEA6801013107F0D3
:10ED100009FF08F00108009A4FEA4803984493005D
:10ED200003EB081301992B4416F8012F186A01EB25
:10ED300081018A4002431A623B7D0134A342DEDC3A
:10ED400002B0BDE8F08100BF2DE9F04F97B06846F2
:10ED5000D1F8013006AF1E7D1D7F796006FB05F3FB
:10ED6000D1F809205C00FA62DA1DD208A0EBC200DB
:10ED7000854604F10803DB08DB0006A8ADEB030DB4
:10ED8000F86006A8ADEB030D06AAADEB030DFB6A18
:10ED9000BC60DB68BA623B620A2322467400A0466C
:10EDA000FF217B61386107F0ECFE06AB7B62B300AC
:10EDB0007B637A697B681F2AD3F8053040F3198199
:10EDC00010464446954901FB02F102EB421200EB6A
:10EDD000421202EBC23201F1404102F140422031C5
:10EDE000013241F01F0103F5B46019625A629A6260
:10EDF00030338342F9D18A480122049089488D2119
:10EE0000039004230020A0460290019205910093F4
:10EE10007C6907F13C0311466420FC63FFF70AFE9E
:10EE2000BC6800212246B86A07F0ABFE2246FF21EB
:10EE3000786A07F0A6FE142344463B6301F0CCFB3E
:10EE400001F002FC0421FB6A4FF0000CDB6800912A
:10EE500096210591724920220491734972200391F1
:10EE60000121CDE9011C0F21FFF7E4FD45B34FF06F
:10EE700000093B6AD7F824A0A3F1040BBB6AA3F1F5
:10EE80000208002E00F0AB80D446DE464346A04484
:10EE90005EF8042F33F8020FBCF800108242C8BF9E
:10EEA00090B28A42B8BF91B2434518802CF8021B39
:10EEB000EED109F101097B6B4D459B44A244E0D1A1
:10EEC0003B6B013B3B63B9D1A046002D35D09B463F
:10EED000BB6AD7F80C90023BFB617B6AD7F81480C1
:10EEE000023B3B633B69BD61A3F1020AB6B15046E8
:10EEF0000021D7F830C0FD6935F8023F3CF802EF39
:10EF000030F8022FA3EB0E039A42C8BF09F8018024
:10EF100001F10101C8BF03808E42EDD1FB690BF105
:10EF2000010B2344FB613B6BA24423443B63BB695D
:10EF3000B1445B45DAD1A046BD69A9217869FB6A75
:10EF400001307861DB680591354904220491364926
:10EF500004460391002001210092CDE901102022F6
:10EF60000F216420FFF766FD3E2C7FF422AFAC2218
:10EF70002B4B00922D4900226420FFF7A3FD0020B7
:10EF8000CDE901000120AD21254B294A00900493D1
:10EF9000FB6864200591039229463246FFF74AFD3B
:10EFA000AF221F4B0092234900226420FFF78AFD05
:10EFB0001B4B4FF0B00C049300230224CDE9013326
:10EFC0001D483B69324603902946CDF814C0009491
:10EFD0006420FFF72FFD4437BD46BDE8F08F09F1EF
:10EFE00001097B6B4D45A0449B44A2447FF449AF8B
:10EFF00066E77A6944461146084800FB02F002EBD6
:10F00000421201EB421202EBC23203F5B461186204
:10F010005A629A6230338B42F9D1ECE620841002B6
:10F0200034AD0100ECAC01009CAC0100F8AC010077
:10F030000CAD010018AD010028AD01002DE9F04F25
:10F04000D2F80180D2F805C098F81C9098F814A066
:10F05000B9F1000F22D04FF0000E0139BAF1000FC4
:10F0600017D00C468678D8F810200EFB06F60AEB6F
:10F07000020712F801BB14F8015F0BF001033344DF
:10F0800003EB43030CEB031303EB5B039742DD73CA
:10F09000EFD10EF1010ECE455144DFD1BDE8F08F26
:10F0A000F0B5DCE9002087B064460F46FFF7C6FFE5
:10F0B000D4E90221002040F227360125CDE90100E4
:10F0C000054C06483B46CDE90304059600956420AF
:10F0D000FFF7B0FC07B0F0BD34AD010064AC010037
:10F0E0002DE9F04F8DB082788A4602EB4202120180
:10F0F00000AFADEB020D6E46F8610021684607F0E7
:10F1000040FD4FF4B4620021C84807F03AFD9AF878
:10F110001450BE6135B3DAF810000124054406E04E
:10F120005368854243EA0E0EC2F804E01AD010F884
:10F13000013B03F0010C4FEA4C0262441F2B04FA1E
:10F1400003FE06EB0212EBDD117A203B8C4604FA3B
:10F1500003F3C1F301010B4363F3010C854282F811
:10F1600008C0E4D19AF81C30BB62002B00F0838108
:10F17000DAF81820002411460120FA62194412F826
:10F18000013B00FA03F3914244EA0304F7D1FB691F
:10F190003C6293F802C0BCF1000F00F07D810021B9
:10F1A000BA69C7F82CA010460D464FF0030B4FF07C
:10F1B000190992463B6AC3F313065FFA86F8C6F351
:10F1C000072E360C01EB41030AEB03135C781A7A25
:10F1D0006FF3C3045C709C7A02F0030224F03F04D6
:10F1E0009C7293F82E401A7224F01F045D7283F80B
:10F1F0002C5083F82D5083F82E4003F1080280F83C
:10F200000BB080F82F909379013123F00F03334333
:10F210008C4582F8048082F805E000F1300093719B
:10F22000D0D14FF040533A6AD7F82CA09A64BB6A09
:10F23000002B00F02A81DAF81830FB6200234FF02F
:10F24000010B7B629946794BBB624FF0000CFB6A65
:10F2500029F0030213F80930BC6A0BFA03F8C8F36B
:10F260001308C8F30D039B00BB604FEA98337B6023
:10F27000131D3A61FB60C7F81480A6464FEA4C059F
:10F28000BB69654403EB051505F13008764628682F
:10F290006968AA68EB68103545450EF1100E0FC677
:10F2A000F4D12388796A9AF80B2061F3090323804B
:10F2B000002A40F0BD8023687A6962F31F3323601F
:10F2C000FB699AF80C00DB783A6A0BFA03F3013811
:10F2D00042EA03019AF81C20032800F2C880DFE804
:10F2E00000F0825B3602206894F82E5043EA10301A
:10F2F00025F01F05C0F31403013A45EA13454A45BA
:10F30000A08584F82E500FDDFA6A4A445078EAB29C
:10F310000BFA00F00343C3F3140322F01F0242EA86
:10F320001342A38584F82E20B9F1000F08D0FA6AA1
:10F330004A4412F8012C0BFA02F21343C3F31403EC
:10F3400083F4FF1383F4FF5383F01F032AE0E36A7F
:10F35000013A4A45C3F3140311DDFA6A4A4450786E
:10F3600094F82E200BFA00F00343C3F3044022F07C
:10F370001F020243A38584F82E20C3F31403B9F1BE
:10F38000000F0FD0FA6A4A4412F8012C0BFA02F26D
:10F390001343C3F3140305E0226843EA1233DB434B
:10F3A000C3F31403E2681940A07B94F82E30C2F333
:10F3B000130222EA0102A18520F00F0023F01F03AF
:10F3C000C1F3044140EA12401943A281A07384F8BA
:10F3D0002E103034BCF1000F15D1DAF818304FF090
:10F3E000010CFB6249E794F82E20C3F31403194083
:10F3F00022F01F0242EA1142A18584F82E20303407
:10F40000BCF1000FE9D07A6A9AF81C302032C2F3BE
:10F4100009027A62BA6A09F1010960324B45BA629F
:10F4200033DDDAF81830FB620FE700BF98000460A4
:10F43000FB6A3A699918FA689D1811F8013B20682F
:10F440000BFA03F3226843EA103363F31F328D4251
:10F450002260F2D12389BA6803F0030313432381A6
:10F46000A37A7A6823F03F031343A37228E7E36A81
:10F47000C3F3140396E7FB6993F802C0BCF1000FD5
:10F4800007D14FF04053C3F848C03437BD46BDE8FC
:10F49000F08FBB6A3B6282E64FF040533A6A9A644F
:10F4A000CCE600BF2DE9F041827800AF02EB4202CA
:10F4B0001201ADEB020D884605460021684607F0B3
:10F4C00060FB302200215B4807F05BFB6FF01F01FF
:10F4D0009DF8013098F80C2003F0F40343F0090381
:10F4E000013A8DF800108DF801306C46032A03D8DC
:10F4F000DFE802F0877302024FF0FF324FF0405115
:10F50000002094F82E3084F82C2043F01F0384F858
:10F510002E3084F82D20C1F83001002104F130058F
:10F520002A462346E172D3F800C05E689868D9681D
:10F530001033AB42C2F800C056609060D16002F157
:10F540001002F0D198F814303BB3D8F8100001261F
:10F5500003EB000C06E05368844543EA0808C2F850
:10F5600004801AD010F8013B03F0010E4FEA4E025E
:10F5700072441F2B06FA03F804EB0212EBDD117A3A
:10F58000203B8E4606FA03F3C1F301010B4363F3FC
:10F59000010E844582F808E0E4D12646DFF894E0C5
:10F5A000F44630687168B268F3681036AE420EF106
:10F5B000100EACE80F00F3D1DFF880C06034654670
:10F5C00030687168B268F3681036A6420CF1100C0E
:10F5D0000FC5F4D1BD46BDE8F0814FF0FF324FF0CA
:10F5E0004051002094F82E3084F82C2023F01F0383
:10F5F00043F00F0384F82E3084F82D20C1F8300139
:10F600008BE701224FF04051E87894F82E30824089
:10F61000C2F3044523F01F0307482B43C2F3072519
:10F6200084F82C2084F82D5084F82E30C1F8300155
:10F6300073E700BF38060460FFFF0F006806046030
:10F64000F0B50D46A9B04C220021044602A807F0EF
:10F6500098FA00204FF040522978ADF8040082F863
:10F66000A8106978BDF80420A87861F38A12C2F363
:10F67000072160F3C601ADF804208DF80510BDF830
:10F68000041002AB0DF12A02598502339342FBD1DB
:10F690004FF04056002286F8A7202F7DC7B14FF0CB
:10F6A000010C2969013911F8013F28A818441C2BC5
:10F6B00000F8982C02F1010208DD96F8A7001D3B26
:10F6C0000CFA03F30343DBB286F8A7309742EAD182
:10F6D00002A915A84C2207F049FA15A94C2209489D
:10F6E00007F044FA4C2215A9074807F03FFA2946CB
:10F6F0002046FFF7F5FC20462946FFF7D3FE0248D7
:10F7000029B0F0BD4C000460000004602DE9F04F0A
:10F71000D0F80D40D0F80160D4F800C0D6F820E051
:10F720009CF800309CF8012096F80090D5185FFAFC
:10F7300085F808F1010B03F1010A0F46591ED0F8B4
:10F74000090089B08EF829B08EF822808EF824A0A6
:10F750008EF82510B9F1000F4CD001328EF8272019
:10F7600000238EF828301A46636893F8008008F06A
:10F770003F0802F114030EEB43039978013268F35A
:10F780000501112A9970F4D119211C4B1C4A83F8E8
:10F790002F1030339342FAD133796BB143685BB1A8
:10F7A000164D9CF80D20314600953846FFF7EAF9D2
:10F7B00023685A781B78D51849F6404301356D0007
:10F7C00093FBF5F54FF4EF7001220021042608ABFE
:10F7D00043F8045D0B4C05900B48CDE90121CDE9C0
:10F7E0000304114600966420FFF724F9034809B08A
:10F7F000BDE8F08F0A3B8EF82730B1E7980004602F
:10F800003806046034AD0100ACAC01002DE9F047CE
:10F81000D0F80D80D0F80150D8F800302C6A93F859
:10F8200001C01B7895F800E00CEB0302D2B202F1A4
:10F83000010A03F101090F46591ED0F8096082B090
:10F8400084F875A084F86E2084F8709084F87110A4
:10F85000BEF1000F41D00CF1010C84F873C00023FD
:10F860001A4684F87430D8F804C09CF8020000F0FE
:10F870003F0002F1140304EB430393F84E100132EE
:10F8800060F30501112A83F84E10F2D11923154AAD
:10F89000154C301D84F82F3082F82F309CF8001062
:10F8A000124AC90107F00EF8D8F80430104A197846
:10F8B00006F10800C90107F005F82B794BB173690F
:10F8C0003BB1D8F800202946527B38460094FFF718
:10F8D000CBF9054802B0BDE8F0870A3B84F87330E5
:10F8E000BDE700BF680604603806046080AC010014
:10F8F00098AC0100F0B500264FF0405304240125D8
:10F90000D0F80D20D0F80110506812684670907839
:10F910004FF00F0E83F82C01D0784FF4B47C83F8AD
:10F920002D01107A83F82A01907A83F82B0110793F
:10F9300083F82E01507983F82F010F78C87883F867
:10F9400025714F7983F88E7083F8840083F8815095
:10F9500083F8806083F8AE4083F8AF400E7993F867
:10F96000890086EA050767F30510022783F88900F6
:10F9700093F8A10066F3041083F8A10083F88D408A
:10F9800083F8B05083F8C5E0A3F8C8C083F8CC7002
:10F99000947B087A83F800418C7983F80541CC790F
:10F9A00083F80A4183F80D01497A83F81011117B1D
:10F9B00083F8DA10D27A83F8A020F0BD4FF04053DC
:10F9C00010B5D0F80D10D0F809204C68526893F8A3
:10F9D00041116078054B02EBC01003EB014180221E
:10F9E00007F0C4F863780133637010BD80070160CD
:10F9F00070B5194B84B01B78044613B105F090FC28
:10FA0000C37ED4F80130DB7A23B3D4F80930DE6842
:10FA100006F1800506F50866A5F180000023194669
:10FA2000DA0182584DF823200133042B1144F7D119
:10FA300000225DF82230D401A1EB430301325B10B8
:10FA4000042A0351F5D10430A842E7D105F5007529
:10FA5000B542E1D104B070BDC51500204FF0405350
:10FA60002DE9F041012604240025D0F80D20D0F81E
:10FA7000011012684FF00F0890784FF0030E83F8D2
:10FA8000E000D07883F8E100107983F8E200507943
:10FA900083F8E300107A83F8E600907A83F8E700B1
:10FAA0004F79C87883F88E7083F8840083F881607A
:10FAB00083F8805083F8AE4083F8AF400F7993F815
:10FAC000890087EA060C6CF305104FF01E0C83F8D2
:10FAD000890093F8A10067F3041083F8A10083F86C
:10FAE0008D4083F8B06083F8C58083F887E0A3F881
:10FAF000C85083F8CCC0907B83F80001887983F8E4
:10FB00000501C87983F80A01497A83F81011117B3D
:10FB100083F8DA10D27A83F8A020BDE8F08100BF24
:10FB20004FF040532DE9F04101260025D0F80D108B
:10FB3000D0F80100D1E900219478497883F8E040B9
:10FB4000D4784FF0040883F8E14014794FF00F0E99
:10FB500083F8E2405479B14083F8E340147A3144A9
:10FB600083F8E640947AC9B283F8E7404779C478CD
:10FB700083F88E7083F8844083F8816083F8805026
:10FB8000077993F8894087EA060C6CF305144FF067
:10FB9000030C83F8894093F8A14067F3041483F8B9
:10FBA000A14083F88D8083F8B06083F8C5E083F8C6
:10FBB00087C0A3F8C85083F8CC10917B83F800115C
:10FBC000817983F80511C17983F80A11417A83F8A4
:10FBD0001011117B83F8DA10D27A83F8A020BDE8E7
:10FBE000F08100BF2DE9F04FA1B006AF07F1680525
:10FBF000634C644E45F8381D07F1540807F1440979
:10FC0000786394E80F0089E80F0007F190034846F5
:10FC10004146C9E902567B66F0F732FB94E80F00D3
:10FC2000594C88E80F00404607F16401C8E90254C6
:10FC3000F0F726FB012000F01FFC002800F09C805C
:10FC4000D0F8016007F10C0EEB4682463446F446CC
:10FC5000337D327FBB63FA6303FB02F206F12003BC
:10FC60007A603B606546E36820686168A26810348A
:10FC70000FC53B680CF1100C9C42F3D100252068A5
:10FC80007B68CCF800003A6B3D74CAF801E0D2F80A
:10FC900009C0D2F80D106A460733DB08A2EBC30295
:10FCA0009546096806AC4B787A68DCF8081020465F
:10FCB000C7F840C03B6006F059FF48F0010249F028
:10FCC00001003B68CDE90020D7F804801946424680
:10FCD0002346012002F090FD3B6C42462146186805
:10FCE00006F044FF40F22F3E01203B6CDFF8A0C03D
:10FCF000DFF8A080BA6B1B68F96BCDF80CC00090E0
:10FD0000CDF814E0CDE90155CDF810806420FEF760
:10FD100091FED7F83CC0AC4515DDB86BD7F840E094
:10FD200000280DDD0023327DDEF8201005FB0232B5
:10FD3000C95C14F80290013349448342A154F2D1C2
:10FD400001356545ECD121463A6B786BFFF776F9C2
:10FD5000D7E90E2140F2393C0020012523460B4C07
:10FD6000CDE90100CDE9048C009503946420FEF7F1
:10FD700061FECAF80160DD466C37BD46BDE8F08F14
:10FD800054AC01003DEB0000A1F0000064AC0100A8
:10FD900070AC010034AD01002DE9F04FADF50D7DE3
:10FDA00006AF78608A4600F057FA061E40F3C58019
:10FDB000002403E00134A64200F0BF802146012068
:10FDC00000F058FA0028F5D007F1140E0546F44665
:10FDD000D0F8014004F12008664620686168A268F6
:10FDE000E368103444450CF1100C0FC6F4D1002622
:10FDF00020684FF4F072CCF800008EF80460C5F86B
:10FE000001E0DAF80D3001211B6807F138005B785A
:10FE10001C46FB6006F0B5FEADF5F16D06AB18466D
:10FE200031464FF4F06206F0ACFE012C40F38980BD
:10FE30000124A146031FDFF82081BB60DAF80550DA
:10FE400005F10F0B05F2AF555846112221460BF173
:10FE5000300B06F096FEAB45F6D101224FF45A73F3
:10FE6000042539496420CDE902610593114607F163
:10FE70001003CDF81080CDF8049000953C61FEF79A
:10FE8000D9FD00F0A9FB00F0DFFB4FF45B732F4AB4
:10FE90000593CDE902624FF0C04320220F21009567
:10FEA000CDF81080CDF804907220FEF7C3FD4FF01E
:10FEB000C043B968DFF8A4C007F13802186851F8E8
:10FEC000045F04338542BCBF14700860634502F1CF
:10FED0000102F3D140F27A331D4A0593CDE9026263
:10FEE00007F13803CDF81080CDE9009620220F21CC
:10FEF0006420FEF79FFDFB680134A3429ED1524669
:10FF0000786807F13801FFF799F840F27E34002253
:10FF10000120104907F13803CDE901220090039137
:10FF2000CDF81080059420220F216420FEF782FD79
:10FF300007F50777BD46BDE8F08F0023D3F8013001
:10FF4000FFDEDFF81480DAE7BCAC0100CCAC0100C6
:10FF500064AC0100D4AC010034AD01008007006046
:10FF600008B500F071FB022000F086FAD0F80930E5
:10FF7000986808BD08B500F067FB012000F07CFA26
:10FF8000D0F80930D86808BD30B4D0F80D20D0F8CA
:10FF90000930526815789DB19C685B68803C03F11C
:10FFA0007C00E41A00EBC515A0F18003221853F879
:10FFB000041F834242F8041FF9D18030A842F3D1D4
:10FFC00030BC7047704700BF002070474FF040536F
:10FFD00093F84121002082F0010283F8412193F837
:10FFE000432182F0010283F84321704708B5F4F7FA
:10FFF00095FC044B044A4FF47A701A60BDE808403F
:020000021000EC
:10000000F5F718B8CC150020450401002DE9F0479C
:10001000482286B0FF212A4806F0B3FD01A8F4F774
:1000200095F8804602A8F4F797F8074603A8F4F776
:1000300099F818F0FF081DD04FF0000A4FF00109A1
:100040001F4E04AD019B082213F80A4028466100A8
:1000500004F0030406F066FD04EBC404049A34447F
:10006000059BA15C09FA03F30AF1010A0B43C2459F
:10007000A354E7D117F0FF071FD04FF000094FF04E
:1000800001080F4E04AD039B082213F809402846CF
:10009000610004F00304043404EBC404344406F0A7
:1000A00041FDDDE90423A15C013308FA03F309F102
:1000B00001090B43B945A354E5D106B0BDE8F0876B
:1000C0009C20002030B5013885B00C460A2810D895
:1000D000DFE800F03B3E0F3B26110F0F2611060014
:1000E00003A8F4F733F82246C1B2039801F01CFDCF
:1000F000A06305B030BD03A8F4F72EF80223C5B203
:1001000003992A460093204604F1150300F094FC5D
:1001100022462946039801F01BFBA06305B030BDC1
:1001200003A8F4F713F80223C5B203992A460093F3
:10013000204604F1150300F07FFC2246294603986F
:1001400000F0F6FFA06305B030BDCB7A002BD0D015
:1001500010462146FFF774FA206205B030BD00BF9B
:100160000138092808D8DFE800F008080807050565
:100170000505050500238B63704700230B6270475C
:10018000037810B5022B04460BD0042B03D10022B8
:10019000D0F801301A6200236374A374E3742375EA
:1001A00010BDD0F809000849043006F017FCD4F857
:1001B00009000649083006F011FC00236374A3749B
:1001C000E374237510BD00BF4CAD01006CAD0100A0
:1001D000002230B504460D4683B002AB43F8042D2F
:1001E00018460E4A152106F06DFB22780C4B294665
:1001F00053F8223020469847C4F80500A0682268CA
:100200006568E168019B98601A605D60D960226949
:1002100001981A61227D1A7503B030BD44AD01000A
:10022000A8AD01000B4B1A680AB90CE01A46D2F8C7
:100230001130002BFAD10023C2F8110043748374EB
:10024000C374037570471860002343748374C374C8
:1002500003757047BC150020054B1B6833B10020A7
:10026000D3F811300130002BFAD17047184670478F
:10027000BC15002070B5164B88B01B687BB10024FC
:1002800002E0D3F8113053B11A788242F9D1013427
:100290000029F6D0A142F4D1184608B070BD40F252
:1002A000B31001220024042608AB43F8041D094DB5
:1002B00005900948CDE90124CDE9030511460096D2
:1002C0006420FEF7B7FB2346184608B070BD00BF98
:1002D000BC15002090AD010098AD010070B5094E2D
:1002E00082B034684CB1084D0194D4F811402946CD
:1002F00001A806F073FB002CF6D10023C6E90033F9
:1003000002B070BDBC15002088AD0100F8B544688E
:100310000546F3F717FFACB123780B2B12D80B4E21
:100320000146074656F8333020469847D4F8110066
:1003300040B10378394606EBC30668607368984796
:100340000120F8BD00206860F8BD00BFE40B00206C
:1003500010B50446F3F7F6FE636843B11C78054A0E
:10036000014652F8342018469047012010BD184627
:1003700010BD00BFE40B002038B544680546F3F714
:10038000E1FE4CB12278054B014653F8323020464D
:10039000984700236B6038BD6C6038BDE40B0020CB
:1003A00070B582B005460C46F3F7CCFE4FF04053D3
:1003B00093F84121014682F0010283F8412193F82C
:1003C000432182F0010283F84321286818B90CE028
:1003D000D0F8110058B10278A242F9D10A4A6860F7
:1003E00002EBC40253689847012002B070BD40F28E
:1003F0001D26064D064C00962B4600222146642001
:10040000FEF760FBF7E700BFE40B002090AD0100B2
:10041000D8AD010038B504680546F3F793FE6CB11A
:100420006B685BB92178064B2A6803EBC1035B68F4
:1004300001466A6020469847012038BD002038BD3B
:10044000E40B002008B572B60848FFF7E3FF58B187
:100450000123074A1375BFF34F8F4FF0405200201E
:10046000044908721370937062B608BDBC15002071
:1004700000001050A4140020054B1B6833B11A78FB
:10048000824203D0D3F81130002BF8D118467047C0
:10049000BC150020044B11B143F820107047034AEB
:1004A00043F82020704700BFB40B0020C5FF0000B8
:1004B000094B70B51C68F3F745FE5CB10546074E65
:1004C00023782046294656F823309847D4F811401F
:1004D000002CF5D170BD00BFBC150020B40B00206E
:1004E00008B5104B5A6802B108BD01461846FFF71F
:1004F00057FF0028F8D00C4B1B682BB1F4F70EFA0D
:100500004FF47A70F4F796FD0123084A1375BFF390
:100510004F8F4FF0405200200549087213709370BE
:1005200008BD00BFBC150020C814002000001050FA
:10053000A414002038B50023064D074C074A08498B
:100540002B7223601160F4F76DFDBDE83840FFF7B2
:1005500079BF00BFA4140020D0150020C8150020CA
:100560004504010010B50024084B094A09491A60E6
:100570000C72F4F757FDF4F7D1F9BDE81040064BC3
:10058000064A4FF47A701A60F4F754BDC81500207B
:10059000EDFF0000A4140020CC150020450401004C
:1005A000002008B5074A084B08491A600872F4F79A
:1005B000B5F9074B074A4FF47A701A60BDE8084056
:1005C000F4F738BDEDFF0000C8150020A41400208A
:1005D000CC15002045040100002330B40124064955
:1005E000064D0748074A0B7207492B60047030BC60
:1005F0001160FFF727BF00BFA4140020D015002012
:10060000C5150020C81500204504010008B5F4F701
:1006100021FD00230249034A0B60136008BD00BF9F
:10062000C8150020D0150020024B5868003018BFB4
:1006300001207047BC150020024B1868B0FA80F00A
:1006400040097047BC15002008B507490820F3F79A
:10065000B5FFFFF72DFFF4F7FDFC00230349044A23
:100660000B60136008BD00BFCDFF0000C81500205F
:10067000D015002008B572B6F4F7ECFC0023084949
:10068000084A0B60136062B6074A516831B1536083
:1006900006490820BDE80840F3F790BF08BD00BF39
:1006A000C8150020D0150020BC150020CDFF00008B
:1006B00008B504490820F3F781FFBDE80840FFF7BB
:1006C000F7BE00BFCDFF000008B50449082006F0C2
:1006D0003FFBBDE80840FFF7EBBE00BFCDFF0000C9
:1006E0000822314838B5314C43682260304A6BB338
:1006F00000251978157002293AD0D3F8113033B398
:100700002948FFF703FE00283DD00123294A13752D
:10071000BFF34F8F4FF040520020274908721370EB
:1007200093701022254B2260D3F80021120708D5C0
:100730000022082422482349C3F880410270C1F8EE
:1007400040214FF0405300225A7038BD13701648B4
:10075000FFF712FE002501201B4B1749154A1B68A5
:1007600008721575002BDCD09847184B1D60D8E730
:10077000D3F80D2051680A784978013A9142BCDAE1
:10078000FFF7E6FD18B901220B4B1A72C9E70123E6
:10079000084A1375BFF34F8F4FF0405206490D7250
:1007A00013709370BDE700BFBC150020140000203B
:1007B000C415002000001050A414002000E100E047
:1007C0001000002000000250C4140020CC150020AE
:1007D000B8B4850005F10A0323F00703002800AF31
:1007E000ADEB030D11DD6B46043A15440239181FB9
:1007F00031F8024F52F8043F03FB04F3AA424FEAD8
:10080000132440F8043F1460F2D1BD46B8BC7047D1
:100810002DE9F043089D1DB34FF04C0C01264FF01D
:100820000009079CD2B20CFB054CC9B29719C0B2A3
:100830000F44A1F10A08A1F1030EFFB280448644DF
:10084000002B14BF45467546A0702671E770617194
:10085000A27184F81990A676E5714C346445EFD105
:10086000BDE8F083F0B5012A83B0164605460C4674
:100870001F462DDC0146684606F054F936B3009B4E
:100880003F2B1D46A8BF3F25019A002B134405F0BE
:100890003F05B8BF00253F2B1A46A8BF3F22002BBB
:1008A0004FF0000102F03F03B8BF002304F1100233
:1008B00007EB420C09B30A19103207EB4202907998
:1008C00065F3050090710131B142F3DB03B0F0BD77
:1008D000104605F0C1FF044106FB04F40F2C294625
:1008E00006DD0122684606F01DF90126009BC7E7D8
:1008F0003246684606F016F9C1E79CF8062063F315
:1009000005028CF80620DEE7F0B5012A83B0154613
:1009100004460E461F462DDC0146684606F002F9E5
:10092000009B2DB33F2B1C46A8BF3F24019A002BF0
:10093000134404F03F04B8BF00243F2B1A46A8BF5D
:100940003F22002B4FF0000102F03F03B8BF00230D
:1009500006F1100207EB420CF1B18A19103207EBD5
:100960004202907964F30500907101318D42F3D118
:1009700003B0F0BD104605F06FFFF30744BF06411A
:100980006E4321462A46684654BF06F1FF360136BB
:1009900006F0C8F8009BC5E79CF8062063F3050243
:1009A0008CF80620E1E700BF70B5DCF80C3086B0AB
:1009B000644600259847FFF747FED4E9012301214B
:1009C000042040F23D269B690295CDE90001064DC9
:1009D00006480596CDE903057220FEF72BF8A368BB
:1009E000986906B070BD00BF34AE010040AE010092
:1009F00070B5644686B0DCF808309847FFF724FEEF
:100A00000022012140F2AB360425636808489B6947
:100A10000292084A0596CDE90320CDE9005114223F
:100A20007220FEF707F86368986906B070BD00BFD2
:100A300034AE010040AE01002DE9F04F87B006AFA3
:100A40004578D7F82890D01D20F0070009FB05F560
:100A5000ADEB000D0DF1180A0E46504600219046F0
:100A60001C4606F08EF8A94541DB4FF0000B08F15B
:100A7000FF3921224FF0FF31204606F082F833780B
:100A80004FFA8BF0B8F1010FE0542DDD4FF0000E5E
:100A90006FEA060C711C11F8012BA356B3F1FF3F4E
:100AA00005D1431CAB42ACBF00235BB2A3549842B8
:100AB0001AD092FBF5F005FB1020012814BF01208D
:100AC0004FF0FF30204482569A420DD00CEB0102C9
:100AD0009145A1EB060200F09580904501DD184696
:100AE000D9E7BEF1000F4CD1BBF1000F46D09123E6
:100AF000DFF828B1009300225B4645496420FDF7EA
:100B0000E1FFB8F1000F6CDD013EB14606EB0801D4
:100B100019F8013F93FBF5F205FB12324945E25407
:100B2000F6D10121972000223A4BCDE904B0CDE95E
:100B3000011203930091234642466420FDF77AFF99
:100B40000AF1FF3316F8012FA256B14503F8012F21
:100B5000F8D1012100249B252F48CDF810B0039037
:100B60005346642042460595CDE901140091FDF7F6
:100B700061FF20460437BD46BDE8F08F4FF0010B02
:100B800077E7012187200022224BDFF890B0CDE9E2
:100B9000011205900091CDE9033B424623466420B3
:100BA000013EFDF747FF06EB08010AF1FF3316F897
:100BB000012FA256B14203F8012FF8D101240021E0
:100BC0008B251548CDE901410390CDF810B0642084
:100BD00053464246059500942146FDF72BFF2046DB
:100BE000C8E70121972500200A4ACDE901100392A8
:100BF000CDF810B023460595009142466420FDF7DC
:100C000019FFA6E79045BCDD4FF0010E184642E7FC
:100C100060AE010084AE010050AE010034AE0100B0
:100C20002DE9F047D2F8017006467A789846012AF5
:100C300018D9002814DD00244FF04C094D1E00E0A7
:100C40007A78510094FBF1F301FB134315F8010F7F
:100C5000611009FB03830134FFF704FEA642EFD1C4
:100C6000BDE8F0870028FBDD6FF0130907F11404DD
:100C70004D1EA9EB070926444FF04C0A00E07A7894
:100C800009EB040114F9013F01EBD17149100AFB92
:100C9000038315F8010FFFF7E5FDB442EFD1BDE87E
:100CA000F08700BF70B5644686B0DCF800200B4BBF
:100CB000FFF7B6FFD4E90123012140F246260020C8
:100CC000074D084C1B68CDE9010005960091CDE960
:100CD00003457220FDF7AEFE06B070BD1408046037
:100CE00034AE010020AE01002DE9F047D2F80170CA
:100CF00098467A78012A1CD9002818DD4D1E212437
:100D00004FF04C092E1800E07A78510094FBF1F373
:100D100001FB134315F8010F04EBD47109FB0383A6
:100D20004910FFF7F1FDAE4204F1FF34ECD1BDE80C
:100D3000F0870028FBDD07F114044D1E26184FF044
:100D400021094FF04C0A00E07A7814F9013F4FEA8C
:100D500069010AFB038315F8010FFFF7D5FDA642D1
:100D600009F1FF39F0D1BDE8F08700BF30B5644626
:100D700087B0DCF800200B4BFFF7B6FF4FF46D7522
:100D80000121002263680848084C1B68CDE9012254
:100D9000CDE903040595009114227220FDF74AFE67
:100DA00007B030BD9806046020AE010034AE0100EB
:100DB000F0B4147980F8E8405579049C80F8E95043
:100DC000957980F8EA50D57980F8EB50957A80F8DB
:100DD000EE50157B80F8EF508D790E7880F88E50AC
:100DE00090F8895045F0300580F8895090F8A1506E
:100DF0006FF3041580F8A150CD7880F8A950002E2B
:100E000051D180F8986090F88B5045F0010580F83A
:100E10008B500125072700264FF0060C80F88D70B7
:100E200080F8B05080F8C56080F8815080F880501C
:100E300080F8AEC080F8AF700D79002C80F8845037
:100E4000557CB8BF033480F89F50957CC4F38F0461
:100E5000DBB280F89E5080F89C60A0F8CA4080F811
:100E6000CD30D37C80F80031CB7980F805310B7A16
:100E700080F80A314B7A80F81031137D80F8DA302F
:100E800090F8A330917D61F3061380F8A33090F8B9
:100E9000A330D17D61F3020380F8A330537DF0BC11
:100EA00080F8A0307047012580F8985090F88B505A
:100EB0006FF3000580F88B50ABE700BF2DE9F047DA
:100EC000D0F80160D0F80930747882B06400D0F8AE
:100ED0000D5033B10F46024619687878264BFFF75C
:100EE0009FFEB76B95F80DC08CB34FF04C09384698
:100EF0004FF0000809FB04790CF01F0C0CF0030EF6
:100F00004FEA8E1E4FEA9C0C002101F1100300EB0A
:100F1000430393F806A0DA790AF03F0A22F00702A9
:100F200001314AEA0E0A42EA0C02112983F806A0AE
:100F3000DA71EAD190F84A3080F8488023F01F0334
:100F400080F8498080F84A304C308145DCD13378D4
:100F50002A78A9786878CDE90074FFF759FC40F643
:100F60001400234600902A4631464FF04050FFF7C8
:100F70001FFF02B0BDE8F0871408046049F6404343
:100F8000014411440331490093FBF1F140F28F1009
:100F900070B501220026042588B008AB43F8041D73
:100FA000064C05900648CDE90126CDE9030411461B
:100FB00000956420FDF73EFD08B070BD34AE010021
:100FC00010AE01002DE9F04FD0F80130D0F80D70CF
:100FD0005C785A798BB0660097F80380002A71D04C
:100FE000D0F80920126A002A6CD0197D97F810B049
:100FF000DB68F1B14FF04C0E94464A4A0CEB010A03
:101000000EFB062E03F1FF3919F8013F5B0866B1AC
:101010001033444A58001118CB799CF800504C32D8
:1010200065F3C7037245CB71F5D10CF1010CD445C2
:10103000EAD1002E67D04C223A490B4602FB061239
:1010400083F825B04C339A42FAD101AD28462422C8
:10105000002105F096FDB8F1010F3DD1002E57D0CB
:10106000A9464FF0000EDFF8C0804946DFF8BCC04B
:10107000002311E0012C05D1032B03F0010201DC58
:10108000724506D003EBC30208781CF80220024325
:101090000A700133082B06D0022CEBD19E45F1D10A
:1010A0000133082BF8D10CF1010CE04501F10101ED
:1010B000DED10EF1010E764509F10909D5D19DF871
:1010C00004100AE001AD28462422002105F059FD54
:1010D000B8F1010FC2D0DEB100214FF0000C114C6D
:1010E0002846002301E010F8011FE2180133092B04
:1010F0001172F8D10CF1010C664504F14C0407DDC6
:1011000015F8091FECE73146242201A805F039FD46
:1011100078783A78B978FFF731FF02480BB0BDE82C
:10112000F08F00BF14080460A52000209C20002040
:101130002DE9F04F83B04C230C4692F8018000AFAC
:101140004FEA480603FB06F3ADEB030D0021914681
:1011500005461A4668467B609A4605F012FD6946C8
:101160005FFA84FC002E53D06B461A240DEB0A0064
:101170005A781C7002F0EC0242F002025A704C33B2
:101180009842F5D1BCF1000F28D000204FF04C0B55
:101190004FF0010E013D05E05369013023436045E6
:1011A00053611ADA15F8013F09EB030292F9152091
:1011B0001F2B0EFA03F40BFB0212EDDD147E203B15
:1011C000A2460EFA03F3C4F301041C43013064F396
:1011D000010A604582F818A0E4DB86B100234C25A3
:1011E0005524B8F1020F07D105FB0312D07C5474CB
:1011F00020F001009474D07401339E42F1DC7A68CF
:10120000054805F0B3FC04480C37BD46BDE8F08F37
:10121000BCF1000FF3D0B8E714080460F0B5D0F8C3
:101220000130D0F809701E7D87B07D6ABB6806B3B7
:1012300000224FF4807C14E0786835F8124050F8B2
:1012400022002402012838BF0120B4FBF0F0B0F5E1
:10125000DC7F28BF4FF4DC7023F812000132B24269
:1012600007D028880028E7D123F812C00132B24203
:10127000F7D140F2F116002002254A78064C0749C2
:10128000CDE90100CDE90314059600950121642004
:10129000FDF7D0FB07B0F0BD34AE0100F4AD0100A6
:1012A0002DE9F04F97B0814606AFDFF8D8C16E4EFA
:1012B00007F11C0807F12C0407F10C05F960BA616D
:1012C00096E80F0088E80F00C8E9025C4046214616
:1012D00007F16803FB63EEF7D3FF96E80F00634E58
:1012E00084E80F00C4E90256204607F13C01EEF7FE
:1012F000C7FFFB6899F80120D3F80160D3F80D50BF
:101300007078D3F809A08001C7E9042A44F00104E9
:1013100005F0A2FAE98948F00105DAF800303A69E7
:10132000CDE9004501F024FBDAE900013D69EB4617
:10133000EA1DAB0022F007020A33ADEB020D23F0E9
:1013400007037A690DF11808002DADEB030D7960E4
:10135000F368946906AED7F80CA014DD002205F1FD
:10136000FF3C9C44013B13F8011F18B110F801E049
:1013700008F802E01CB154F8211046F82210634529
:1013800002F10102EFD1F0B140F20B2205920022EE
:10139000CDE901220122364B11460092354A6420E4
:1013A000CDE9033243462A46FDF744FBDAF8013023
:1013B000DAF80D10DA789AF800300132092B497BFF
:1013C0001ED0052B3ED094B100240420012140F210
:1013D0002A2C0294CDE90001264C27483346CDE95A
:1013E00003042A46CDF814C06420FDF723FB4946C8
:1013F000F868DD46FFF712FF4437BD46BDE8F08FC1
:101400007B6840F64A30CDE903630091CDE901588D
:101410004FF4F0734FF4487101F072FB40F21A2C54
:101420000420164A1349002304910121CDE9011338
:101430007B6800900392CDF814C02A466420FDF723
:10144000F9FAC0E77B6840F64A30CDE903630091C2
:10145000CDE9015882234FF4487101F051FB40F26D
:10146000262C0420064ADDE7E4AD0100A50C0100AE
:1014700098AE010034AE0100B4AE0100A0AE010090
:10148000ACAE0100A9090100F8B59B0003F10A0404
:1014900024F0070400AF002AADEB040DEC460CDD90
:1014A000BC69ACF10405013C224414F8016F51F809
:1014B0002660944245F8046FF7D11A46614605F05C
:1014C00055FBBD46F8BD00BF10B5D0F80140D0F8BF
:1014D00009204B789169227DE46882B00846009427
:1014E000FFF7D2FF02B010BD70B5D0F80150D0F8B0
:1014F0000940EE6882B04B782A7DE168A0690096C9
:10150000FFF7C2FF287DA269A16802B0BDE8704064
:10151000FFF75EB9D0F809304A7898699200D96827
:1015200005F024BB2DE9F047D0F80160D0F8093070
:10153000747882B06400D0F80D5033B10F46024683
:1015400019683878264BFFF7CFFBB76B95F80DC0BD
:101550008CB34FF04C0938464FF0000809FB047972
:101560000CF01F0C0CF0030E4FEA8E1E4FEA9C0C81
:10157000002101F1100300EB430393F806A0DA7990
:101580000AF03F0A22F0070201314AEA0E0A42EA53
:101590000C02112983F806A0DA71EAD190F84A30DA
:1015A00080F8488023F01F0380F8498080F84A3093
:1015B0004C308145DCD133782A78A9786878CDE938
:1015C0000074FFF725F94FF4D360234600902A46B4
:1015D00031464FF04050FFF7EBFB02B0BDE8F0871B
:1015E000980604602DE9F04FD0F80130D0F80D7066
:1015F0005C785A798BB0660097F80380002A72D025
:10160000D0F80920106A00286DD01A7DD96897F8A3
:1016100010E0E2B14FF04C0ADFF8289101EB020C28
:10162000013811F8013B10F8015FC3F1210393FB6E
:10163000F6F206FB12320AFB029223F0010320337A
:101640001344DA79614565F3C702DA71E9D1002EF6
:101650006AD04C223B490B4602FB061283F825E078
:101660004C339A42FAD101AD28462422002105F0DC
:1016700088FAB8F1010F40D1002E5AD04FF0040C77
:10168000A946DFF8C88006EB0C0A49462E48ACF1A3
:10169000040E002312E0012C05D1032B03F00102FC
:1016A00001DD724507D003EBC30291F800B0825C04
:1016B00042EA0B020A700133082B06D0022CEAD151
:1016C0009C45F0D10133082BF8D10130804501F160
:1016D0000101DED10CF1010CE24509F10909D4D177
:1016E0009DF804100AE001AD28462422002105F0EF
:1016F00048FAB8F1010FBFD0DEB100214FF0000C65
:10170000104C2846002301E010F8011FE2180133B5
:10171000092B1172F8D10CF1010C664504F14C044F
:1017200007DD15F8091FECE73146242201A805F072
:1017300028FA78783A78B978FFF720FC01480BB09E
:10174000BDE8F08F980604609C200020A5200020B2
:101750002DE9F04F83B04C23567800AF750003FBA2
:1017600005F3ADEB030D9046834689461A4668465D
:1017700000217B609A466C4605F003FA002D5BD091
:101780006B4600200DEB0A015A78187002F0EC024B
:1017900042F012025A704C339942F5D1B9F1000F60
:1017A0002EDD00214FF04C0A4FF0010E0BF1FF3CF3
:1017B00007E05369013143EA0B0B8945C2F814B0C5
:1017C0001DDD1CF8013F08EB0302C3F1210092F973
:1017D00015201F280EFA00FB0AFB0242E9DD107EED
:1017E000C3F1010383460EFA03F3C0F3010018436B
:1017F000013160F3010B894582F818B0E1DC8DB14D
:1018000000234FF04C0C6FF05500022E07D10CFB5B
:101810000342D17C507421F001019074D1740133E2
:101820009D42F2DC7A682146054805F09FF904489C
:101830000C37BD46BDE8F08FB9F1000FF2DDB0E71F
:101840009806046070B5D0F8092086B0546A936891
:10185000218851B356689D1E301F383601E034F898
:10186000021F50F8042F0902012A38BF0122B1FBE0
:10187000F2F2B2F5DC7F28BF4FF4DC72864225F825
:10188000022FECD140F29935002202240C480D4978
:10189000CDE90122CDE90310059500941422012120
:1018A0006420FDF7C7F806B070BD4FF480709A1E33
:1018B00003F11C0122F8020F8A42FBD1E2E700BFCC
:1018C00034AE0100F4AD01002DE9F04F95B06F4E3C
:1018D00006AF07F11405DFF8D0C1B9603A6196E8A8
:1018E0000F0085E80F0007F1600307F124047B6314
:1018F00007F10803C5F80CC028462146AB60EEF797
:10190000BFFC96E80F00624E84E80F0007F1080361
:10191000C4E90236204607F13401EEF7B1FCBB689A
:1019200044F00104D3F80160D3F809907078C7F847
:101930000C90D3F80D8045F00105800104F08CFF78
:10194000B8F80E10D9F800301422CDE9004501F0A6
:101950000FF8357DEA46EA1DAB0002F4FC720A334B
:10196000ADEB020D03F4FF63F9680DF11808ADEB60
:10197000030DF268D9E9000306AE7B608C69D7F8E5
:10198000089085B10023013A12F8011F18B110F830
:1019900001C008F803C01CB154F8211046F8231008
:1019A00001339D42F0D100B340F26532059200222E
:1019B0004FF0010B374BCDE90122374A5946CDE9AB
:1019C0000332CDF800B043462A466420FDF732F8D2
:1019D000D9F80130D9F80D10DA7899F800305A4466
:1019E0000A2B497B1DD0062B3DD094B140F28534A3
:1019F000002001214FF0040C05940290264C27484A
:101A00003346CDE903042A46CDE900C16420FDF741
:101A100011F8D546B868FFF715FF3C37BD46BDE85D
:101A2000F08F7B6840F64A30CDE903630091CDE941
:101A300001584FF4F0734FF4487101F061F840F22F
:101A4000753C0420164A144904910021CDE901B1E6
:101A500059467B6800900392CDF814C02A46642052
:101A6000FCF7E8FFC1E77B6840F64A30CDE9036345
:101A70000091CDE9015882234FF4487101F040F8FC
:101A800040F2813C0420074ADDE700BFE4AD0100DD
:101A90006D0D0100C0AE010034AE0100DCAE0100EE
:101AA000C8AE0100D4AE0100F109010010B5D0F8B4
:101AB0000140D0F809200B789169227DE46882B05A
:101AC00008460094FFF7E0FC02B010BD70B5D0F8F6
:101AD0000150D0F80940EE6882B00B782A7DE168A9
:101AE000A0690096FFF7D0FC287DA269A16802B02A
:101AF000BDE87040FEF76CBE4FF0405393F84111C3
:101B0000D0F80930090401F1C041D86801F58431E9
:101B1000502205F02BB800BFD0F809300A78986938
:101B20009200D96805F022B82DE9F0474C2692F8CA
:101B3000018000AF4FEA480406FB04F6ADEB060D4A
:101B4000824689466846324600216D4605F019F8FE
:101B5000002C5ED06B461A200DEB06015A781870E7
:101B600002F0EC0242F002025A704C339942F5D175
:101B700019F0FF012AD00AF1FF304FF04C094FF065
:101B8000010E014405E05369814243EA0C035361AD
:101B90001BD010F8013F93FBF4F204FB12321F2B11
:101BA0000EFA03FC09FB0252EDDD92F818C0203B4F
:101BB000E2460EFA03F3CCF3010C43EA0C0363F3A1
:101BC000010A814282F818A0E3D1F4B12B465521D5
:101BD0002E44B8F1020F05D1DA7C597422F00102CB
:101BE0009974DA744C339E42F3D100264FF04C08BE
:101BF0000A4B08FB065118464C2204F0B7FF034677
:101C00000136B44203F15403F3D10448BD46BDE8A4
